:04000C00CA640000C2
:10001000026500003A65000072650000AA650000F4
:04004800226600002C
:0400540058670000E9
:04007800E26500003D
:0400A0006C68000088
:100400003220EF00C3202000008041001040BA00DD
:100410000160EF00000006000A0D0000416C0000C2
:100420006C20000044650000636F000064650000FC
:1004300072730000206C00006F61000064650000B2
:10044000640A00000D0000003220EF0003232000AA
:10045000008041001040BA000160EF00000006007B
:100460000A0D0000496E0000707500007420000045
:10047000257500003A200000200000003220EF0027
:10048000A3242000008041001040BA000160EF006A
:1004900000000600313000003830000070200000FD
:1004A00028350000392E00003934000029200000D2
:1004B00044650000636F0000646500007220000066
:1004C000436F00006E660000696700002044000072
:1004D0006F6E0000650A00000D0000003220EF0082
:1004E000A3272000008041001040BA000160EF0007
:1004F000000006003130000038300000702000009D
:100500002835000030290000204400006563000009
:100510006F64000065720000204300006F6E0000F1
:100520006669000067200000446F00006E650000EF
:100530000A0D0000000000003220EF00832A200096
:10054000008041001040BA000160EF00000006008A
:1005500031300000383000006920000028350000EC
:10056000392E0000393400002920000044650000C5
:10057000636F00006465000072200000436F00009C
:100580006E66000069670000204400006F6E000086
:10059000650A00000D0000003220EF00832D2000CE
:1005A000008041001040BA000160EF00000006002A
:1005B000313000003830000069200000283500008C
:1005C0003029000020440000656300006F640000D3
:1005D00065720000204300006F6E00006669000035
:1005E00067200000446F00006E6500000A0D0000E7
:1005F000000000003220EF00633020000080410046
:100600001040BA000160EF00000006003732000021
:100610003070000028350000392E00003934000009
:100620002920000044650000636F0000646500003D
:1006300072200000436F00006E66000069670000D2
:10064000204400006F6E0000650A00000D000000ED
:100650003220EF0043332000008041001040BA00F8
:100660000160EF000000060037320000307000002B
:100670002835000030290000204400006563000098
:100680006F64000065720000204300006F6E000080
:100690006669000067200000446F00006E6500007E
:1006A0000A0D0000000000003220EF000336200099
:1006B000008041001040BA000160EF000000060019
:1006C000363400003020000078200000343800006C
:1006D000302800003630000029200000456E000060
:1006E000636F00006465000072200000436F00002B
:1006F0006E66000069670000204400006F6E000015
:10070000650A00000D0000003220EF0003392000D0
:10071000008041001040BA000160EF0000000600B8
:100720003830000030200000782000003630000013
:100730003028000036300000292000004465000009
:10074000636F00006465000072200000436F0000CA
:100750006E66000069670000204400006F6E0000B4
:10076000650A00000D0000003220EF00033C20006D
:10077000008041001040BA000160EF000000060058
:1007800031300000323400002078000020370000B3
:1007900036380000283600003029000020440000D0
:1007A000656300006F640000657200002043000074
:1007B0006F6E00006669000067200000446F000053
:1007C0006E6500000A0D0000000000000000E0005F
:1007D0004220AF0004003700793E0900000000000D
:1007E0000000E900F9FF370000000600C7A2A800DA
:0C07F000000009000000000000000600EE
:10180000B46E0400020000003220EF0003C120008B
:10181000008041001040BA000160EF0000000600A7
:1018200031320000383000002078000020370000FE
:10183000363800002836000030290000204400001F
:10184000656300006F6400006572000020430000C3
:101850006F6E00006669000067200000446F0000A2
:101860006E6500000A0D0000000000003220EF004D
:1018700023C42000008041001040BA000160EF0046
:1018800000000600313200003830000020780000EF
:1018900020310000303200003428000036300000D3
:1018A0002920000044650000636F000064650000AB
:1018B00072200000436F00006E6600006967000040
:1018C000204400006F6E0000650A00000D0000005B
:1018D0003220EF0043C72000008041001040BA00D2
:1018E0000160EF00000006003133000036360000D2
:1018F000207800002037000036380000283600002D
:101900003029000020440000656300006F6400007F
:1019100065720000204300006F6E000066690000E1
:1019200067200000446F00006E6500000A0D000093
:10193000000000003220EF0063CA20000080410058
:101940001040BA000160EF000000060031340000D2
:1019500030300000207800002031000030350000D9
:1019600030280000363000002920000044650000C7
:10197000636F00006465000072200000436F000088
:101980006E66000069670000204400006F6E000072
:10199000650A00000D0000003220EF0083CD20001A
:1019A000008041001040BA000160EF000000060016
:1019B0003136000030300000207800002031000077
:1019C00032300000302800003630000029200000AE
:1019D00044650000636F0000646500007220000031
:1019E000436F00006E66000069670000204400003D
:1019F0006F6E0000650A00000D0000003220EF004D
:101A0000A3D02000008041001040BA000160EF0028
:101A10000000060053440000204E00005453000014
:101A20004320000028200000532D000056690000CC
:101A3000646500006F290000204400006563000019
:101A40006F64000065720000204300006F6E0000AC
:101A50006669000067200000446F00006E650000AA
:101A60000A0D0000000000003220EF0003D4200027
:101A7000008041001040BA000160EF000000060045
:101A80005344000020500000414C00002020000082
:101A9000285300002D56000069640000656F0000A7
:101AA0002920000044650000636F000064650000A9
:101AB00072200000436F00006E660000696700003E
:101AC000204400006F6E0000650A00000D00000059
:101AD0003220EF00E30120008301500005003100B7
:101AE00043D82000008041001040BA000160EF00A0
:101AF0000000060040D82000838141008081410021
:101B00001380BA00000006005344430020206F00F9
:101B10004E546E005343660020286900204367003E
:101B20006F6D2000706F440073696F0074656E0004
:101B30002920650044650A00636F0D00646500009C
:101B4000722000003220EF00C3012000830150000A
:101B500005003100E3DB2000008041001040BA00A6
:101B60000160EF0000000600E0DB200083814100FF
:101B7000808141001380BA000000060053444300F6
:101B800020506F00414C6E00202866002043690001
:101B90006F6D6700706F20007369440074656F009B
:101BA00029206E0044656500636F0A0064650D00BE
:101BB000722000003220EF0063DE20000080410030
:101BC0001040BA000160EF0000000600313900004B
:101BD0003230000020780000203100003230000058
:101BE0003020000028360000304800007A2900002C
:101BF0002D2000004E4F000054200000737500009F
:101C0000707000006F72000074650000640A0000CC
:101C10000D0000003220EF0063E120000080410051
:101C20001040BA000160EF0000000600556E000091
:101C30006B6E00006F7700006E0A00000D00000060
:101C40003220EF00C3E22000008041001040BA00C3
:101C50000160EF00000006000A0D0000456E000064
:101C6000636F000064650000722000006C6F00006C
:101C700061640000656400000A0D000000000000BF
:101C80003220EF00C3E42000008041001040BA0081
:101C90000160EF00000006000A0D00005658000029
:101CA000503A0000200000003220EF0003E6200040
:101CB000008041001040BA000160EF000000060003
:101CC000313000003830000070200000283500005E
:101CD000392E00003934000029200000456E000034
:101CE000636F00006465000072200000436F000015
:101CF0006E66000069670000204400006F6E0000FF
:101D0000650A00000D0000003220EF0003E920000A
:101D1000008041001040BA000160EF0000000600A2
:101D200031300000383000007020000028350000FD
:101D300030290000204500006E6300006F64000041
:101D400065720000204300006F6E000066690000AD
:101D500067200000446F00006E6500000A0D00005F
:101D6000000000003220EF00E3EB20000080410083
:101D70001040BA000160EF000000060031300000A2
:101D8000383000006920000028350000392E00009E
:101D90003934000029200000456E0000636F000008
:101DA0006465000072200000436F00006E66000052
:101DB00069670000204400006F6E0000650A0000A3
:101DC0000D0000003220EF00E3EE20000080410013
:101DD0001040BA000160EF00000006003130000042
:101DE000383000006920000028350000302900004C
:101DF000204500006E6300006F6400006572000003
:101E0000204300006F6E000066690000672000003C
:101E1000446F00006E6500000A0D00000000000025
:101E20003220EF00C3F12000008041001040BA00D2
:101E30000160EF0000000600373200003070000043
:101E400028350000392E0000393400002920000018
:101E5000456E0000636F00006465000072200000A2
:101E6000436F00006E6600006967000020440000B8
:101E70006F6E0000650A00000D0000003220EF00C8
:101E8000A3F42000008041001040BA000160EF0080
:101E900000000600373200003070000028350000D6
:101EA00030290000204500006E6300006F640000D0
:101EB00065720000204300006F6E0000666900003C
:101EC00067200000446F00006E6500000A0D0000EE
:101ED000000000003220EF0063F720000080410086
:101EE0001040BA000160EF0000000600383000002A
:101EF000302000007820000036300000302800003C
:101F00003630000029200000456E0000636F00009D
:101F10006465000072200000436F00006E660000E0
:101F200069670000204400006F6E0000650A000031
:101F30000D0000003220EF0063FA20000080410015
:101F40001040BA000160EF000000060031300000D0
:101F500032340000207800002037000036380000BE
:101F60002836000030290000204500006E63000084
:101F70006F64000065720000204300006F6E000077
:101F80006669000067200000446F00006E65000075
:101F90000A0D0000000000003220EF0083FD200049
:101FA000008041001040BA000160EF000000060010
:101FB0003132000038300000207800002037000067
:101FC0003638000028360000302900002045000087
:101FD0006E6300006F640000657200002043000023
:101FE0006F6E00006669000067200000446F00000B
:101FF0006E6500000A0D0000000000003220EF00B6
:10200000A3002100008041001040BA000160EF00F1
:102010000000060031320000383000002078000057
:10202000203100003032000034280000363000003B
:1020300029200000456E0000636F00006465000009
:1020400072200000436F00006E66000069670000A8
:10205000204400006F6E0000650A00000D000000C3
:102060003220EF00C3032100008041001040BA007D
:102070000160EF000000060031330000363600003A
:102080002078000020370000363800002836000095
:1020900030290000204500006E6300006F640000DE
:1020A00065720000204300006F6E0000666900004A
:1020B00067200000446F00006E6500000A0D0000FC
:1020C000000000003220EF00E30621000080410004
:1020D0001040BA000160EF0000000600313400003B
:1020E0003030000020780000203100003035000042
:1020F000302800003630000029200000456E000026
:10210000636F00006465000072200000436F0000F0
:102110006E66000069670000204400006F6E0000DA
:10212000650A00000D0000003220EF00030A2100C4
:10213000008041001040BA000160EF00000006007E
:1021400031360000303000002078000020310000DF
:102150003230000030280000363000002920000016
:10216000456E0000636F000064650000722000008F
:10217000436F00006E6600006967000020440000A5
:102180006F6E0000650A00000D0000003220EF00B5
:10219000230D2100008041001040BA000160EF00D3
:1021A00000000600313900003230000020780000C5
:1021B00020310000323000003028000036300000AE
:1021C00029200000456E0000636F00006465000078
:1021D00072200000436F00006E6600006967000017
:1021E000204400006F6E0000650A00000D00000032
:1021F0003220EF00E3012000830150000500310090
:1022000043112100008041001040BA000160EF003E
:1022100000000600401121008381410080814100BF
:102220001380BA000000060053444300202D6F00C5
:1022300020376E0032306600207869002034670055
:1022400038302000202844004E546F0053436E0065
:1022500029206500456E0A00636F0D00646500006B
:10226000722000003220EF00E313210000804100C3
:102270001040BA000160EF00000006005344000067
:10228000203700003638000020780000203500009C
:102290003736000020280000504100004C29000083
:1022A000204500006E6300006F640000657200004E
:1022B000204300006F6E0000666900006720000088
:1022C000446F00006E6500000A0D00000000000071
:1022D0003220EF000302200083015000050031008E
:1022E00043182100008041001040BA000160EF0057
:1022F00000000600401821008381410080814100D8
:102300001380BA000000060053442000202D430033
:1023100020286F0034386E0030696600207969002B
:10232000506267005072200029204400284E6F0040
:1023300054536E004329650020450A006E630D006A
:102340006F640000657200003220EF00E30120009E
:102350008301500005003100031C21000080410072
:102360001040BA000160EF0000000600001C2100D0
:1023700083814100808141001380BA000000060083
:102380005344430020286F0035376E0036696600DD
:1023900020796900506267005072200029204400B3
:1023A00028506F00414C6E0029206500456E0A00E0
:1023B000636F0D0064650000722000003220EF00A2
:1023C000A31E2100008041001040BA000160EF0010
:1023D000000006000A0D00005658000050280000BA
:1023E00072770000293A0000000000003220EF0060
:1023F00023202100008041001040BA000160EF005E
:10240000000006000A0D0000565800005028000089
:10241000772900003A200000000000003220EF0081
:10242000A3212100008041001040BA000160EF00AC
:10243000000006000A0D0000565800005028000059
:10244000722900003A200000000000003220EF0056
:1024500023232100008041001040BA000160EF00FA
:10246000000006005772000069740000652000003B
:10247000254C0000580A00000D0000003220EF003B
:10248000A3242100008041001040BA000160EF0049
:10249000000006005772000069740000652000000B
:1024A000254C0000582C00002052000065610000FF
:1024B00064200000254C0000580A00000D000000B8
:1024C0003220EF00C3262100008041001040BA00F6
:1024D0000160EF00000006004D64000000000000F5
:1024E0003220EF00C3272100008041001040BA00D5
:1024F0000160EF00000006004C67000000000000D3
:102500003220EF00C3282100008041001040BA00B3
:102510000160EF0000000600536D000000000000A5
:102520003220EF00C3292100008041001040BA0092
:102530000160EF000000060055520000000000009E
:102540003220EF00C32A2100008041001040BA0071
:102550000160EF00000006004C5200000000000087
:102560003220EF00C32B2100008041001040BA0050
:102570000160EF00000006004C4D0000000000006C
:102580003220EF00C32C2100008041001040BA002F
:102590000160EF00000006004C4C0000000000004D
:1025A0003220EF00C32D2100008041001040BA000E
:1025B0000160EF0000000600554C00000000000024
:1025C0003220EF00C32E2100008041001040BA00ED
:1025D0000160EF000000060050490000503A000082
:1025E00020250000732C00004C2000002573000003
:1025F000000000003220EF000303200083015000A0
:102600000500310063312100008041001040BA0014
:102610000160EF000000060060312100838141006D
:10262000808141001380BA00000006000D0A2C00D2
:102630000D0A450052656E006164640044754300F4
:10264000616C68005561610072747200506F3D00EA
:10265000727425002C5032006F727800743D2C008B
:10266000257557002C426100756669006665740027
:10267000723D3D00254C2500582C6C0053697500B7
:102680007A650A003D250D00327800003220EF0007
:1026900023352100008041001040BA000160EF00A6
:1026A000000006000D0A0000526500006164000091
:1026B00044750000616C00005561000072740000F8
:1026C000506F00007274000028250000752900007A
:1026D0003A200000000000003220EF008337210084
:1026E000008041001040BA000160EF0000000600C9
:1026F0002D200000546900006D6500006F7500001A
:1027000074280000256C0000782900000A0D0000E4
:10271000000000003220EF006339210000804100FA
:102720001040BA000160EF00000006002D200000FC
:1027300045720000726F000072280000256C0000D6
:10274000782900000A0D0000000000003220EF0090
:10275000E30120008301500005003100233C2100EB
:10276000008041001040BA000160EF000000060048
:10277000203C210083814100808141001380BA0008
:10278000000006000D0A780028552C00322944006C
:1027900045726100726F7400725B610042493A00D9
:1027A0002C202500504532002C2078004645290079
:1027B0005D280A004C530D00523A000025320000FB
:1027C0003220EF00C33E2100008041001040BA00DB
:1027D0000160EF00000006000D0A0000285500000F
:1027E0003229000045720000726F0000725B000029
:1027F0004F76000065720000727500006E5D00008B
:10280000284C0000535200003A25000032780000A6
:102810002C44000061740000613A00002532000081
:10282000782900000A0D0000000000003220EF00AF
:10283000E301200083015000050031002343210003
:10284000008041001040BA000160EF000000060067
:102850002043210083814100808141001380BA0020
:10286000000006000D0A780028552C00312944008C
:1028700045726100726F7400725B610042493A00F8
:102880002C202500504532002C2078004645290098
:102890005D280A004C530D00523A0000253200001A
:1028A0003220EF00C3452100008041001040BA00F3
:1028B0000160EF00000006000D0A0000285500002E
:1028C0003129000045720000726F0000725B000049
:1028D0004F76000065720000727500006E5D0000AA
:1028E000284C0000535200003A25000032780000C6
:1028F0002C44000061740000613A000025320000A1
:10290000782900000A0D0000000000003220EF00CE
:1029100023492100008041001040BA000160EF000F
:102920000000060045720000726F0000723A00005D
:10293000204900006E760000616C000069640000B0
:10294000204D0000657300007361000067650000A2
:102950002825000032780000290A00000D00000040
:102960003220EF00C34B2100008041001040BA002C
:102970000160EF00000006000A0D00004275000033
:102980006666000065720000204F0000766500005A
:10299000724C00006170000020450000727200005F
:1029A0006F7200000D0A0000000000003220EF00EE
:1029B000234E2100008041001040BA000160EF006A
:1029C000000006002050000043430000205000009B
:1029D000726F000067720000616D0000204D000002
:1029E0006F64000065200000200000003220EF002E
:1029F00023502100008041001040BA000160EF0028
:102A00000000060020200000202000002020000000
:102A100020200000202000002020000020200000B6
:102A20002020000020200000200000003220EF00C5
:102A300023522100008041001040BA000160EF00E5
:102A400000000600202000005570000064610000B6
:102A5000746900006E67000020430000616D000093
:102A60006572000061200000200000003220EF00AD
:102A700023542100008041001040BA000160EF00A3
:102A800000000600507200006573000065740000CD
:102A90002025000075200000506100006E610000DC
:102AA000736F00006E69000063200000436F000038
:102AB0006D7000006C650000746500000A0D000078
:102AC000000000003220EF00E356210000804100AA
:102AD0001040BA000160EF00000006002050000026
:102AE000726500007365000074200000253300004B
:102AF000750A00000D0000003220EF00835821000D
:102B0000008041001040BA000160EF0000000600A4
:102B100050720000657300006574000020250000FD
:102B200075200000536F00006E7900002F430000F5
:102B3000616E00006F6E0000204300006F6D0000AA
:102B4000706C000065740000650A00000D00000054
:102B50003220EF00435B2100008041001040BA00AA
:102B60000160EF0000000600507200006573000075
:102B700065740000202500007520000054720000DC
:102B8000616E000073690000746900006F6E0000E0
:102B90000A0D0000000000003220EF00835D2100DC
:102BA000008041001040BA000160EF000000060004
:102BB000507200006573000065740000202500005D
:102BC0007520000054720000616E000073690000FF
:102BD000746900006F6E000028730000290A00006D
:102BE0000D0000003220EF00E35F21000080410073
:102BF0001040BA000160EF000000060050720000B3
:102C00006573000065740000202500007520000039
:102C100054720000616E0000736900007469000066
:102C20006F6E000028670000290A00000D000000F8
:102C30003220EF0043622100008041001040BA00C2
:102C40000160EF00000006002050000072650000E7
:102C5000736500007420000025330000752000001B
:102C60004C6F00006164000065640000000000001B
:102C70003220EF0043642100008041001040BA0080
:102C80000160EF00000006002050000043430000F8
:102C90002050000072650000736500007420000081
:102CA00025330000752000004C6F000061640000B7
:102CB00065640000000000003220EF008366210000
:102CC000008041001040BA000160EF0000000600E3
:102CD00020200000202000002020000020200000F4
:102CE00020200000202000002020000020200000E4
:102CF00020200000000000003220EF008368210047
:102D0000008041001040BA000160EF0000000600A2
:102D1000536500006C200000495200002D50000057
:102D2000726500007365000074200000312000000F
:102D300020200000000000003220EF00836A210004
:102D4000008041001040BA000160EF000000060062
:102D5000536500006C200000495200002D50000017
:102D600072650000736500007420000030200000D0
:102D700020200000000000003220EF00836C2100C2
:102D8000008041001040BA000160EF000000060022
:102D9000536500006C200000495200002D500000D7
:102DA000726500007365000074200000312500008A
:102DB00063200000000000003220EF00836E21003D
:102DC000008041001040BA000160EF0000000600E2
:102DD000536500006C200000495200002D50000097
:102DE000726500007365000074200000302500004B
:102DF00063200000000000003220EF0083702100FB
:102E0000008041001040BA000160EF0000000600A1
:102E1000536500006C200000495200002D50000056
:102E20007265000073650000742000002533000007
:102E300075200000000000003220EF0083722100A6
:102E4000008041001040BA000160EF000000060061
:102E5000536500006C200000495200002D50000016
:102E600072650000736500007420000025320000C8
:102E700075200000000000003220EF008374210064
:102E8000008041001040BA000160EF000000060021
:102E90000A0D00005265000061640000204300003C
:102EA0006F6E00006669000067280000257500004D
:102EB000293A0000200000003220EF008376210034
:102EC000008041001040BA000160EF0000000600E1
:102ED0002043000068650000636B0000737500000C
:102EE0006D3D000025320000782000005361000095
:102EF0006D6500000A0D0000000000003220EF00A8
:102F0000E30120008301500005003100A379210076
:102F1000008041001040BA000160EF000000060090
:102F2000A079210083814100808141001380BA0093
:102F3000000006002043200068654400636B6900C0
:102F4000737566006D286600253265007829720069
:102F50003D436500616C6E00637574006C610A002E
:102F600074650D0064280A0025320D0078290000E0
:102F70003220EF00437C2100008041001040BA0065
:102F80000160EF0000000600436800006563000078
:102F90006B730000756D0000205200006561000039
:102FA0006420000025320000782C0000204300003F
:102FB000616C0000637500006C61000074650000C6
:102FC0006420000025320000780A00000D00000097
:102FD0003220EF00437F2100008041001040BA0002
:102FE0000160EF0000000600436F00006E66000005
:102FF00069670000205300006176000065640000EE
:103000000A0D0000000000003220EF0003812100C3
:10301000008041001040BA000160EF00000006008F
:10302000526500006164000020450000455000002A
:10303000726F00006D20000046610000696C0000A6
:10304000656400002D200000526500006C6F0000D8
:1030500061640000204400006566000061750000A6
:103060006C740000730A00000D0000003220EF00B5
:10307000C301200083015000050031002385210099
:10308000008041001040BA000160EF00000006001F
:103090002085210083814100808141001380BA0096
:1030A00000000600284450006F53720061766F00E4
:1030B00065446D0065662000617546006C746100B2
:1030C0007329690053616C0076656500436F640085
:1030D0006E660A0069670D00454500003220EF006A
:1030E000A3872100008041001040BA000160EF007A
:1030F000000006004C6F000063200000254C00001B
:10310000782C0000205000007265000073650000FC
:1031100074200000256400000A0D0000000000007B
:103120003220EF000302200083015000050031002F
:10313000C38A2100008041001040BA000160EF0006
:1031400000000600C08A2100838141008081410087
:103150001380BA000000060050494200502047008A
:10316000536128007665250020507500726529009E
:103170007365200074204600257547002053280001
:10318000656C2500656375007420290045720A008E
:10319000726F0D00722000003220EF00838D21003D
:1031A000008041001040BA000160EF0000000600FE
:1031B00020500000495000002053000061760000BC
:1031C0006520000025750000204500007272000097
:1031D0006F720000000000003220EF0003022000A8
:1031E00083015000050031008390210000804100E0
:1031F0001040BA000160EF0000000600809021003E
:1032000083814100808141001380BA0000000600E4
:10321000537475006F7229006520200050495000DA
:1032200050206F005072720065737400657428003E
:103230002825250075297500204E29006F200A00D9
:1032400043610D006D6500007261000028250000DB
:103250003220EF00030220008301500005003100FE
:1032600043942100008041001040BA000160EF004B
:1032700000000600409421008381410080814100CC
:103280001380BA000000060050494400502061003D
:10329000537474006F7261006520200050725000FA
:1032A00065736F0065747200282574007529280005
:1032B00020432500616D75006572290061280A00B0
:1032C00025750D00292000003220EF00C3012000E9
:1032D0008301500005003100039821000080410067
:1032E0001040BA000160EF000000060000982100C5
:1032F00083814100808141001380BA0000000600F4
:103300005049280050202500537475006F72290021
:1033100065202000507246006573470065742800E0
:10332000202525007520750045722900726F0A005E
:1033300072200D00424700003220EF00839A2100E6
:10334000008041001040BA000160EF00000006005C
:10335000205000004950000020530000746F00000E
:1033600072650000202500007520000045720000F5
:10337000726F0000720000003220EF00839C210079
:10338000008041001040BA000160EF00000006001C
:103390005049000050200000536100007665000095
:1033A00020420000472000005072000065730000BA
:1033B0006574000020250000750A00000D00000063
:1033C0003220EF00C39E2100008041001040BA006F
:1033D0000160EF000000060050490000502000008E
:1033E0005361000076650000205000007265000007
:1033F0007365000074200000257500002045000062
:10340000727200006F720000204200004728000026
:1034100025750000290A00000D0000003220EF0091
:10342000A3A12100008041001040BA000160EF001C
:1034300000000600504900005020000053610000C9
:103440007665000020460000472000005072000012
:10345000657300006574000020250000750A0000F7
:103460000D0000003220EF00E3A3210000804100A6
:103470001040BA000160EF00000006005049000053
:1034800050200000536100007665000020500000CD
:10349000726500007365000074200000257500004F
:1034A00020450000727200006F720000204600008C
:1034B0004728000025750000290A00000D000000C3
:1034C0003220EF00C3A62100008041001040BA0066
:1034D0000160EF000000060050490000502000008D
:1034E00050720000657300006574000073200000D6
:1034F000467500006C6C000028250000752900004E
:103500000A0D0000000000003220EF0003A9210096
:10351000008041001040BA000160EF00000006008A
:103520004C6F000063200000254C0000782C000048
:10353000205000004950000020500000726500003B
:103540007365000074200000256400000A0D00006F
:10355000000000003220EF0063AB2100008041003A
:103560001040BA000160EF00000006005265000044
:1035700061640000204C00006F6300002025000003
:103580004C7800002C200000436100006D650000B5
:1035900072610000202500006420000050430000FC
:1035A0004320000050720000657300006574000045
:1035B00020250000640A00000D0000003220EF000A
:1035C000A3AE2100008041001040BA000160EF006E
:1035D000000006005361000076650000204C0000EA
:1035E0006F630000202500004C7800002C200000B4
:1035F000436100006D65000072610000202500003D
:10360000642000005043000043200000507200007E
:10361000657300006574000020250000640A000046
:103620000D0000003220EF00E3B1210000804100D6
:103630001040BA000160EF0000000600536F000068
:103640006E79000020450000564900002D4400001E
:103650003330000020200000202000002020000047
:10366000200000003220EF00E3B321000080410081
:103670001040BA000160EF0000000600536F000028
:103680006E79000020450000564900002D440000DE
:10369000333000002F4400003331000020200000B0
:1036A000200000003220EF00E3B52100008041003F
:1036B0001040BA000160EF000000060056610000F3
:1036C00064640000696F0000204100006464000031
:1036D0002D6100002D430000616D000020200000DE
:1036E000200000003220EF00E3B7210000804100FD
:1036F0001040BA000160EF0000000600536F0000A8
:103700006E79000020450000564900002D4400005D
:103710003130000030200000202000002020000078
:10372000200000003220EF00E3B9210000804100BA
:103730001040BA000160EF00000006005641000092
:1037400044440000494F000020480000442D000080
:103750003138000020200000202000002020000040
:10376000200000003220EF00E3BB21000080410078
:103770001040BA000160EF0000000600536F000027
:103780006E79000020450000564900002D440000DD
:103790003730000020200000202000002020000002
:1037A000200000003220EF00E3BD21000080410036
:1037B0001040BA000160EF0000000600536F0000E7
:1037C0006E79000020420000524300002D330000BB
:1037D00030300000202000002020000020200000C9
:1037E000200000003220EF00E3BF210000804100F4
:1037F0001040BA000160EF0000000600536F0000A7
:103800006E79000020420000524300002D48000065
:103810003730000030200000202000002020000071
:10382000200000003220EF00E3C1210000804100B1
:103830001040BA000160EF0000000600536F000066
:103840006E79000020420000524300002D5A000013
:103850003730000030200000202000002020000031
:10386000200000003220EF00E3C32100008041006F
:103870001040BA000160EF0000000600536F000026
:103880006E79000020420000524300002D5A0000D3
:1038900033330000302000002020000020200000F2
:1038A000200000003220EF00E3C52100008041002D
:1038B0001040BA000160EF0000000600536F0000E6
:1038C0006E79000020450000564900002D48000098
:1038D00044310000202000002020000020200000B3
:1038E000200000003220EF00E3C7210000804100EB
:1038F0001040BA000160EF000000060050610000B7
:103900006E610000736F00006E69000063200000AC
:10391000415700002D4800004531000030300000C4
:10392000200000003220EF00E3C9210000804100A8
:103930001040BA000160EF0000000600436500007F
:10394000696C0000696E0000675600004945000080
:103950005720000020200000202000002020000030
:10396000200000003220EF00E3CB21000080410066
:103970001040BA000160EF00000006004361000043
:103980006E6E00006F6E000020560000432D000098
:1039900043350000306900002F7200002020000035
:1039A000200000003220EF00E3CD21000080410024
:1039B0001040BA000160EF00000006004361000003
:1039C0006E6E00006F6E000020420000552D00005A
:1039D0003435000048200000202000002020000096
:1039E000200000003220EF00E3CF210000804100E2
:1039F0001040BA000160EF000000060043610000C3
:103A00006E6E00006F6E000020420000552D000019
:103A10003530000048200000202000002020000059
:103A2000200000003220EF00E3D12100008041009F
:103A30001040BA000160EF0000000600556E000063
:103A40006B6E00006F7700006E2000004361000085
:103A50006D65000072610000202000002020000041
:103A6000200000003220EF00E3D32100008041005D
:103A70001040BA000160EF000000060000000000E6
:103A80003220EF00C3D42100008041001040BA0072
:103A90000160EF0000000600486F00007374000032
:103AA0002053000065720000696100006C20000076
:103AB000496E000070750000743A00002045000057
:103AC0006E610000626C0000656400000000000090
:103AD0003220EF0043D72100008041001040BA009F
:103AE0000160EF0000000600486F000073740000E2
:103AF0002053000065720000696100006C20000026
:103B0000496E000070750000743A00002044000007
:103B100069730000616200006C65000064000000D1
:103B20003220EF00C3D92100008041001040BA00CC
:103B30000160EF000000060053650000726900009C
:103B4000616C000020450000636800006F3A0000CF
:103B5000204500006E610000626C0000656400009A
:103B6000000000003220EF00E3DB21000080410074
:103B70001040BA000160EF0000000600536500002D
:103B800072690000616C000020450000636800005D
:103B90006F3A000020440000697300006162000079
:103BA0006C650000640000003220EF0003DE21009D
:103BB000008041001040BA000160EF0000000600E4
:103BC0005365000072690000616C0000204900002C
:103BD0006E6600006F3A0000204F00006E0000008B
:103BE0003220EF00C3DF2100008041001040BA0006
:103BF0000160EF00000006005365000072690000DC
:103C0000616C0000204900006E6600006F3A000001
:103C1000204F000066660000000000003220EF0028
:103C2000A3E12100008041001040BA000160EF00D4
:103C300000000600546100006C6C00007920000058
:103C40004C650000766500006C3A000020410000E1
:103C50006374000069760000652000004C6F00006E
:103C6000770000003220EF00E3E3210000804100F4
:103C70001040BA000160EF0000000600546100002F
:103C80006C6C0000792000004C6500007665000037
:103C90006C3A000020410000637400006976000067
:103CA000652000004869000067680000000000000F
:103CB0003220EF0043E62100008041001040BA00AE
:103CC0000160EF0000000600446900006167000029
:103CD0006E6F00007374000069630000204D0000E7
:103CE0006F640000653A0000204F00006E00000085
:103CF0003220EF0043E82100008041001040BA006C
:103D00000160EF00000006004469000061670000E8
:103D10006E6F00007374000069630000204D0000A6
:103D20006F640000653A0000204F000066660000E6
:103D3000000000003220EF0063EA21000080410013
:103D40001040BA000160EF0000000600536500005B
:103D500072690000616C000020440000696100008D
:103D6000672000004D6F0000646500003A200000ED
:103D70004F6E0000000000003220EF0083EC2100B5
:103D8000008041001040BA000160EF000000060012
:103D90005365000072690000616C0000204400005F
:103DA00069610000672000004D6F0000646500003D
:103DB0003A2000004F660000660000003220EF004D
:103DC000A3EE2100008041001040BA000160EF0026
:103DD000000006004578000074650000726E000067
:103DE000616C0000205400007269000067670000E9
:103DF0006572000073200000496E000069740000C5
:103E0000696100006C6900007A65000064000000D0
:103E10003220EF0043F12100008041001040BA0041
:103E20000160EF00000006004578000074650000A6
:103E3000726E0000616C0000205400007269000086
:103E40006767000065720000732000006E6F00005D
:103E500074200000496E0000697400006961000070
:103E60006C6900007A650000640000003220EF00F9
:103E700023F42100008041001040BA000160EF00EF
:103E80000000060054720000616E000073690000BB
:103E9000746900006F6E0000204D00006F64000028
:103EA000653A0000204D0000697800000000000025
:103EB0003220EF0043F62100008041001040BA009C
:103EC0000160EF000000060054720000616E000007
:103ED00073690000746900006F6E0000204D0000DF
:103EE0006F640000653A0000204300007574000014
:103EF000000000003220EF0063F821000080410044
:103F00001040BA000160EF0000000600547200008B
:103F1000616E000073690000746900006F6E00003C
:103F2000204D00006F640000653A0000205700003B
:103F300069700000650000003220EF0083FA210064
:103F4000008041001040BA000160EF000000060050
:103F5000576900007065000020520000696700008A
:103F600068740000202D00003E2000004C65000019
:103F700066740000000000003220EF0083FC210086
:103F8000008041001040BA000160EF000000060010
:103F90005769000070650000204C00006566000055
:103FA000742000002D3E00002052000069670000D0
:103FB00068740000000000003220EF0083FE210042
:103FC000008041001040BA000160EF0000000600D0
:103FD0002020000057690000706500002054000098
:103FE0006F700000202D00003E200000426F000096
:103FF00074200000000000003220EF008300220047
:10400000008041001040BA000160EF00000006008F
:104010002020000057690000706500002042000069
:104020006F740000202D00003E200000546F00003F
:1040300070200000000000003220EF008302220008
:10404000008041001040BA000160EF00000006004F
:10405000202000002057000069700000652000004B
:104060004C520000202D00003E200000554C000066
:1040700020200000000000003220EF008304220016
:10408000008041001040BA000160EF00000006000F
:10409000202000002057000069700000652000000B
:1040A0004C4C0000202D00003E2000005552000026
:1040B00020200000000000003220EF0083062200D4
:1040C000008041001040BA000160EF0000000600CF
:1040D00020200000205700006970000065200000CB
:1040E00055520000202D00003E2000004C4C0000E6
:1040F00020200000000000003220EF008308220092
:10410000008041001040BA000160EF00000006008E
:10411000202000002057000069700000652000008A
:10412000554C0000202D00003E2000004C520000A5
:1041300020200000000000003220EF00830A22004F
:10414000008041001040BA000160EF00000006004E
:104150002020000057690000706500002054000016
:104160006F200000436500006E740000657200005F
:1041700020200000000000003220EF00830C22000D
:10418000008041001040BA000160EF00000006000E
:104190005769000070650000204C0000203E0000C0
:1041A000436500006E740000657200003C20000052
:1041B00052200000000000003220EF00830E220099
:1041C000008041001040BA000160EF0000000600CE
:1041D000576900007065000020540000203E000078
:1041E000436500006E740000657200003C20000012
:1041F00042200000000000003220EF008310220067
:10420000008041001040BA000160EF00000006008D
:10421000202000002020000020200000204E000070
:104220006F6E0000652000002020000020200000AC
:1042300020200000000000003220EF008312220046
:10424000008041001040BA000160EF00000006004D
:104250004D65000064690000756D000000000000FD
:104260003220EF00C3132200008041001040BA004A
:104270000160EF00000006004C6100007267000062
:10428000650000003220EF00E314220000804100AE
:104290001040BA000160EF0000000600536D0000FE
:1042A000616C00006C0000003220EF000316220059
:1042B000008041001040BA000160EF0000000600DD
:1042C0005570000070650000722000005269000007
:1042D00067680000742D00002573000000000000D6
:1042E0003220EF00C3172200008041001040BA00C6
:1042F0000160EF00000006004C6F000077650000D1
:10430000722000005269000067680000742D0000F0
:1043100025730000000000003220EF008319220006
:10432000008041001040BA000160EF00000006006C
:104330004C6F000077650000722000004D6900009E
:10434000646400006C6500002D250000730000000F
:104350003220EF00431B2200008041001040BA00D1
:104360000160EF00000006004C6F00007765000060
:10437000722000004C650000667400002D250000CE
:10438000730000003220EF00E31C22000080410097
:104390001040BA000160EF000000060055700000F8
:1043A00070650000722000004C650000667400001B
:1043B0002D250000730000003220EF00831E220034
:1043C000008041001040BA000160EF0000000600CC
:1043D000205000004950000020530000697A00007E
:1043E000653A0000204D000065640000697500001A
:1043F0006D200000000000003220EF00832022002A
:10440000008041001040BA000160EF00000006008B
:10441000205000004950000020530000697A00003D
:10442000653A0000204C00006172000067650000E2
:1044300020200000000000003220EF008322220034
:10444000008041001040BA000160EF00000006004B
:10445000205000004950000020530000697A0000FD
:10446000653A0000205300006D6100006C6C000094
:1044700020200000000000003220EF0083242200F2
:10448000008041001040BA000160EF00000006000B
:104490002050000049500000204C00006F630000D5
:1044A00061740000696F00006E200000313A000066
:1044B00055520000000000003220EF008326220049
:1044C000008041001040BA000160EF0000000600CB
:1044D0002050000049500000204C00006F63000095
:1044E00061740000696F00006E200000323A000025
:1044F0004C520000000000003220EF008328220010
:10450000008041001040BA000160EF00000006008A
:104510002050000049500000204C00006F63000054
:1045200061740000696F00006E200000333A0000E3
:104530004C4D0000000000003220EF00832A2200D2
:10454000008041001040BA000160EF00000006004A
:104550002050000049500000204C00006F63000014
:1045600061740000696F00006E200000343A0000A2
:104570004C4C0000000000003220EF00832C220091
:10458000008041001040BA000160EF00000006000A
:104590002050000049500000204C00006F630000D4
:1045A00061740000696F00006E200000353A000061
:1045B000554C0000000000003220EF00832E220046
:1045C000008041001040BA000160EF0000000600CA
:1045D000466F000072650000677200006F75000092
:1045E0006E640000000000003220EF000330220063
:1045F000008041001040BA000160EF00000006009A
:1046000042610000636B0000677200006F7500007C
:104610006E640000000000003220EF0083312200B1
:10462000008041001040BA000160EF000000060069
:104630005061000073730000204F00006E200000E6
:104640005374000061740000757300003A2000008C
:1046500041630000746900007665000000000000FE
:104660003220EF00C3332200008041001040BA0026
:104670000160EF000000060050610000737300004D
:10468000204F00006E200000537400006174000091
:10469000757300003A200000496E0000616300005D
:1046A0007469000076650000000000003220EF0011
:1046B00023362200008041001040BA000160EF0064
:1046C00000000600506100007373000020520000DB
:1046D00065730000706F00006E73000065200000BD
:1046E0005374000061740000757300003A200000EC
:1046F000506500006E640000696E000067000000F5
:104700003220EF00C3382200008041001040BA0080
:104710000160EF00000006005061000073730000AC
:104720002052000065730000706F00006E7300007F
:104730006520000053740000617400007573000070
:104740003A200000496400006C6500000000000091
:104750003220EF00433B2200008041001040BA00AD
:104760000160EF0000000600506100006E2F0000A5
:10477000546900006C740000205300007461000054
:1047800074750000733A000020410000637400005B
:1047900069760000650000003220EF00833D2200B2
:1047A000008041001040BA000160EF0000000600E8
:1047B000506100006E2F0000546900006C7400000E
:1047C000205300007461000074750000733A00000B
:1047D00020490000646C0000650000003220EF00FA
:1047E000A33F2200008041001040BA000160EF00AA
:1047F000000006005A6F00006F6D0000205300009B
:104800007461000074750000733A000020410000DC
:104810006374000069760000650000003220EF003C
:10482000A3412200008041001040BA000160EF0067
:10483000000006005A6F00006F6D0000205300005A
:104840007461000074750000733A00002049000094
:10485000646C0000650000003220EF0083432200FA
:10486000008041001040BA000160EF000000060027
:10487000505400005A200000536500006E64000090
:104880002053000074610000746500003A200000AD
:10489000506500006E640000696E00006700000053
:1048A0003220EF00C3452200008041001040BA00D2
:1048B0000160EF0000000600505400005A20000084
:1048C000536500006E640000205300007461000016
:1048D000746500003A200000496400006C65000027
:1048E000000000003220EF00E3472200008041007A
:1048F0001040BA000160EF00000006005072000096
:10490000657300006574000020500000726F0000A5
:1049100067720000616D0000204D00006F640000B0
:10492000653A0000204F00006E0000003220EF00CA
:10493000234A2200008041001040BA000160EF00CD
:1049400000000600507200006573000065740000EE
:1049500020500000726F000067720000616D00005F
:10496000204D00006F640000653A0000204F0000F9
:1049700066660000000000003220EF00834C220039
:10498000008041001040BA000160EF000000060006
:104990004844000020310000303800003070000032
:1049A00020350000392E000039340000487A00001C
:1049B000200000003220EF00634E22000080410002
:1049C0001040BA000160EF000000060048440000FB
:1049D0002031000030380000307000002035000029
:1049E000304800007A200000202000002000000055
:1049F0003220EF0043502200008041001040BA00F6
:104A00000160EF0000000600484400002031000073
:104A1000303800003069000020350000392E0000D9
:104A200039340000487A0000200000003220EF00F6
:104A300023522200008041001040BA000160EF00C4
:104A4000000006004844000020310000303800001B
:104A50003069000020350000304800007A20000056
:104A600020200000200000003220EF00035422002C
:104A7000008041001040BA000160EF000000060015
:104A80004844000020200000373200003070000051
:104A900020350000392E000039340000487A00002B
:104AA000200000003220EF00E3552200008041008A
:104AB0001040BA000160EF0000000600484400000A
:104AC0002020000037320000307000002035000048
:104AD000304800007A200000202000002000000064
:104AE0003220EF00C3572200008041001040BA007E
:104AF0000160EF0000000600485600002020000082
:104B000036340000307800002034000038300000D7
:104B100020360000304800007A0000003220EF000C
:104B2000A3592200008041001040BA000160EF004C
:104B30000000060048560000202000003830000029
:104B400030780000203600003030000020360000B1
:104B5000304800007A0000003220EF00835B220022
:104B6000008041001040BA000160EF000000060024
:104B70004856000020310000303200003478000038
:104B80002037000036380000203600003048000092
:104B90007A0000003220EF00635D220000804100B7
:104BA0001040BA000160EF00000006004856000007
:104BB000203100003238000030780000203700003B
:104BC0003638000020360000304800007A0000002F
:104BD0003220EF00435F2200008041001040BA0005
:104BE0000160EF0000000600485600002031000080
:104BF00032380000307800003130000032340000DC
:104C000020360000304800007A0000003220EF001B
:104C100023612200008041001040BA000160EF00D3
:104C20000000060048560000203100003336000026
:104C300036780000203700003638000020360000AB
:104C4000304800007A0000003220EF0003632200A9
:104C5000008041001040BA000160EF000000060033
:104C60004856000020310000343000003078000049
:104C700031300000353000002036000030480000A0
:104C80007A0000003220EF00E3642200008041003F
:104C90001040BA000160EF00000006004856000016
:104CA0002031000036300000307800003132000042
:104CB0003030000020360000304800007A0000004C
:104CC0003220EF00C3662200008041001040BA008D
:104CD0000160EF000000060048560000203100008F
:104CE00039320000307800003132000030300000EE
:104CF00020360000304800007A0000003220EF002B
:104D0000A3682200008041001040BA000160EF005B
:104D100000000600202000004E6F000074200000FC
:104D200041760000616900006C610000626C000067
:104D300065200000200000003220EF00836A22007E
:104D4000008041001040BA000160EF000000060042
:104D50005344000020340000383000006920000077
:104D6000323900002E390000374800007A20000058
:104D7000200000003220EF00636C22000080410020
:104D80001040BA000160EF0000000600534400002C
:104D9000204E00005453000043200000532D00001B
:104DA00056690000646500006F20000020000000CC
:104DB0003220EF00436E2200008041001040BA0014
:104DC0000160EF00000006005344000020350000A1
:104DD000373600006920000032350000487A0000B4
:104DE0002020000020200000200000003220EF00E2
:104DF00023702200008041001040BA000160EF00E3
:104E0000000006005344000020500000414C000008
:104E1000205300002D56000069640000656F0000FB
:104E200020200000200000003220EF00037222004A
:104E3000008041001040BA000160EF000000060051
:104E40005344000020340000383000006920000086
:104E50007950000062500000722000002020000005
:104E6000200000003220EF00E373220000804100A8
:104E70001040BA000160EF0000000600534400003B
:104E8000204E00005453000043200000436F0000F8
:104E90006D7000006F730000697400006500000011
:104EA0003220EF00C3752200008041001040BA009C
:104EB0000160EF00000006005344000020350000B0
:104EC0003736000069200000795000006250000071
:104ED0007220000020200000200000003220EF009F
:104EE000A3772200008041001040BA000160EF006B
:104EF000000006005344000020500000414C000018
:104F0000204300006F6D0000706F000073690000A7
:104F100074650000200000003220EF008379220039
:104F2000008041001040BA000160EF000000060060
:104F30004E6F00006E650000000000003220EF00A0
:104F4000A37A2200008041001040BA000160EF0007
:104F5000000006000A0D0000553500005F49000002
:104F60005352000020250000325800002025000088
:104F70003258000020250000325800002025000093
:104F800032580000202500003258000000000000C8
:104F90003220EF00437D2200008041001040BA0023
:104FA0000160EF0000000600553500005F42000080
:104FB0003020000049530000522D000045720000CF
:104FC0007220000025320000582000002532000029
:104FD0005820000025320000582000002532000033
:104FE000582000005B250000325800005D0A0000D8
:104FF0000D0000003220EF0063802200008041009D
:105000001040BA000160EF000000060055350000B6
:105010005F4200003120000049530000522D000083
:105020004572000072200000253200005820000068
:1050300025320000582000002532000058200000D2
:105040005B250000325800005D2000002532000082
:10505000580A00000D0000003220EF008383220078
:10506000008041001040BA000160EF00000006001F
:10507000553500005F420000332000004953000016
:10508000522D000045720000722000002532000001
:10509000582000005B250000325800005D20000011
:1050A0002532000058200000253200005820000062
:1050B00025320000582000000A0D0000000000000A
:1050C0003220EF00E3012000830150000500310091
:1050D000C3872200008041001040BA000160EF0049
:1050E00000000600C08722008381410080814100CA
:1050F0001380BA00000006000A0D4C00553158001C
:10510000303120005F49250053524C0020255800C3
:105110004C582000202525004C584C0020205800D9
:1051200055310A0030300D005F4900005352000035
:10513000202500003220EF00638A22000080410019
:105140001040BA000160EF00000006000A0D0000E8
:1051500028490000646C00006529000050490000E7
:10516000502000005472000069670000676500006D
:105170007220000025750000207500006E6C000094
:105180006174000063680000656400002E00000088
:105190003220EF00438D2200008041001040BA0011
:1051A0000160EF00000006000A0D0000202D000045
:1051B0002D200000446F00006E650000202D0000CF
:1051C0002D0A00000D0000003220EF00A302200095
:1051D000830150000500310003902200008041004F
:1051E0001040BA000160EF000000060000902200AD
:1051F00083814100808141001380BA0000000600D5
:105200000A0D3000547228006967250067654C005C
:105210007220780063682900616E200067656E0067
:10522000206E5700426E6F006B3072005F316B0072
:1052300030283100254C360078292800206E2500C2
:1052400050724C0065765800426E29006B300000A9
:105250005F3100003220EF006393220000804100A4
:105260001040BA000160EF00000006000A0D0000C7
:105270004E65000077200000416300007469000063
:105280007665000020500000726500007365000024
:105290007428000025750000290000003220EF006E
:1052A000A3952200008041001040BA000160EF0089
:1052B000000006000A0D00004F6C00006420000092
:1052C0004163000074690000766500002050000012
:1052D00072650000736500007428000025750000E9
:1052E00029200000756E00006C61000074630000EE
:1052F00068650000640000003220EF00A302200077
:105300008301500005003100839922000080410094
:105310001040BA000160EF000000060080992200F2
:1053200083814100808141001380BA0000000600A3
:105330000A0D3200547228006967250067654C0029
:105340007220780063682900616E200067656E0036
:10535000206E5700426E6F006B3072005F336B003F
:1053600032283100254C360078292800206E25008F
:1053700050724C0065765800426E29006B30000078
:105380005F3300003220EF008302200083015000D1
:1053900005003100E39D2200008041001040BA006A
:1053A0000160EF0000000600E09D220083814100C3
:1053B000808141001380BA00000006000A0D34000D
:1053C000547228006967250067654C0072207800D8
:1053D00063682900616E200067656E00206E5700CB
:1053E000426E6F006B3072005F346B002825310015
:1053F0004C783600292028006E50250072654C003C
:10540000764258006E6B2900305F00003220EF00BA
:10541000A3022000830150000500310023A22200D6
:10542000008041001040BA000160EF00000006005B
:1054300020A2220083814100808141001380BA00B4
:10544000000006000A0D310054722800696725002B
:1054500067654C007220780063682900616E200047
:1054600067656E00206E5700426E6F006B317200F0
:105470005F326B0031283100254C36007829280036
:10548000206E250050724C0065765800426E29004F
:105490006B3100005F3200003220EF00A3022000D9
:1054A000830150000500310083A6220000804100E6
:1054B0001040BA000160EF000000060080A6220044
:1054C00083814100808141001380BA000000060002
:1054D0000A0D3300547228006967250067654C0087
:1054E0007220780063682900616E200067656E0095
:1054F000206E5700426E6F006B3172005F346B009C
:1055000033283100254C360078292800206E2500EC
:1055100050724C0065765800426E29006B310000D5
:105520005F3400003220EF00E3A922000080410038
:105530001040BA000160EF00000006000A0D0000F4
:1055400055310000303000005F5500003130000060
:10555000315F0000495300005220000050720000EB
:105560006573000065740000733A000020000000BD
:105570003220EF0043AC2200008041001040BA000E
:105580000160EF00000006000A0D0000416300000A
:1055900074690000766500005072000065730000B9
:1055A000657400003D250000750A00000D00000034
:1055B0003220EF0043AE2200008041001040BA00CC
:1055C0000160EF00000006000A0D000046690000BF
:1055D00072730000742000005374000065700000B6
:1055E000000000003220EF00E3AF22000080410005
:1055F0001040BA000160EF00000006000A0D000034
:105600002846000053290000536B00006970000019
:1056100020700000726500007365000074200000B7
:1056200025750000206100006374000069760000A9
:10563000652E0000000000003220EF0083B222003F
:10564000008041001040BA000160EF000000060039
:105650000A0D000028460000532900005072000087
:1056600065730000657400002025000075200000AF
:10567000736500006C6500006374000065640000E1
:105680002E0000003220EF00E3B422000080410031
:105690001040BA000160EF00000006000A0D000093
:1056A0004C6100007374000020530000746500001A
:1056B000700000003220EF00030220008301500040
:1056C0000500310063B72200008041001040BA009D
:1056D0000160EF000000060060B7220083814100F6
:1056E000808141001380BA00000006000A0D74009A
:1056F000284C690053296E004163670074692000DB
:105700007665750020506E0072656C0073656100EF
:10571000742074002575630020256800752F2E0005
:105720002575000020770000616900003220EF003D
:1057300023BA2200008041001040BA000160EF004F
:10574000000006000A0D0000284C0000532900004C
:1057500050490000502000005472000069670000AA
:1057600067650000722000002575000020250000FC
:10577000752F000025750000206600006F75000081
:105780006E6400002E0000003220EF0003BD2200F6
:10579000008041001040BA000160EF0000000600E8
:1057A0000A0D0000284C0000532900004F6C000037
:1057B00064200000507200006573000065740000F2
:1057C0002025000075200000257500002F25000011
:1057D00075200000666F0000756E0000642E0000EA
:1057E000000000003220EF00E301200083015000A0
:1057F00005003100E3C02200008041001040BA00E3
:105800000160EF0000000600E0C02200838141003B
:10581000808141001380BA00000006000A0D740068
:10582000284C690053296E00504967005020200021
:105830005472750069676E0067656C0072206100C4
:105840002575740020256300752F680025752E00CE
:1058500020770000616900003220EF0083C322003E
:10586000008041001040BA000160EF000000060017
:105870000A0D0000202D00002D200000446F0000C4
:105880006E650000205000004950000020540000C8
:10589000726900006767000065720000204C00001C
:1058A0006174000063680000656400002D2D000035
:1058B0000A0D0000000000003220EF0083C6220025
:1058C000008041001040BA000160EF0000000600B7
:1058D0000A0D0000284C0000532900005049000028
:1058E00050200000547200006967000067650000E6
:1058F000722000002575000020730000656C000018
:105900006563000074650000642E00000000000064
:105910003220EF0043C92200008041001040BA004D
:105920000160EF00000006000A0D0000284C000096
:1059300053290000536B00006970000020700000C4
:10594000726500007365000074200000257500007A
:10595000206100006374000069760000652E00007D
:10596000000000003220EF00E3CB22000080410065
:105970001040BA000160EF00000006000A0D0000B0
:10598000284C00005329000050720000657300008D
:10599000657400002025000075200000736500007C
:1059A0006C65000063740000656400002E00000058
:1059B0003220EF0043CE2200008041001040BA00A8
:1059C0000160EF00000006000A0D00004D750000A8
:1059D0006C740000692000005374000065700000C2
:1059E000000000003220EF00E3CF220000804100E1
:1059F0001040BA000160EF00000006000A0D000030
:105A0000284D0000532900006E7000002050000057
:105A100072650000736500007420000025750000A9
:105A200020730000656C0000656300007465000071
:105A3000642E0000000000003220EF0083D222001C
:105A4000008041001040BA000160EF000000060035
:105A50000A0D0000536B000069700000284D000023
:105A600053290000706D0000205000007265000096
:105A7000736500007420000025750000202E0000D2
:105A8000000000003220EF00E3D42200008041003B
:105A90001040BA000160EF00000006000A0D00008F
:105AA000536B000069700000284D0000532900006E
:105AB0002050000072650000736500007420000033
:105AC0002575000020250000752000002825000015
:105AD0007529000020530000616D0000652E000054
:105AE000000000003220EF00E3D7220000804100D8
:105AF0001040BA000160EF00000006000A0D00002F
:105B0000536B000069700000284D0000532900000D
:105B100020500000726500007365000074200000D2
:105B200025750000202500007520000028250000B4
:105B30007529000020530000656C000065630000BB
:105B400074650000642E0000000000003220EF00A9
:105B500023DB2200008041001040BA000160EF000A
:105B6000000006000A0D0000536B00006970000081
:105B7000284D0000532900002050000072650000ED
:105B800073650000742000002575000020200000CF
:105B9000536500006C6500006374000065640000DC
:105BA0002E0000003220EF00E3DD220000804100E3
:105BB0001040BA000160EF00000006000A0D00006E
:105BC000536B000069700000284D0000532900004D
:105BD0006E610000205000007265000073650000D7
:105BE00074200000257500002025000075200000AD
:105BF000536500006C65000063740000656400007C
:105C00002E0000003220EF00C3012000830150006D
:105C100005003100E3E12200008041001040BA009D
:105C20000160EF0000000600E0E1220083814100F6
:105C3000808141001380BA00000006000A0D250093
:105C4000284D75005329290020502000726553000B
:105C50007365650074206C005B256500755D6300ED
:105C6000205B7400257565005D20640025752E009D
:105C7000202800003220EF00E301200083015000C3
:105C80000500310063E52200008041001040BA00A9
:105C90000160EF000000060060E522008381410002
:105CA000808141001380BA00000006000A0D7500D3
:105CB000284D2900532920002050530072656500AB
:105CC00073656C00742065005B256300755D74006E
:105CD0002025650075206400205B2E0025750000DE
:105CE0005D200000282500003220EF00E3012000A5
:105CF000830150000500310003E9220000804100CB
:105D00001040BA000160EF000000060000E9220028
:105D100083814100808141001380BA0000000600A9
:105D20000A0D7500284D29005329200020505300EA
:105D30007265650073656C007420650025756300ED
:105D4000205B7400257565005D206400205B2E00DB
:105D5000257500005D200000282500003220EF009E
:105D6000230220008301500005003100A3EC220033
:105D7000008041001040BA000160EF000000060002
:105D8000A0EC220083814100808141001380BA0091
:105D9000000006000A0D7300284D650053297400A9
:105DA000204D2000756C2500746975002D50200071
:105DB0007265250073657500742020006E6F2500E4
:105DC000742075004163200074692E007665000020
:105DD00020500000726500003220EF0043022000D6
:105DE000830150000500310083F022000080410053
:105DF0001040BA000160EF000000060080F02200B1
:105E000083814100808141001380BA0000000600B8
:105E10000A0D2000284D250053297500204D200033
:105E2000756C5B00746925002D50750072655D000E
:105E300073652000742020006E6F5B0074202500C5
:105E4000666F7500756E5D006420200050722E0034
:105E500065730000657400003220EF00230220000B
:105E6000830150000500310083F4220000804100CE
:105E70001040BA000160EF000000060080F422002C
:105E800083814100808141001380BA000000060038
:105E90000A0D5D00284D200053292500206E750055
:105EA0006F742000204D2000756C2500746975000A
:105EB0002D50200072652800736525007420750040
:105EC0005072290065732E0065740000205B00008D
:105ED000257500003220EF002302200083015000CE
:105EE0000500310063F82200008041001040BA0034
:105EF0000160EF000000060060F82200838141008D
:105F0000808141001380BA00000006000A0D5B008A
:105F1000284D250053297500206E5D006F74200008
:105F2000204D2000756C2500746975002D502000EF
:105F30007265280073652500742075005072290071
:105F400065732E0065740000202500007520000098
:105F50003220EF00230220008301500005003100B1
:105F600043FC2200008041001040BA000160EF00B5
:105F70000000060040FC2200838141008081410036
:105F80001380BA00000006000A0D2500284D750098
:105F900053292000206E20006F745B00204D2500E7
:105FA000756C750074695D002D50200072652800C5
:105FB00073652500742075005072290065732E00EA
:105FC0006574000020250000752000003220EF00DD
:105FD000030320008301500005003100230023004B
:105FE000008041001040BA000160EF000000060090
:105FF0002000230083814100808141001380BA008A
:10600000000006000A0D74004E6F650020532E003C
:10601000746553007020790069647300656E7400C4
:106020007469650066696D0065644600206E6C00E9
:106030004163610074696700766531005374200024
:1060400065703D00203D250025323200782C780017
:1060500043750A0072720D00656E000074530000F3
:10606000746100003220EF00E30323000080410050
:106070001040BA000160EF0000000600204E000052
:106080006F740000204600006F7500006E64000011
:106090000A0D0000000000003220EF0083052300FD
:1060A000008041001040BA000160EF0000000600CF
:1060B00020420000746E00002825000032780000A5
:1060C0002F250000752900002D4700007270000088
:1060D000312000000A0D0000000000003220EF0017
:1060E000A3072300008041001040BA000160EF00C8
:1060F00000000600202000004D61000073740000C5
:1061000065720000205000006F770000657200008B
:10611000204F000066660000200000003220EF00E3
:10612000A3092300008041001040BA000160EF0085
:1061300000000600202000004D6100007374000084
:1061400065720000205000006F770000657200004B
:10615000204F00006E200000200000003220EF00E1
:10616000A30B2300008041001040BA000160EF0043
:10617000000006002043000075740000204F00005E
:106180006E0A00000D0000003220EF00030D230016
:10619000008041001040BA000160EF0000000600DE
:1061A00020200000202000002020000020200000EF
:1061B0004375000074200000202000002020000013
:1061C00020200000200000003220EF00030F2300F9
:1061D000008041001040BA000160EF00000006009E
:1061E0002057000069700000652000004F6E00001D
:1061F0000A0D0000000000003220EF008310230091
:10620000008041001040BA000160EF00000006006D
:10621000202000002020000020200000202000007E
:106220005769000070650000202000002020000059
:1062300020200000200000003220EF008312230005
:10624000008041001040BA000160EF00000006002D
:10625000204D000069780000204F00006E0A000009
:106260000D0000003220EF00E31323000080410006
:106270001040BA000160EF0000000600202000007E
:10628000202000002020000020200000204D0000E1
:10629000697800002020000020200000202000005D
:1062A000200000003220EF00E315230000804100B1
:1062B0001040BA000160EF0000000600204D000011
:1062C000756C0000746900002053000074650000C4
:1062D000702000004F6E00000A0D0000000000005A
:1062E0003220EF00C3172300008041001040BA00A5
:1062F0000160EF00000006002020000020200000C8
:10630000204D0000756C00007469000020530000EF
:1063100074650000702000002020000020000000B4
:106320003220EF00C3192300008041001040BA0062
:106330000160EF0000000600204C000061730000C7
:10634000742000005374000065700000204F0000AE
:106350006E0A00000D0000003220EF00831B2300B6
:10636000008041001040BA000160EF00000006000C
:106370002020000020200000204C0000617300005D
:10638000742000005374000065700000202000009D
:1063900020200000200000003220EF00831D230099
:1063A000008041001040BA000160EF0000000600CC
:1063B0002046000069720000737400002053000042
:1063C00074650000702000004F6E00000A0D000090
:1063D000000000003220EF00631F23000080410016
:1063E0001040BA000160EF0000000600202000000D
:1063F0002020000020460000697200007374000035
:106400002053000074650000702000002020000070
:10641000200000003220EF006321230000804100B3
:106420001040BA000160EF000000060020200000CC
:106430002020000020500000726F000067720000F2
:10644000616D0000204F0000666600002020000003
:10645000200000003220EF00632323000080410071
:106460001040BA000160EF0000000600205000005C
:10647000726F000067720000616D0000204F000025
:10648000666600000A0D0000000000003220EF00E8
:1064900023252300008041001040BA000160EF0076
:1064A00000000600202000002020000020500000F6
:1064B000726F000067720000616D0000204F0000E5
:1064C0006E20000020200000200000003220EF009D
:1064D00023272300008041001040BA000160EF0034
:1064E0000000060020500000726F0000677200007C
:1064F000616D0000204F00006E0A00000D000000DA
:106500003220EF00C3282300008041001040BA0071
:106510000160EF00000006002050000072650000DE
:10652000736500007444000069730000616200003C
:106530006C650000204F000066660000200000002F
:106540003220EF00C32A2300008041001040BA002F
:106550000160EF000000060020500000726500009E
:1065600073650000744400006973000061620000FC
:106570006C650000204F0000666600000A0D0000F8
:10658000000000003220EF00E32C230000804100D7
:106590001040BA000160EF0000000600205000002B
:1065A00072650000736500007444000069730000A8
:1065B000616200006C650000204F00006E2000004A
:1065C000200000003220EF00E32E23000080410075
:1065D0001040BA000160EF000000060020500000EB
:1065E0007265000073650000744400006973000068
:1065F000616200006C650000204F00006E0A000020
:106600000D0000003220EF00E33023000080410045
:106610001040BA000160EF00000006002D470000A6
:1066200072700000323A000020420000746E0000D8
:1066300028250000327800002F2500007529000071
:10664000204D0000656E0000750A00000D0000007E
:106650003220EF0043332300008041001040BA0095
:106660000160EF00000006002020000050470000FD
:106670004D2000004D6F00006465000020410000C7
:1066800063740000697600006520000020000000AF
:106690003220EF0043352300008041001040BA0053
:1066A0000160EF000000060020420000746E000050
:1066B00028250000327800002F25000075290000F1
:1066C0002D47000072700000330000003220EF0000
:1066D00023372300008041001040BA000160EF0022
:1066E00000000600204900006E7000007574000074
:1066F000203600000A0D0000000000003220EF00EC
:10670000A3382300008041001040BA000160EF0070
:1067100000000600202000002020000020200000B3
:10672000496E0000707500007420000036200000E3
:106730002020000020200000200000003220EF0078
:10674000A33A2300008041001040BA000160EF002E
:1067500000000600204900006E7000007574000003
:10676000203500000A0D0000000000003220EF007C
:10677000233C2300008041001040BA000160EF007C
:106780000000060020200000202000002020000043
:10679000496E000070750000742000003520000074
:1067A0002020000020200000200000003220EF0008
:1067B000233E2300008041001040BA000160EF003A
:1067C00000000600204900006E7000007574000093
:1067D000203400000A0D0000000000003220EF000D
:1067E000A33F2300008041001040BA000160EF0089
:1067F00000000600202000002020000020200000D3
:10680000496E000070750000742000003420000004
:106810002020000020200000200000003220EF0097
:10682000A3412300008041001040BA000160EF0046
:1068300000000600204900006E7000007574000022
:10684000203300000A0D0000000000003220EF009D
:1068500023432300008041001040BA000160EF0094
:106860000000060020200000202000002020000062
:10687000496E000070750000742000003320000095
:106880002020000020200000200000003220EF0027
:1068900023452300008041001040BA000160EF0052
:1068A00000000600204900006E70000075740000B2
:1068B000203200000A0D0000000000003220EF002E
:1068C000A3462300008041001040BA000160EF00A1
:1068D00000000600202000002020000020200000F2
:1068E000496E000070750000742000003220000026
:1068F0002020000020200000200000003220EF00B7
:10690000A3482300008041001040BA000160EF005E
:1069100000000600204900006E7000007574000041
:10692000203100000A0D0000000000003220EF00BE
:10693000234A2300008041001040BA000160EF00AC
:106940000000060020200000202000002020000081
:10695000496E0000707500007420000031200000B6
:106960002020000020200000200000003220EF0046
:10697000234C2300008041001040BA000160EF006A
:10698000000006002050000049500000204F000089
:106990006E0A00000D0000003220EF00834D23003E
:1069A000008041001040BA000160EF0000000600C6
:1069B000202000002020000020200000504900007E
:1069C000502000004F6E000020200000202000001A
:1069D00020200000200000003220EF00834F230021
:1069E000008041001040BA000160EF000000060086
:1069F0002050000049500000204F00006666000053
:106A00000A0D0000000000003220EF0003512300B7
:106A1000008041001040BA000160EF000000060055
:106A2000202000002020000020200000504900000D
:106A3000502000004F66000066200000202000006B
:106A400020200000200000003220EF00035323002C
:106A5000008041001040BA000160EF000000060015
:106A60002050000049500000204E00006F740000CC
:106A7000204500006E610000626C0000656400004B
:106A80000A0D0000000000003220EF000355230033
:106A9000008041001040BA000160EF0000000600D5
:106AA00020500000495000002043000068610000B1
:106AB0006E670000653A0000204600006F7200001B
:106AC00065670000726F0000756E0000640A0000C8
:106AD0000D0000003220EF006357230000804100CA
:106AE0001040BA000160EF000000060050430000B3
:106AF000686100006E67000065200000466F0000BE
:106B000072650000677200006F7500006E6400001F
:106B1000000000003220EF00635923000080410094
:106B20001040BA000160EF00000006002050000095
:106B30004950000020430000686100006E670000BB
:106B4000653A000020420000616300006B670000AE
:106B5000726F0000756E0000640A00000D000000F6
:106B60003220EF00C35B2300008041001040BA00D8
:106B70000160EF0000000600504300006861000063
:106B80006E6700006520000042610000636B00003A
:106B9000677200006F7500006E6400000000000066
:106BA0003220EF00C35D2300008041001040BA0096
:106BB0000160EF00000006002D4700007270000029
:106BC0003428000054610000736B0000293A000073
:106BD00020420000746E000028250000327800007A
:106BE0002F250000752900000A0D0000000000009C
:106BF0003220EF0043602300008041001040BA00C3
:106C00000160EF00000006000A0D000020200000D7
:106C10002020000041750000746F000050720000D9
:106C200065730000656E0000746500007225000049
:106C3000730A00000D0000003220EF008362230081
:106C4000008041001040BA000160EF000000060023
:106C50000A0D00002020000020200000436F0000EB
:106C60006E740000726F00006C5600004945000011
:106C7000572000005848000044250000730A000017
:106C80000D0000003220EF00E3642300008041008B
:106C90001040BA000160EF00000006002020000054
:106CA00020200000436F00006D700000696C000040
:106CB000656400003A200000257300002061000098
:106CC00074200000257300000A0D00000000000081
:106CD0003220EF0043672300008041001040BA00DB
:106CE0000160EF0000000600313400002D4A000072
:106CF000756C00002D310000300000003220EF00E4
:106D0000A3682300008041001040BA000160EF003A
:106D100000000600313700003A330000383A000026
:106D200034310000000000003220EF00036A23002D
:106D3000008041001040BA000160EF000000060032
:106D400020460000696E0000646900006E67000064
:106D500020430000616D0000657200006173000057
:106D6000000000003220EF00E36B230000804100B0
:106D70001040BA000160EF00000006002020000073
:106D8000205200006573000065740000205600006A
:106D900069640000656F0000202000000000000012
:106DA0003220EF00C36D2300008041001040BA0084
:106DB0000160EF0000000600204300006C65000049
:106DC00061720000696E00006720000050720000D0
:106DD0006573000065740000730000003220EF004E
:106DE000A36F2300008041001040BA000160EF0053
:106DF00000000600204300006C6500006172000086
:106E0000696E000067200000416C00006C200000EB
:106E100020200000000000003220EF0083712300DA
:106E2000008041001040BA000160EF000000060041
:106E3000205200006573000074610000727400004D
:106E40002053000079730000746500006D2000007D
:106E5000000000003220EF00637323000080410037
:106E60001040BA000160EF0000000600456E00000F
:106E7000616200006C650000204800006F73000034
:106E8000742000005365000072690000616C00000E
:106E9000000000003220EF006375230000804100F5
:106EA0001040BA000160EF000000060044690000D5
:106EB00073610000626C00006520000053650000F3
:106EC00072690000616C000020200000202000009A
:106ED000000000003220EF006377230000804100B3
:106EE0001040BA000160EF00000006000A0D00002B
:106EF000436F00006D6D0000616E000064200000B3
:106F0000436F00006D7000006C6500007465000048
:106F10000A0D00003E0000003220EF0083792300BC
:106F2000008041001040BA000160EF000000060040
:106F3000202000002053000061760000696E0000F0
:106F400067200000436F00006E6600006967000064
:106F500020200000000000003220EF00837B23008F
:106F6000008041001040BA000160EF000000060000
:106F7000202000005368000075740000646F00005A
:106F8000776E000020410000637400006976000005
:106F900065200000000000003220EF00837D230008
:106FA000008041001040BA000160EF0000000600C0
:106FB00020430000616D0000657200006120000048
:106FC000506F000077650000726400006F7700006A
:106FD0006E200000000000003220EF00837F2300BD
:106FE000008041001040BA000160EF000000060080
:106FF00020420000746E0000282500003278000056
:107000002F250000752900002D4700007270000038
:10701000352000000A0D0000000000003220EF00C3
:10702000A3812300008041001040BA000160EF00FE
:1070300000000600507200006F63000065730000DE
:10704000732000005072000065730000657400003A
:107050002042000075740000746F00006E20000074
:10706000257500000A0D0000000000003220EF002E
:1070700023842300008041001040BA000160EF002B
:1070800000000600566100006C69000064200000EA
:107090005072000065730000657400002025000038
:1070A000750A00000D0000003220EF000386230067
:1070B000008041001040BA000160EF0000000600AF
:1070C0005072000065730000657400002025000008
:1070D00033750000205400006F2000004869000054
:1070E00067680000000000003220EF0003882300E2
:1070F000008041001040BA000160EF00000006006F
:1071000050720000657300006574000020250000C7
:1071100075200000746F000020680000696700009F
:10712000680A00000D0000003220EF00038A2300EF
:10713000008041001040BA000160EF00000006002E
:10714000507200006F670000726100006D20000047
:107150004D6F0000646500000A0D00000000000093
:107160003220EF00C38B2300008041001040BA00A2
:107170000160EF00000006004D7500006C74000017
:107180006953000074650000700A00000D000000E3
:107190003220EF00438D2300008041001040BA00F0
:1071A0000160EF00000006004669000072730000F5
:1071B0007453000074650000700A00000D000000A8
:1071C0003220EF00C38E2300008041001040BA003F
:1071D0000160EF00000006004C61000073740000C5
:1071E00053740000657000000A0D000000000000EC
:1071F0003220EF0043902300008041001040BA008D
:107200000160EF00000006002050000072650000E1
:107210007365000074200000253300007520000015
:10722000537400006F7200006564000000000000ED
:107230003220EF0043922300008041001040BA004A
:107240000160EF000000060020520000657400009D
:10725000726900006576000065200000536500003B
:1072600074740000696E0000677300000000000085
:107270003220EF0043942300008041001040BA0008
:107280000160EF0000000600476500007420000068
:10729000436100006D650000726100002044000041
:1072A00061740000610A00000D0000003220EF0050
:1072B00023962300008041001040BA000160EF00D7
:1072C0000000060020530000746F0000726500008B
:1072D00020500000726500007365000074200000FB
:1072E0002533000075200000000000003220EF0070
:1072F00023982300008041001040BA000160EF0095
:1073000000000600537400006F720000652000004A
:1073100050720000657300006574000020250000B5
:1073200075200000436F00006D7000006C65000068
:10733000746500000A0D0000000000003220EF001C
:10734000A39A2300008041001040BA000160EF00C2
:107350000000060020500000726500007365000008
:1073600074200000253300007520000046610000F5
:10737000696C000065640000000000003220EF002E
:10738000A39C2300008041001040BA000160EF0080
:1073900000000600537400006F72000065200000BA
:1073A0005072000065730000657400002025000025
:1073B0007520000046610000696C000065640000F3
:1073C0000A0D0000000000003220EF00039F2300A0
:1073D000008041001040BA000160EF00000006008C
:1073E00050720000657300006574000020250000E5
:1073F00033750000203D000020500000495000007F
:1074000020200000000000003220EF0003A1230034
:10741000008041001040BA000160EF00000006004B
:1074200050720000657300006574000020250000A4
:10743000752000003D20000050490000500A000067
:107440000D0000003220EF00E3A223000080410085
:107450001040BA000160EF0000000600507200000A
:107460006573000065740000202500007520000091
:10747000746F00006F2000006869000067680000FA
:107480000A0D0000000000003220EF0003A52300D9
:10749000008041001040BA000160EF0000000600CB
:1074A000507200006573000065740000204D0000FC
:1074B0006F640000650A00000D0000003220EF003C
:1074C000A3A62300008041001040BA000160EF0035
:1074D00000000600202000005265000061640000EA
:1074E00020500000726500007365000074200000E9
:1074F0002533000075200000000000003220EF005E
:10750000A3A82300008041001040BA000160EF00F2
:1075100000000600507200006573000065740000F2
:107520002025000075200000666F0000756E0000C9
:10753000640A00000D0000003220EF0083AA23003F
:10754000008041001040BA000160EF00000006001A
:107550005072000065730000657400002025000073
:10756000752000004C61000073740000537400002B
:10757000657000000A0D0000000000003220EF00DE
:10758000A3AC2300008041001040BA000160EF006E
:107590000000060050720000657300006574000072
:1075A000202500007520000046690000727300006D
:1075B0007453000074650000700A00000D000000A4
:1075C0003220EF00C3AE2300008041001040BA001B
:1075D0000160EF00000006005072000065730000BB
:1075E0006574000020250000752000004D75000026
:1075F0006C7400006953000074650000700A00009C
:107600000D0000003220EF00E3B0230000804100B5
:107610001040BA000160EF00000006005072000048
:1076200065730000657400002025000075200000CF
:107630002853000074650000705000006F73000054
:1076400073690000626C000065290000506F000043
:1076500073730000696200006C6500000A0D000091
:10766000000000003220EF00E3B32300008041005F
:107670001040BA000160EF000000060050720000E8
:10768000657300006574000020250000752000006F
:10769000436100006D65000072610000204600003B
:1076A0006F7500006E6400000A0D0000000000000D
:1076B0003220EF0043B62300008041001040BA00A2
:1076C0000160EF000000060020200000557000005F
:1076D00064610000746900006E67000020430000D0
:1076E000616D000065720000612000000000000074
:1076F0003220EF0043B82300008041001040BA0060
:107700000160EF0000000600436100006D200000F2
:107710004E6F00007441000076610000696C00004B
:1077200020500000726500007365000074200000A6
:1077300025750000200A00000D0000003220EF0037
:10774000A3BA2300008041001040BA000160EF009E
:10775000000006004E6F0000436100006D20000035
:107760005072000065730000657400002025000061
:10777000752000000A0D0000000000003220EF001C
:10778000A3BC2300008041001040BA000160EF005C
:1077900000000600205000007265000073650000C4
:1077A0007420000025330000752000004C6F00009D
:1077B00061640000656400000A0D00000000000024
:1077C0003220EF00C3BE2300008041001040BA0009
:1077D0000160EF000000060020200000204E0000A5
:1077E0006F20000050720000657300006574000097
:1077F000202500003375000020200000000000005C
:107800003220EF00C3C02300008041001040BA00C6
:107810000160EF0000000600507200006573000078
:107820006574000020250000752000004E6F0000E8
:1078300074200000466F0000756E0000640A0000AE
:107840000D0000003220EF00E3C223000080410061
:107850001040BA000160EF0000000600536B00000A
:10786000697000002D460000532000005072000097
:10787000657300006574000020250000752000007D
:107880004E6F000074200000466F0000756E00000F
:10789000640A00000D0000003220EF0083C52300C1
:1078A000008041001040BA000160EF0000000600B7
:1078B00050720000657300006574000020440000F1
:1078C00069730000616200006C650000640A0000DA
:1078D0000D0000003220EF0063C72300008041004C
:1078E0001040BA000160EF000000060020500000C8
:1078F000726500007365000074730000204400008E
:1079000069730000616200006C6500006420000083
:10791000200000003220EF0063C9230000804100F6
:107920001040BA000160EF0000000600504900005E
:107930005020000050720000657300006574000064
:10794000204D00006F640000650A00000D0000007B
:107950003220EF0043CB2300008041001040BA00EA
:107960000160EF00000006005049000050200000B8
:10797000507200006573000065740000202500004F
:1079800075200000666F0000756E0000640A00003C
:107990000D0000003220EF0063CD23000080410085
:1079A0001040BA000160EF000000060050490000DE
:1079B00050200000507200006573000065740000E4
:1079C0002025000075200000436100006D65000067
:1079D00072610000204600006F7500006E640000B8
:1079E0000A0D0000000000003220EF0003D0230049
:1079F000008041001040BA000160EF000000060066
:107A000050490000502000005072000065730000D3
:107A10006574000020250000752000005061000002
:107A20006E610000736F00006E690000632000004B
:107A3000436F00006D7000006C650000746500000D
:107A40000A0D0000000000003220EF0003D32300E5
:107A5000008041001040BA000160EF000000060005
:107A60005049000050200000507200006573000073
:107A7000657400002025000075200000536F000091
:107A80006E7900002F430000616E00006F6E0000F1
:107A9000204300006F6D0000706C000065740000F2
:107AA000650A00000D0000003220EF0003D623001D
:107AB000008041001040BA000160EF0000000600A5
:107AC0005049000050200000507200006573000013
:107AD000657400002025000075200000436100004F
:107AE0006D2000004E6F00007441000076610000C0
:107AF000696C00000A0D0000000000003220EF0059
:107B0000A3D82300008041001040BA000160EF00BC
:107B10000000060050490000502000005072000094
:107B200065730000657400002025000075200000CA
:107B30004E6F0000436100006D0A00000D00000060
:107B40003220EF00C3DA2300008041001040BA0069
:107B50000160EF00000006005049000050200000C6
:107B6000507200006573000065740000202500005D
:107B70007520000054720000616E000073690000FF
:107B8000746900006F6E00000A0D00000000000024
:107B90003220EF0043DD2300008041001040BA0096
:107BA0000160EF0000000600504900005020000076
:107BB000507200006573000065740000202500000D
:107BC0007520000054720000616E000073690000AF
:107BD000746900006F6E000028730000290A00001D
:107BE0000D0000003220EF00E3DF230000804100A1
:107BF0001040BA000160EF0000000600504900008C
:107C00005020000050720000657300006574000091
:107C1000202500007520000054720000616E0000F5
:107C200073690000746900006F6E0000286700002F
:107C3000290A00000D0000003220EF0083E223003B
:107C4000008041001040BA000160EF000000060013
:107C500020500000495000002050000072650000D4
:107C600073650000742000002533000075200000BB
:107C70004C6F000061640000656400000A0D0000A4
:107C8000000000003220EF00E3E423000080410008
:107C90001040BA000160EF000000060050490000EB
:107CA00050200000507200006573000065740000F1
:107CB00020250000752000004E6F00007420000099
:107CC000466F0000756E0000640A00000D000000A1
:107CD0003220EF0043E72300008041001040BA004B
:107CE0000160EF00000006000A0D0000436800007C
:107CF0006B540000726100006E540000696D00005A
:107D0000654500006E6300006F640000657200004E
:107D100028250000303400004C78000029000000C5
:107D20003220EF00C3E92300008041001040BA0078
:107D30000160EF00000006002054000072610000A6
:107D40006E540000696D000065200000256300008E
:107D50002E250000633000002073000065630000E2
:107D6000000000003220EF00E3EB23000080410020
:107D70001040BA000160EF00000006000A0D00008C
:107D8000436800006B5A00006F6F00006D450000F3
:107D90006E6300006F64000065720000282500001B
:107DA000303400004C780000290000003220EF0041
:107DB00023EE2300008041001040BA000160EF0074
:107DC00000000600202000004D6100007820000027
:107DD0005A6F00006F6D0000202500007500000044
:107DE0003220EF00C3EF2300008041001040BA00B2
:107DF0000160EF00000006000A0D0000436800006B
:107E00006B500000616E0000456E0000636F000063
:107E1000646500007228000025300000344C00002A
:107E200078290000000000003220EF0003F2230058
:107E3000008041001040BA000160EF000000060021
:107E4000202000004D6100007820000050610000FB
:107E50006E20000025750000000000003220EF00B9
:107E6000A3F32300008041001040BA000160EF003E
:107E7000000006000A0D0000436800006B5400007B
:107E8000696C0000744500006E6300006F640000C0
:107E90006572000028250000303400004C78000096
:107EA000290000003220EF00E3F5230000804100AC
:107EB0001040BA000160EF00000006002020000022
:107EC0004D61000078200000546900006C740000CF
:107ED00020250000750000003220EF0083F723000A
:107EE000008041001040BA000160EF000000060071
:107EF0000A0D0000436800006B4600006F6300003D
:107F000075730000456E0000636F0000646500003B
:107F10007228000025300000344C00007829000051
:107F2000000000003220EF00E3F923000080410050
:107F30001040BA000160EF00000006000A0D0000CA
:107F4000436800006B490000726900007350000034
:107F50006F730000456E0000636F000064650000F1
:107F60007228000025300000344C00007829000001
:107F7000000000003220EF0063FC2300008041007D
:107F80001040BA000160EF00000006000A0D00007A
:107F9000436800006B52000065640000456E0000FD
:107FA000636F000064650000722800002530000047
:107FB000344C000078290000000000003220EF005F
:107FC000A3FE2300008041001040BA000160EF00D2
:107FD000000006000A0D0000436800006B4200002C
:107FE0006C750000654500006E6300006F64000062
:107FF0006572000028250000303400004C78000035
:10800000290000003220EF00E3002400008041003E
:108010001040BA000160EF00000006000A0D0000E9
:10802000436800006B440000657400006169000053
:108030006C4500006E6300006F6400006572000014
:1080400028250000303400004C7800002900000092
:108050003220EF0043032400008041001040BA00AA
:108060000160EF00000006000A0D000043680000F8
:108070006B470000616900006E5000006F730000E4
:10808000456E0000636F0000646500007228000008
:1080900025300000344C000078290000000000006A
:1080A0003220EF00C3052400008041001040BA00D8
:1080B0000160EF00000006003E2500007320000074
:1080C0004E6F000074200000466F0000756E0000C7
:1080D000640A00000D3E0000000000003220EF00A6
:1080E000A3072400008041001040BA000160EF00A7
:1080F00000000600436F00006D700000696C000016
:10810000656400003A200000257300002061000033
:1081100074200000257300000A0D0000000000001C
:108120003220EF00E3012000830150000500310000
:10813000C30A2400008041001040BA000160EF0033
:1081400000000600C00A24008381410080814100B4
:108150001380BA00000006000D0A50005379720027
:1081600073746500656D7300205365006574740059
:1081700074693A006E672000733A25000A0D6400A6
:108180000A0D0A0044650D0066610000756C000070
:10819000742000003220EF00630D240000804100B5
:1081A0001040BA000160EF000000060041630000CB
:1081B000746900007665000020430000616D0000D6
:1081C00065720000613A000020250000730A00007B
:1081D0000D0000003220EF00630F240000804100FA
:1081E0001040BA000160EF0000000600436100008B
:1081F0006D6500007261000020530000656C000096
:1082000065630000743A000020250000750A000034
:108210000D0000003220EF006311240000804100B7
:108220001040BA000160EF00000006002049000085
:108230006E7000007574000020530000656C000033
:1082400065630000743A000020250000750A0000F4
:108250000D0000003220EF00631324000080410075
:108260001040BA000160EF00000006000D0A000097
:10827000576900007065000020440000657300002D
:108280006372000069700000746900006F6E000086
:108290003A200000257300000A0D000000000000D5
:1082A0003220EF00C3152400008041001040BA00C6
:1082B0000160EF00000006000A0D000050490000B8
:1082C00050200000446500007363000072690000E4
:1082D00070740000696F00006E3A000020250000F5
:1082E000730A00000D0000003220EF000318240084
:1082F000008041001040BA000160EF00000006005D
:10830000504900005020000043680000616E0000EA
:10831000676500003A200000257300000A0D000088
:10832000000000003220EF00E3192400008041002B
:108330001040BA000160EF00000006004F75000019
:108340007470000075740000204600006F72000019
:108350006D610000743A000020250000730A0000DF
:108360000D0000003220EF00E31B240000804100DC
:108370001040BA000160EF0000000600506F0000DE
:10838000727400002025000075200000496E000076
:108390007075000074200000466F0000726D0000D0
:1083A000617400003A200000257300000A0D0000EF
:1083B000000000003220EF00430320008301500042
:1083C00005003100631F2400008041001040BA0006
:1083D0000160EF0000000600601F2400838141005F
:1083E000808141001380BA00000006000A0D610080
:1083F00050616E006E532000706554006564690022
:1084000020206D0020206500546920006C7420003D
:10841000537050006565610064206E002020650087
:108420005A6F6C006F6D200053704C0065656900D9
:108430006420670020496800646C74006520730044
:1084400052650A0074750D00726E00002020000055
:10845000547200003220EF00E3022000830150003C
:108460000500310063242400008041001040BA0060
:108470000160EF00000006006024240083814100B9
:10848000808141001380BA000000060020202000F7
:108490002025200064202000202020002020200013
:1084A00020202500202075002020200025642000A9
:1084B000202020002020200020202000202020003C
:1084C00020202000256420002020200020202500DE
:1084D0002020640020200A0020200D0025640A00CE
:1084E00020200D00202000003220EF00032824006F
:1084F000008041001040BA000160EF00000006005B
:108500000A0D0000507200006573000065740000E1
:10851000733A00000A0D00000A0D00000000000080
:108520003220EF00E30220008301500005003100FB
:10853000C32A2400008041001040BA000160EF000F
:1085400000000600C02A2400838141008081410090
:108550001380BA000000060050725A0065206F00B8
:1085600053726F0063206D004D6F20006465200022
:108570006C205400202072002020610020206E001A
:1085800020207300202020002020200020204600F2
:1085900020206C002020610020506700616E730075
:1085A000202020002020200054690A006C740D0057
:1085B000202000003220EF00632E240000804100C4
:1085C0001040BA000160EF00000006004F6E00008E
:1085D0006C79000020540000726100006E7300008E
:1085E00069740000696F00006E2000002020000008
:1085F000200000003220EF00230220008301500001
:108600000500310063312400008041001040BA00B1
:108610000160EF000000060060312400838141000A
:10862000808141001380BA0000000600253332002B
:1086300075205800202520006420200020252000DF
:10864000313820007320200020202500254C3200E6
:1086500058205800202520004C58200020200A00D7
:10866000254C0D005820000020200000202500008F
:108670003220EF0043342400008041001040BA0053
:108680000160EF00000006000A0D000050490000E4
:1086900050200000507200006573000065740000F7
:1086A000733A00000A0D00000A0D000000000000EF
:1086B0003220EF00E302200083015000050031006A
:1086C00043372400008041001040BA000160EF00F1
:1086D0000000060040372400838141008081410072
:1086E0001380BA000000060050725A0065206F0027
:1086F00053726F0063206D004D6F20006465200091
:108700006C202000202054002020790020207000C0
:10871000202065002020200020202000202046006E
:1087200020206C002020610020506700616E7300E3
:10873000202020002020200054690A006C740D00C5
:10874000202000003220EF00E33A240000804100A6
:108750001040BA000160EF00000006000A0D0000A2
:108760005043000043200000507200006573000079
:1087700065740000733A00000A0D00000A0D000045
:10878000000000003220EF0063032000830150004E
:1087900005003100E33D2400008041001040BA0094
:1087A0000160EF0000000600E03D240083814100ED
:1087B000808141001380BA0000000600436172000E
:1087C0006D20690050727300652020004D6F2000FD
:1087D000646547006C2061002020690020206E0045
:1087E0002020200020202000202052002020650092
:1087F00020506400616E20002020200020202000F6
:1088000020544200696C6C0074207500205A650089
:108810006F6F20006D204400204665006F63740078
:1088200075732E00204900003220EF00034224001F
:10883000008041001040BA000160EF000000060017
:10884000205B000049720000697300002C460000A4
:108850006F630000757300002C4100005742000058
:108860002C200000424C0000435D0000205400001A
:10887000726100006E73000020200000466C000052
:1088800061670000730A00000D0A00000D0000007F
:108890003220EF00C30220008301500005003100A8
:1088A00043462400008041001040BA000160EF0000
:1088B0000000060040462400838141008081410081
:1088C0001380BA0000000600202558006420200014
:1088D000202520003264250020204C00253158003E
:1088E00038732000255820002558250025584C00B5
:1088F00020205800254C200058202000202525004D
:108900004C58320020204C00254C580058202000A4
:10891000202520004C58200020202000254C00005D
:108920003220EF00C3492400008041001040BA000B
:108930000160EF00000006004F6E000020200000E4
:10894000200000003220EF00E34A240000804100B4
:108950001040BA000160EF00000006004F66000002
:1089600066200000200000003220EF00034C2400AD
:10897000008041001040BA000160EF0000000600D6
:108980002020000020200000253200005820000098
:1089900020200000202000002532000058000000A8
:1089A0003220EF00C34D2400008041001040BA0087
:1089B0000160EF00000006000A0D000043610000A6
:1089C0006D2000004D6F0000646500006C0A00001F
:1089D0000D0000003220EF00634F240000804100B2
:1089E0001040BA000160EF000000060020250000E2
:1089F00064200000204E00006F2000004361000052
:108A00006D650000726100000A0D000000000000AA
:108A10003220EF0043512400008041001040BA0092
:108A20000160EF00000006000A0D0000454500004F
:108A3000507200006F6D000020440000756D000052
:108A4000703A00000A0D0000000000003220EF0024
:108A500023532400008041001040BA000160EF0061
:108A6000000006000A0D000045450000507200009D
:108A70006F6D0000204300006F6E0000666900000B
:108A800067200000447500006D7000003A0A000085
:108A90000D0000003220EF006355240000804100EB
:108AA0001040BA000160EF00000006000A0D00004F
:108AB00045450000507200006F6D0000205000001E
:108AC00072650000736500007420000044750000AA
:108AD0006D7000003A0A00000D0000003220EF0027
:108AE000A3572400008041001040BA000160EF004D
:108AF000000006000A0D000045450000507200000D
:108B00006F6D0000204800006967000068200000C9
:108B1000447500006D7000003A0A00000D0000006E
:108B20003220EF00C3592400008041001040BA00F9
:108B30000160EF00000006000A0D0000454500003E
:108B4000507200006F6D0000205000004343000091
:108B50002050000072650000736500007420000062
:108B6000447500006D7000003A0A00000D0000001E
:108B70003220EF0003022000830150000500310085
:108B8000435D2400008041001040BA000160EF0006
:108B900000000600405D2400838141008081410087
:108BA0001380BA00000006000A0D720045456500FA
:108BB000507273006F6D65002050740049502000A2
:108BC000204644006F72750065676D00726F70001B
:108BD000756E3A0064200A0043610D006D65000067
:108BE00072610000205000003220EF00036024007A
:108BF000008041001040BA000160EF000000060054
:108C000020200000202000002020000000000000A4
:108C10003220EF00E3012000830150000500310005
:108C200043622400008041001040BA000160EF0060
:108C300000000600406224008381410080814100E1
:108C40001380BA00000006000A0D65000A0D7300CB
:108C50005265700061646F0020496E0032437300FA
:108C6000204D650075783D00204125006464320088
:108C70007265580073730A003D250D0032580000DC
:108C8000205200003220EF00E36424000080410005
:108C90001040BA000160EF00000006004D750000B2
:108CA00078200000577200006974000065420000DF
:108CB00079740000653D0000257500000A0D000074
:108CC000000000003220EF00C301200083015000AB
:108CD00005003100E3672400008041001040BA0025
:108CE0000160EF0000000600E0672400838141007E
:108CF000808141001380BA00000006000A0D580070
:108D00000A0D2C00577244006974610065207400DC
:108D10004932610063203D004D7525007820320006
:108D2000416458006472200065730A00733D0D00B1
:108D3000253200003220EF00636A240000804100E9
:108D40001040BA000160EF00000006000A0D0000AC
:108D50000A0D0000204900006E760000616C0000E2
:108D6000696400002052000065670000697300001C
:108D7000746500007220000028250000732900009F
:108D80000A0D0000000000003220EF00036D2400F7
:108D9000008041001040BA000160EF0000000600B2
:108DA0000A0D00000A0D0000204900006E76000048
:108DB000616C00006964000020490000326300001B
:108DC00020410000646400007265000073730000BD
:108DD0002028000025730000290A00000D00000073
:108DE0003220EF00C36F2400008041001040BA0021
:108DF0000160EF00000006000A0D00000A0D0000EF
:108E0000204900006E760000616C0000696400007B
:108E10002049000032630000205200006567000016
:108E200069730000746500007220000028250000AE
:108E3000732900000A0D0000000000003220EF003E
:108E4000430220008301500005003100A373240079
:108E5000008041001040BA000160EF0000000600F1
:108E6000A073240083814100808141001380BA00F7
:108E7000000006000A0D58000A0D2000526552003D
:108E800061646500204973003243700020416F0027
:108E900064646E0072657300737365003D253D0068
:108EA00032582500205232006567580069730A0065
:108EB00074650D00723D0000253200003220EF0085
:108EC000030220008301500005003100A377240035
:108ED000008041001040BA000160EF000000060071
:108EE000A077240083814100808141001380BA0073
:108EF000000006000A0D32000A0D580057722C00BF
:108F0000697444006520610041647400647261000A
:108F100065733D00733D250025323200582C580002
:108F20005265200067690A0073740D0065720000C5
:108F30003D2500003220EF00430220008301500055
:108F400005003100637B2400008041001040BA001E
:108F50000160EF0000000600607B24008381410077
:108F6000808141001380BA00000006000A0D520003
:108F70000A0D6500204967006E766900616C730018
:108F8000696474002049650032637200204120004A
:108F90006464280072652500737373002825290016
:108FA00073290A0020610D006E6400002F6F00001D
:108FB000722000003220EF00637E24000080410018
:108FC0001040BA000160EF00000006000A0D00002A
:108FD0000A0D0000204E00006F20000064610000B8
:108FE000746100000A0D0000000000003220EF0054
:108FF00023802400008041001040BA000160EF008F
:10900000000006000A0D000053500000492D00002A
:1090100057720000697400006520000025320000CE
:1090200078250000327800000A0D000000000000E2
:109030003220EF0043822400008041001040BA003B
:109040000160EF00000006000A0D00003E20000055
:1090500050490000503D00004F660000660A0000C5
:109060000D3E0000200000003220EF0003842400A9
:10907000008041001040BA000160EF0000000600CF
:109080000A0D00003E20000050490000503D000045
:109090004F6E00000A0D00003E200000000000009E
:1090A0003220EF00C3852400008041001040BA0048
:1090B0000160EF00000006000A0D00003E200000E5
:1090C00044690000616700003D4F00006E0A000027
:1090D0000D3E0000200000003220EF0083872400B6
:1090E000008041001040BA000160EF00000006005F
:1090F0000A0D00003E200000446900006167000086
:109100003D4F0000666600000A0D00003E20000092
:10911000000000003220EF0063892400008041003D
:109120001040BA000160EF00000006000A0D0000C8
:109130003E20000050490000502000004C6F00000D
:1091400063610000746900006F6E00003D30000034
:109150003A4E00006F6E0000650A00000D3E0000F0
:10916000200000003220EF00E38B2400008041004B
:109170001040BA000160EF00000006000A0D000078
:109180003E20000050490000502000004C6F0000BD
:1091900063610000746900006F6E00003D310000E3
:1091A0003A550000520A00000D3E00002000000069
:1091B0003220EF00438E2400008041001040BA00AE
:1091C0000160EF00000006000A0D00003E200000D4
:1091D00050490000502000004C6F00006361000007
:1091E000746900006F6E00003D3200003A4C0000D0
:1091F000520A00000D3E0000200000003220EF0067
:10920000A3902400008041001040BA000160EF00EC
:10921000000006000A0D00003E200000504900003A
:10922000502000004C6F0000636100007469000072
:109230006F6E00003D3300003A4C00004D0A000004
:109240000D3E0000200000003220EF0003932400B8
:10925000008041001040BA000160EF0000000600ED
:109260000A0D00003E200000504900005020000080
:109270004C6F000063610000746900006F6E0000B5
:109280003D3400003A4C00004C0A00000D3E000046
:10929000200000003220EF00639524000080410090
:1092A0001040BA000160EF00000006000A0D000047
:1092B0003E20000050490000502000004C6F00008C
:1092C00063610000746900006F6E00003D350000AE
:1092D0003A5500004C0A00000D3E0000200000003E
:1092E0003220EF00C3972400008041001040BA00F4
:1092F0000160EF00000006000A0D00003E200000A3
:10930000506F000077650000723D00004F6E000056
:109310000A0D00003E200000000000003220EF0097
:10932000A3992400008041001040BA000160EF00C2
:10933000000006000A0D00003E200000506F0000F3
:1093400077650000723D00004F660000660A00006D
:109350000D3E0000200000003220EF00839B24001F
:10936000008041001040BA000160EF0000000600DC
:109370000A0D00003E200000534400006961000017
:10938000673D00004F6E00000A0D00003E20000007
:10939000000000003220EF00639D240000804100A7
:1093A0001040BA000160EF00000006000A0D000046
:1093B0003E2000005344000069610000673D00004A
:1093C0004F660000660A00000D3E0000200000000D
:1093D0003220EF00439F2400008041001040BA007B
:1093E0000160EF00000006000A0D00003E200000B2
:1093F000546100006C6C0000793D00004163000086
:109400007469000076650000204C00006F77000052
:109410000A0D00003E200000000000003220EF0096
:10942000A3A12400008041001040BA000160EF00B9
:10943000000006000A0D00003E20000054610000FC
:109440006C6C0000793D000041630000746900000D
:10945000766500002048000069670000680A000087
:109460000D3E0000200000003220EF0003A4240085
:10947000008041001040BA000160EF0000000600CB
:109480000A0D00003E20000050490000502000005E
:10949000536900007A6500003D5300006D610000D3
:1094A0006C6C00000A0D00003E200000000000006F
:1094B0003220EF0043A62400008041001040BA0093
:1094C0000160EF00000006000A0D00003E200000D1
:1094D0005049000050200000536900007A650000E8
:1094E0003D4D000065640000697500006D0A0000D4
:1094F0000D3E0000200000003220EF0083A8240071
:10950000008041001040BA000160EF00000006003A
:109510000A0D00003E2000005049000050200000CD
:10952000536900007A6500003D4C00006172000044
:10953000676500000A0D00003E20000000000000EA
:109540003220EF002302200083015000050031008B
:10955000C3AB2400008041001040BA000160EF005E
:1095600000000600C0AB24008381410080814100DF
:109570001380BA00000006000A0D61003E20690059
:109580004A53740044375400302069002D206D0088
:109590004A6F65007973280074692500636B750054
:1095A000205329006C6F0A0077200D0044373E00DD
:1095B000302020004F6E00002C5700003220EF00BA
:1095C000230220008301500005003100A3AF2400D6
:1095D000008041001040BA000160EF00000006006A
:1095E000A0AF240083814100808141001380BA0034
:1095F000000006000A0D57003E2061004A53690032
:1096000044377400302054002D2069004A6F6D00EB
:109610007973650074692800636B25002053750019
:109620006C6F290077200A0044370D0030203E007F
:109630004F662000662C00003220EF0083B2240029
:10964000008041001040BA000160EF0000000600F9
:109650000A0D00003E2000005072000065730000FB
:10966000657400007320000044690000736100000D
:10967000626C0000656400000A0D00003E200000DE
:10968000000000003220EF00E3B42400008041001D
:109690001040BA000160EF00000006000A0D000053
:1096A0003E200000507200006573000065740000E9
:1096B00073200000456E0000616200006C650000D0
:1096C000640A00000D3E0000200000003220EF0080
:1096D00023B72400008041001040BA000160EF0071
:1096E000000006000A0D00003E200000436100005B
:1096F0006D650000726100002025000064200000FC
:10970000496E0000766100006C690000640A000088
:109710000D3E0000200000003220EF0083B924003D
:10972000008041001040BA000160EF000000060018
:10973000203000003A5700006970000065200000EA
:10974000523E00004C0000003220EF0003BB24001A
:10975000008041001040BA000160EF0000000600E8
:10976000203100003A5700006970000065200000B9
:109770004C3E0000520000003220EF0083BC240069
:10978000008041001040BA000160EF0000000600B8
:10979000203200003A570000697000006520000088
:1097A000546F0000703E0000426F00007400000023
:1097B0003220EF0043BE2400008041001040BA0078
:1097C0000160EF0000000600203300003A5700005F
:1097D0006970000065200000426F0000743E0000C8
:1097E000546F0000700000003220EF0003C024001E
:1097F000008041001040BA000160EF000000060048
:10980000203400003A4300006F7200006E650000D3
:10981000722000004C5200003E5500004C00000039
:109820003220EF00C3C12400008041001040BA0084
:109830000160EF0000000600203500003A43000000
:109840006F7200006E650000722000004C4C00003A
:109850003E550000520000003220EF0083C3240078
:10986000008041001040BA000160EF0000000600D7
:10987000203600003A4300006F7200006E65000061
:1098800072200000555200003E4C00004C000000C9
:109890003220EF0043C52400008041001040BA0090
:1098A0000160EF0000000600203700003A4300008E
:1098B0006F7200006E65000072200000554C0000C1
:1098C0003E4C0000520000003220EF0003C724008D
:1098D000008041001040BA000160EF000000060067
:1098E000203800003A570000697000006520000031
:1098F0004F750000743E0000436500006E74000068
:1099000065720000000000003220EF0003C924004F
:10991000008041001040BA000160EF000000060026
:10992000203900003A5700006970000065200000EF
:109930004C3E0000436500006E740000657200003C
:109940003C520000000000003220EF0003CB240056
:10995000008041001040BA000160EF0000000600E6
:1099600020310000303A00005769000070650000A7
:10997000205400003E430000656E00007465000046
:10998000723C0000420000003220EF0003CD2400B2
:10999000008041001040BA000160EF0000000600A6
:1099A000202000003A4E00006F6E0000652000008D
:1099B000536500006C65000063740000656400007E
:1099C000000000003220EF00E3CE240000804100C0
:1099D0001040BA000160EF00000006000A0D000010
:1099E0003E200000576900007065000053650000CC
:1099F0006C3D0000257300000A0D00003E200000B1
:109A0000000000003220EF00E3D02400008041007D
:109A10001040BA000160EF00000006000A0D0000CF
:109A20003E200000496400006C6500005274000094
:109A30006E3D0000256400002053000065630000B7
:109A40006F6E0000647300000A0D00003E200000ED
:109A5000000000003220EF0063D3240000804100AA
:109A60001040BA000160EF00000006000A0D00007F
:109A70003E200000504900005020000043680000D4
:109A8000616E0000676500003D42000061630000F8
:109A90006B670000726F0000756E0000640A0000C2
:109AA0000D3E0000200000003220EF0003D624000D
:109AB000008041001040BA000160EF000000060085
:109AC0000A0D00003E200000504900005020000018
:109AD00043680000616E0000676500003D460000BD
:109AE0006F72000065670000726F0000756E000005
:109AF000640A00000D3E0000200000003220EF004C
:109B0000A3D82400008041001040BA000160EF009B
:109B1000000006000A0D00003E2000005061000019
:109B20006E53000070650000656400003D25000074
:109B3000640A00000D3E0000200000003220EF000B
:109B4000A3DA2400008041001040BA000160EF0059
:109B5000000006000A0D00003E20000054720000C4
:109B60006967000067650000727300002044000010
:109B700069730000616200006C650000640A000007
:109B80000D3E0000200000003220EF0003DD240025
:109B9000008041001040BA000160EF0000000600A4
:109BA0000A0D00003E2000005472000069670000AA
:109BB0006765000072730000204500006E610000C0
:109BC000626C0000656400000A0D00003E20000089
:109BD000000000003220EF0063DF2400008041001D
:109BE0001040BA000160EF00000006000A0D0000FE
:109BF0003E200000546900006C74000053700000A7
:109C000065650000643D0000256400000A0D000049
:109C10003E200000000000003220EF0083E124001D
:109C2000008041001040BA000160EF000000060013
:109C30000A0D00003E2000005A6F00006F6D00000A
:109C40005370000065650000643D0000256400005D
:109C50000A0D00003E200000000000003220EF004E
:109C6000A3E32400008041001040BA000160EF002F
:109C7000000006002020000020200000496E0000A7
:109C800069740000204D000075780000202000005D
:109C9000200000003220EF0063E524000080410036
:109CA0001040BA000160EF00000006002020000014
:109CB00020200000496E000069740000205600005A
:109CC00069640000656F0000202000002020000073
:109CD000000000003220EF0063E724000080410014
:109CE0001040BA000160EF000000060020200000D4
:109CF000496E000069740000205300007562000086
:109D00005379000073740000656D0000202000008E
:109D1000000000003220EF0063E9240000804100D1
:109D20001040BA000160EF00000006000A0D0000BC
:109D30003E53000065740000446500006661000049
:109D4000756C00007420000025640000200A0000EB
:109D50000D3E0000200000003220EF0083EB2400C5
:109D6000008041001040BA000160EF0000000600D2
:109D70000A0D00003E2000005365000072690000DB
:109D8000616C000045630000686F00003D45000005
:109D90006E610000626C0000656400000A0D000046
:109DA0003E200000000000003220EF0003EE2400FF
:109DB000008041001040BA000160EF000000060082
:109DC0000A0D00003E20000053650000726900008B
:109DD000616C000045630000686F00003D440000B6
:109DE00069730000616200006C650000640A000095
:109DF0000D3E0000200000003220EF0083F0240020
:109E0000008041001040BA000160EF000000060031
:109E10000A0D00003E20000053650000726900003A
:109E2000616C0000496E0000666F00003D45000057
:109E30006E610000626C0000656400000A0D0000A5
:109E40003E200000000000003220EF0003F3240059
:109E5000008041001040BA000160EF0000000600E1
:109E60000A0D00003E2000005365000072690000EA
:109E7000616C0000496E0000666F00003D44000008
:109E800069730000616200006C650000640A0000F4
:109E90000D3E0000200000003220EF0083F524007A
:109EA000008041001040BA000160EF000000060091
:109EB000536500006172000063680000696E000075
:109EC00067200000666F00007220000041740000EF
:109ED00074610000636800006564000020430000B6
:109EE000616D000065720000617300000D0A0000E2
:109EF000000000003220EF0063F8240000804100E1
:109F00001040BA000160EF00000006000A0D0000DA
:109F1000506F00007274000020250000643A0000B9
:109F20000A0D0000000000003220EF0003FA2400B8
:109F3000008041001040BA000160EF000000060000
:109F40000A0D0000436100006D65000072610000B1
:109F5000205300006561000072630000682000006B
:109F6000436F00006D7000006C65000074650000B8
:109F70000A0D00000A0000003220EF0083FC2400DC
:109F8000008041001040BA000160EF0000000600B0
:109F900020560000432D00004335000030690000CA
:109FA00020200000205000006F720000742000008C
:109FB00030200000200000003220EF0083FE24004B
:109FC000008041001040BA000160EF000000060070
:109FD000436100006E6F00006E20000044650000C9
:109FE0007465000063740000656400000D0A0000E1
:109FF000000000003220EF006300250000804100D7
:10A000001040BA000160EF0000000600204E000082
:10A010006F200000436100006D2000002020000040
:10A02000205000006F7200007420000030200000FB
:10A03000200000003220EF00630225000080410074
:10A040001040BA000160EF00000006000D0A000099
:10A05000506100006E610000736F00006E690000C7
:10A0600063200000415700002D48000045310000EA
:10A07000303000000D0A0000000000003220EF0028
:10A08000A3042500008041001040BA000160EF00E9
:10A090000000060020410000572D00004845000048
:10A0A0003130000030200000205000006F720000AE
:10A0B0007420000030200000200000003220EF005B
:10A0C000A3062500008041001040BA000160EF00A7
:10A0D00000000600204700006574000038200000E2
:10A0E000000000003220EF00E3072500008041005F
:10A0F0001040BA000160EF000000060020200000C0
:10A10000202D00002D2000002532000058200000E6
:10A110002D2D00000A0D0000000000003220EF008D
:10A12000A3092500008041001040BA000160EF0043
:10A13000000006000A0D000020200000206700003B
:10A140006574000031360000200000003220EF006E
:10A15000230B2500008041001040BA000160EF0091
:10A160000000060020200000202D00002D2000000F
:10A17000254C0000582000002D2D0000200A000072
:10A180000D0000003220EF00E30C250000804100AC
:10A190001040BA000160EF00000006000A0D000048
:10A1A00020200000206700006574000033320000AA
:10A1B000200000003220EF00630E250000804100E7
:10A1C0001040BA000160EF000000060020200000EF
:10A1D000202D00002D200000254C000058200000FC
:10A1E0002D2D00000A0D0000000000003220EF00BD
:10A1F00023102500008041001040BA000160EF00EC
:10A20000000006000A0D000020430000616D000000
:10A210006572000061540000797000006520000044
:10A22000000000003220EF00E31125000080410013
:10A230001040BA000160EF00000006000D0A0000A7
:10A24000536F00006E790000204500005649000061
:10A250002D4400003330000028720000290D00005A
:10A260000A0000003220EF00E313250000804100C7
:10A270001040BA000160EF00000006002045000019
:10A28000564900002D4400003330000028720000C1
:10A29000295000006F720000742000003020000080
:10A2A000200000003220EF00E3152500008041006F
:10A2B0001040BA000160EF0000000600496E000087
:10A2C000766100006C6900006420000043610000BA
:10A2D0006D650000726100000D0A000000000000C2
:10A2E0003220EF00C3172500008041001040BA0063
:10A2F0000160EF0000000600204900006E760000BB
:10A30000616C00006964000020430000616D000082
:10A3100065720000610000003220EF008319250003
:10A32000008041001040BA000160EF00000006000C
:10A330000D0A0000536F00006E79000020450000F8
:10A34000564900002D440000333000002F33000038
:10A35000312000000D0A0000000000003220EF0054
:10A36000A31B2500008041001040BA000160EF00EF
:10A370000000060020450000564900002D44000062
:10A38000333000002F330000315000006F720000A6
:10A390007420000030200000200000003220EF0078
:10A3A000A31D2500008041001040BA000160EF00AD
:10A3B000000006000D0A0000536F00006E790000D7
:10A3C00020450000564900002D44000033300000B5
:10A3D0000D0A0000000000003220EF00831F25005E
:10A3E000008041001040BA000160EF00000006004C
:10A3F00020450000564900002D4400003330000085
:10A4000020200000205000006F7200007420000027
:10A4100030200000200000003220EF0083212500C2
:10A42000008041001040BA000160EF00000006000B
:10A430000D0A00005661000064640000696F0000AE
:10A4400020410000646400002D4100002D43000005
:10A45000616D00000D0A0000000000003220EF00D6
:10A46000A3232500008041001040BA000160EF00E6
:10A470000000060020410000646400002D4100003F
:10A480002D430000616D0000205000006F7200003D
:10A490007420000030200000200000003220EF0077
:10A4A000A3252500008041001040BA000160EF00A4
:10A4B000000006000D0A0000536F00006E790000D6
:10A4C00020450000564900002D44000031300000B6
:10A4D000300D00000A0000003220EF008327250025
:10A4E000008041001040BA000160EF00000006004B
:10A4F00020450000564900002D4400003130000086
:10A5000030200000205000006F7200007420000016
:10A5100030200000200000003220EF0083292500B9
:10A52000008041001040BA000160EF00000006000A
:10A530000D0A0000536F00006E79000020450000F6
:10A54000564900002D440000373000000D0A00007D
:10A55000000000003220EF00632B25000080410046
:10A560001040BA000160EF00000006002045000026
:10A57000564900002D440000373000002020000024
:10A58000205000006F720000742000003020000096
:10A59000200000003220EF00632D250000804100E4
:10A5A0001040BA000160EF00000006000D0A000034
:10A5B000536F00006E7900002042000052430000FB
:10A5C000482D000037300000300D00000A00000068
:10A5D0003220EF00432F2500008041001040BA00D8
:10A5E0000160EF000000060020420000524300001E
:10A5F000482D0000373000003020000020500000BF
:10A600006F72000074200000302000002000000065
:10A610003220EF0043312500008041001040BA0095
:10A620000160EF00000006000D0A0000456C00000C
:10A630006D6F000020430000616D00006572000036
:10A64000610D00000A0000003220EF0003332500F6
:10A65000008041001040BA000160EF0000000600D9
:10A66000204500006C6D00006F20000020200000DD
:10A6700020200000205000006F72000074200000B5
:10A6800030200000200000003220EF0003352500BC
:10A69000008041001040BA000160EF000000060099
:10A6A0000D0A0000536F00006E7900002042000088
:10A6B000524300002D330000303000000D0A00002E
:10A6C000000000003220EF00E3362500008041004A
:10A6D0001040BA000160EF000000060020420000B8
:10A6E000524300002D3300003030000020200000D5
:10A6F000205000006F720000742000003020000025
:10A70000200000003220EF00E338250000804100E7
:10A710001040BA000160EF00000006000D0A0000C2
:10A72000536F00006E790000204200005243000089
:10A730002D5A000037300000300D00000A000000E4
:10A740003220EF00C33A2500008041001040BA00DB
:10A750000160EF00000006002042000052430000AC
:10A760002D5A00003730000030200000205000003B
:10A770006F720000742000003020000020000000F4
:10A780003220EF00C33C2500008041001040BA0099
:10A790000160EF00000006000D0A0000536F00008A
:10A7A0006E79000020420000524300002D5A000044
:10A7B00033330000300D00000A0000003220EF00AB
:10A7C000A33E2500008041001040BA000160EF0068
:10A7D0000000060020420000524300002D5A0000F5
:10A7E0003333000030200000205000006F72000062
:10A7F0007420000030200000200000003220EF0014
:10A80000A3402500008041001040BA000160EF0025
:10A81000000006000D0A000056610000646400009C
:10A82000696F000020480000442D0000313800000E
:10A830000D0A0000000000003220EF0083422500D6
:10A84000008041001040BA000160EF0000000600E7
:10A8500020200000484400002D3100003820000076
:10A8600020200000205000006F72000074200000C3
:10A8700030200000200000003220EF00834425003B
:10A88000008041001040BA000160EF0000000600A7
:10A890000D0A0000536F00006E7900002045000093
:10A8A000564900002D480000443100000D0A000008
:10A8B000000000003220EF006346250000804100C8
:10A8C0001040BA000160EF000000060020450000C3
:10A8D000564900002D4800004431000020200000AF
:10A8E000205000006F720000742000003020000033
:10A8F000200000003220EF00634825000080410066
:10A900001040BA000160EF00000006000D0A0000D0
:10A910005661000064640000696F0000204300007D
:10A92000656900006C6900006E6700005649000010
:10A93000455700000D0A0000000000003220EF0023
:10A94000A34A2500008041001040BA000160EF00DA
:10A950000000060020430000562F00004356000070
:10A960004D50000020200000205000006F720000B9
:10A970007420000030200000200000003220EF0092
:10A98000A34C2500008041001040BA000160EF0098
:10A9900000000600556E00006B6E00006F7700002F
:10A9A0006E200000436100006D65000072610000D0
:10A9B0000D0A0000000000003220EF00834E250049
:10A9C000008041001040BA000160EF000000060066
:10A9D000205500006E6B00006E6F0000776E000067
:10A9E00020200000205000006F7200007420000042
:10A9F00030200000200000003220EF0083502500AE
:10AA0000008041001040BA000160EF000000060025
:10AA10000A0D000020410000542F00004D440000AA
:10AA20005F4D00006F640000654900006E7100001A
:10AA3000200000003220EF0063522500008041001A
:10AA40001040BA000160EF00000006000D0A00008F
:10AA50002057000061690000745300006F6E000011
:10AA600079410000636B0000000000003220EF001D
:10AA700023542500008041001040BA000160EF001F
:10AA8000000006000D0A0000205700006169000068
:10AA9000745300006F6E0000790000003220EF0058
:10AAA000A3552500008041001040BA000160EF006E
:10AAB000000006002A57000061690000745300007E
:10AAC0006F6E0000790000003220EF000357250070
:10AAD000008041001040BA000160EF000000060055
:10AAE0000A0D000057610000697400005265000003
:10AAF00073700000536F00006E7900003A20000070
:10AB0000000000003220EF00E358250000804100E3
:10AB10001040BA000160EF0000000600202D000088
:10AB200020540000696D0000656F0000757400001E
:10AB30002025000075200000286D0000732900000A
:10AB40000D0A0000000000003220EF00035B25002A
:10AB5000008041001040BA000160EF0000000600D4
:10AB6000436100006E630000656C0000205300002C
:10AB700031200000000000003220EF00835C25003F
:10AB8000008041001040BA000160EF0000000600A4
:10AB9000436100006E630000656C000020530000FC
:10ABA00032200000000000003220EF00035E25008C
:10ABB000008041001040BA000160EF000000060074
:10ABC0000A0D0000202000002047000065740000EE
:10ABD0004252000043500000616E000054690000C2
:10ABE0006C740000506F0000732000000000000033
:10ABF0003220EF0043602500008041001040BA0081
:10AC00000160EF000000060020200000202D000061
:10AC10002D200000503A0000254C0000582C000068
:10AC2000543A0000254C0000582000002D2D000053
:10AC30000A0D0000000000003220EF0083622500B2
:10AC4000008041001040BA000160EF0000000600E3
:10AC5000205D00000A0D0000000000003220EF001F
:10AC6000A3632500008041001040BA000160EF009E
:10AC7000000006000D0A0000205700006169000076
:10AC800074430000616E00006F6E00000000000061
:10AC90003220EF0043652500008041001040BA00DB
:10ACA0000160EF0000000600202D0000205400008D
:10ACB000696D0000656F00007574000020250000BC
:10ACC0006C750000202800006D730000290D000045
:10ACD0000A0000003220EF00636725000080410079
:10ACE0001040BA000160EF00000006000D0A0000ED
:10ACF000205700006169000074500000616E000080
:10AD0000617300006F6E00006963000000000000C6
:10AD10003220EF0043692500008041001040BA0056
:10AD20000160EF000000060020200000205300001A
:10AD300059530000544500004D2000004D450000CF
:10AD40004E550000202000002020000000000000E0
:10AD50003220EF00436B2500008041001040BA0014
:10AD60000160EF00000006002020000020530000DA
:10AD700065720000696100006C200000496E0000EF
:10AD8000707500007420000020200000000000000A
:10AD90003220EF00436D2500008041001040BA00D2
:10ADA0000160EF000000060020200000205300009A
:10ADB00065720000696100006C20000045630000BE
:10ADC000686F00002020000020200000000000002C
:10ADD0003220EF00436F2500008041001040BA0090
:10ADE0000160EF000000060020200000205300005A
:10ADF00065720000696100006C200000496E00006F
:10AE0000666F0000202000002020000000000000ED
:10AE10003220EF0043712500008041001040BA004D
:10AE20000160EF000000060020200000205000001C
:10AE3000616E0000656C0000204C00006967000036
:10AE40006874000073200000202000000000000053
:10AE50003220EF0043732500008041001040BA000B
:10AE60000160EF00000006002020000020430000E9
:10AE70006C65000061720000204D0000656D0000EF
:10AE80006F72000079200000202000000000000008
:10AE90003220EF0043752500008041001040BA00C9
:10AEA0000160EF00000006002020000020430000A9
:10AEB0006C650000617200002050000072650000A7
:10AEC0007365000074730000202000000000000083
:10AED0003220EF0043772500008041001040BA0087
:10AEE0000160EF0000000600202000005472000006
:10AEF000616E000073690000746900006F6E0000ED
:10AF000020540000696D0000652000000000000072
:10AF10003220EF0043792500008041001040BA0044
:10AF20000160EF00000006002020000054720000C5
:10AF3000616E000073690000746900006F6E0000AC
:10AF4000204D00006F64000065200000000000003C
:10AF50003220EF00437B2500008041001040BA0002
:10AF60000160EF000000060020200000576900008B
:10AF70007065000020530000656C000065630000F0
:10AF8000746900006F6E00002020000000000000C7
:10AF90003220EF00437D2500008041001040BA00C0
:10AFA0000160EF0000000600202000002053000098
:10AFB00065740000746C0000652000005469000096
:10AFC0006D6500002020000020200000000000002F
:10AFD0003220EF00437F2500008041001040BA007E
:10AFE0000160EF000000060020200000202000008B
:10AFF00020200000546100006C6C000079200000EB
:10B000002020000020200000202000000000000080
:10B010003220EF0043812500008041001040BA003B
:10B020000160EF000000060020200000496E0000D3
:10B030006974000020540000726900006767000016
:10B040006572000073200000202000000000000056
:10B050003220EF0043832500008041001040BA00F9
:10B060000160EF00000006002020000020500000DA
:10B070007265000073650000742000003637000020
:10B080002D370000322000002020000000000000CA
:10B090003220EF0043852500008041001040BA00B7
:10B0A0000160EF0000000600205600004944000047
:10B0B000454F0000204900004E500000555400004C
:10B0C000204D0000454E000055200000000000000B
:10B0D0003220EF0043872500008041001040BA0075
:10B0E0000160EF0000000600202000004341000046
:10B0F0004D2000005345000041520000434800002D
:10B10000204D0000454E00005520000000000000CA
:10B110003220EF0043892500008041001040BA0032
:10B120000160EF0000000600202000002020000049
:10B13000204100006C6C0000205000006F72000085
:10B140007473000020200000202000000000000098
:10B150003220EF00438B2500008041001040BA00F0
:10B160000160EF0000000600202000002020000009
:10B1700020200000506F000072740000203000009A
:10B1800031200000202000002020000000000000EE
:10B190003220EF00438D2500008041001040BA00AE
:10B1A0000160EF00000006002020000020200000C9
:10B1B00020200000506F000072740000203000005A
:10B1C00032200000202000002020000000000000AD
:10B1D0003220EF00438F2500008041001040BA006C
:10B1E0000160EF0000000600202000002020000089
:10B1F00020200000506F000072740000203000001A
:10B20000332000002020000020200000000000006B
:10B210003220EF0043912500008041001040BA0029
:10B220000160EF0000000600202000002020000048
:10B2300020200000506F00007274000020300000D9
:10B24000342000002020000020200000000000002A
:10B250003220EF0043932500008041001040BA00E7
:10B260000160EF0000000600202000002020000008
:10B2700020200000506F0000727400002030000099
:10B2800035200000202000002020000000000000E9
:10B290003220EF0043952500008041001040BA00A5
:10B2A0000160EF00000006002020000020200000C8
:10B2B00020200000506F0000727400002030000059
:10B2C00036200000202000002020000000000000A8
:10B2D0003220EF0043972500008041001040BA0063
:10B2E0000160EF0000000600202000002020000088
:10B2F000204D0000414900004E2000004D45000057
:10B300004E5500002020000020200000000000001A
:10B310003220EF0043992500008041001040BA0020
:10B320000160EF00000006002020000052650000D0
:10B3300073630000616E000020430000616D000037
:10B340006572000061730000202000000000000012
:10B350003220EF00439B2500008041001040BA00DE
:10B360000160EF00000006002020000020520000D5
:10B3700065730000636100006E20000056690000E4
:10B38000646500006F200000202000000000000025
:10B390003220EF00439D2500008041001040BA009C
:10B3A0000160EF0000000600202000002056000091
:10B3B00069640000656F0000204F00007574000094
:10B3C00070750000742000002020000000000000C4
:10B3D0003220EF00439F2500008041001040BA005A
:10B3E0000160EF00000006002056000069640000C4
:10B3F000656F0000204900006E7000007574000049
:10B40000204D0000656E0000752000000000000067
:10B410003220EF0043A12500008041001040BA0017
:10B420000160EF00000006002053000044200000EF
:10B4300056690000646500006F200000466F000040
:10B44000726D000061740000202000000000000008
:10B450003220EF0043A32500008041001040BA00D5
:10B460000160EF0000000600204400006566000057
:10B47000617500006C7400002050000072650000CF
:10B4800073650000742000004E6F00000000000093
:10B490003220EF0043A52500008041001040BA0093
:10B4A0000160EF00000006002020000020440000A2
:10B4B00065660000617500006C7400002054000097
:10B4C000696D00006572000020200000000000008F
:10B4D0003220EF0043A72500008041001040BA0051
:10B4E0000160EF00000006002050000072650000BF
:10B4F0007365000074200000506100006E200000A1
:10B50000537000006565000064200000000000002A
:10B510003220EF0043A92500008041001040BA000E
:10B520000160EF000000060020500000726500007E
:10B530007365000074200000546900006C74000002
:10B5400020530000706500006564000000000000EA
:10B550003220EF0043AB2500008041001040BA00CC
:10B560000160EF000000060020500000726500003E
:10B5700073650000742000005A6F00006F6D0000BA
:10B5800020530000706500006564000000000000AA
:10B590003220EF0043AD2500008041001040BA008A
:10B5A0000160EF0000000600202000004361000061
:10B5B0006D200000536500006172000063680000A8
:10B5C000204D0000656E00007520000000000000A6
:10B5D0003220EF0043AF2500008041001040BA0048
:10B5E0000160EF0000000600202000002020000085
:10B5F0005379000073740000656D0000204D000059
:10B60000656E000075200000202000000000000092
:10B610003220EF0043B12500008041001040BA0005
:10B620000160EF0000000600202000002041000023
:10B63000757400006F540000726100006B20000000
:10B64000496E0000707500007420000000000000CA
:10B650003220EF0043B32500008041001040BA00C3
:10B660000160EF0000000600202000002020000004
:10B67000504900005020000054720000696700002B
:10B68000676500007220000020200000000000001C
:10B690003220EF0043B52500008041001040BA0081
:10B6A0000160EF000000060020500000495000003B
:10B6B0002054000072690000676700006572000096
:10B6C000204D00006F6400006520000000000000B5
:10B6D0003220EF0043B72500008041001040BA003F
:10B6E0000160EF0000000600202000002020000084
:10B6F00020200000537400006172000074200000DC
:10B700002020000020200000202000000000000079
:10B710003220EF0043B92500008041001040BA00FC
:10B720000160EF0000000600204E00006F74000072
:10B730002041000076610000696C00006162000039
:10B740006C650000202000002020000000000000A8
:10B750003220EF0043BB2500008041001040BA00BA
:10B760000160EF0000000600202000004D6F000087
:10B770006D6500006E7400006172000079200000A9
:10B7800020200000202000002020000000000000F9
:10B790003220EF0043BD2500008041001040BA0078
:10B7A0000160EF0000000600202000004C61000056
:10B7B0007463000068650000642000002020000021
:10B7C00020200000202000002020000000000000B9
:10B7D0003220EF0043BF2500008041001040BA0036
:10B7E0000160EF00000006002053000071750000AA
:10B7F000656500007A650000202000002020000020
:10B800002020000020200000202000000000000078
:10B810003220EF0043C12500008041001040BA00F3
:10B820000160EF0000000600204C0000657400007D
:10B830007465000072200000426F00007820000054
:10B840002020000020200000202000000000000038
:10B850003220EF0043C32500008041001040BA00B1
:10B860000160EF000000060020430000726F00003E
:10B870007020000020200000202000002020000078
:10B8800020200000202000002020000000000000F8
:10B890003220EF0043C52500008041001040BA006F
:10B8A0000160EF0000000600204800004420000076
:10B8B00031300000383000007020000035390000C1
:10B8C0002E390000344800007A20000000000000FB
:10B8D0003220EF0043C72500008041001040BA002D
:10B8E0000160EF0000000600204800004420000036
:10B8F000313000003830000070200000353000008A
:10B90000487A0000202000002020000000000000F5
:10B910003220EF0043C92500008041001040BA00EA
:10B920000160EF00000006002048000044200000F5
:10B930003130000038300000692000003539000047
:10B940002E390000344800007A200000000000007A
:10B950003220EF0043CB2500008041001040BA00A8
:10B960000160EF00000006002048000044200000B5
:10B970003130000038300000692000003530000010
:10B98000487A000020200000202000000000000075
:10B990003220EF0043CD2500008041001040BA0066
:10B9A0000160EF0000000600204800004420000075
:10B9B00020370000323000007020000035390000D0
:10B9C0002E390000344800007A20000000000000FA
:10B9D0003220EF0043CF2500008041001040BA0024
:10B9E0000160EF0000000600204800004420000035
:10B9F0002037000032300000702000003530000099
:10BA0000487A0000202000002020000000000000F4
:10BA10003220EF0043D12500008041001040BA00E1
:10BA20000160EF00000006002048000056200000E2
:10BA30002036000034300000782000003438000048
:10BA40003020000036300000487A0000000000007E
:10BA50003220EF0043D32500008041001040BA009F
:10BA60000160EF00000006002048000056200000A2
:10BA70002038000030300000782000003630000010
:10BA80003020000036300000487A0000000000003E
:10BA90003220EF0043D52500008041001040BA005D
:10BAA0000160EF0000000600204800005620000062
:10BAB00031300000323400007820000037360000BA
:10BAC0003820000036300000487A000000000000F6
:10BAD0003220EF0043D72500008041001040BA001B
:10BAE0000160EF0000000600204800005620000022
:10BAF0003132000038300000782000003736000076
:10BB00003820000036300000487A000000000000B5
:10BB10003220EF0043D92500008041001040BA00D8
:10BB20000160EF00000006002048000056200000E1
:10BB3000313200003830000078310000303200002F
:10BB40003420000036300000487A00000000000079
:10BB50003220EF0043DB2500008041001040BA0096
:10BB60000160EF00000006002048000056200000A1
:10BB700031390000323000007831000032300000EE
:10BB80003020000036300000487A0000000000003D
:10BB90003220EF0043DD2500008041001040BA0054
:10BBA0000160EF0000000600205300004420000068
:10BBB0004E5400005343000020320000392E000094
:10BBC00039370000487A0000202000000000000003
:10BBD0003220EF0043DF2500008041001040BA0012
:10BBE0000160EF0000000600205300004420000028
:10BBF000504100004C2000002020000032350000A1
:10BC0000487A0000202000002020000000000000F2
:10BC10003220EF0043E12500008041001040BA00CF
:10BC20000160EF00000006002053000044200000E7
:10BC300034380000306900002020000079500000F6
:10BC40006250000072200000202000000000000070
:10BC50003220EF0043E32500008041001040BA008D
:10BC60000160EF00000006002053000044200000A7
:10BC700035370000366900002020000079500000B0
:10BC80006250000072200000202000000000000030
:10BC90003220EF0043E52500008041001040BA004B
:10BCA0000160EF00000006002020000020200000BE
:10BCB00020200000202000004F4E00002020000027
:10BCC00020200000202000002020000000000000B4
:10BCD0003220EF0043E72500008041001040BA0009
:10BCE0000160EF000000060020200000202000007E
:10BCF00020200000204F00004646000020200000C9
:10BD00002020000020200000202000000000000073
:10BD10003220EF0043E92500008041001040BA00C6
:10BD20000160EF000000060020200000202000003D
:10BD300020200000204700006C6F000062610000BE
:10BD40006C200000202000002020000000000000E7
:10BD50003220EF0043EB2500008041001040BA0084
:10BD60000160EF00000006002020000020200000FD
:10BD70002020000042790000205000007265000081
:10BD80007365000074200000202000000000000007
:10BD90003220EF0043ED2500008041001040BA0042
:10BDA0000160EF000000060020200000205200008B
:10BDB0006967000068740000207400006F200000B4
:10BDC0004C650000667400002020000000000000A8
:10BDD0003220EF0043EF2500008041001040BA0000
:10BDE0000160EF000000060020200000204C000051
:10BDF0006566000074200000746F0000205200008F
:10BE00006967000068740000202000000000000046
:10BE10003220EF0043F12500008041001040BA00BD
:10BE20000160EF0000000600202000002054000008
:10BE30006F700000207400006F200000426F00004F
:10BE4000747400006F6D00002020000000000000EE
:10BE50003220EF0043F32500008041001040BA007B
:10BE60000160EF00000006002020000020420000DA
:10BE70006F740000746F00006D200000746F00008C
:10BE8000205400006F70000020200000000000001F
:10BE90003220EF0043F52500008041001040BA0039
:10BEA0000160EF0000000600204400006E52000018
:10BEB0006967000068740000207400006F200000B3
:10BEC000557000004C650000667400000000000022
:10BED0003220EF0043F72500008041001040BA00F7
:10BEE0000160EF0000000600204400006E4C0000DE
:10BEF0006566000074200000746F0000205500008B
:10BF000070520000696700006874000000000000C3
:10BF10003220EF0043F92500008041001040BA00B4
:10BF20000160EF0000000600205500007052000084
:10BF30006967000068740000207400006F20000032
:10BF4000446E00004C6500006674000000000000B4
:10BF50003220EF0043FB2500008041001040BA0072
:10BF60000160EF000000060020550000704C00004A
:10BF70006566000074200000746F0000204400001B
:10BF80006E52000069670000687400000000000045
:10BF90003220EF0043FD2500008041001040BA0030
:10BFA0000160EF0000000600204100006C6C000002
:10BFB000536900006465000073200000746F000086
:10BFC00020430000656E00007420000000000000A7
:10BFD0003220EF0043FF2500008041001040BA00EE
:10BFE0000160EF0000000600204C000065660000C4
:10BFF000743E0000436500006E740000657200002E
:10C000003C520000696700006874000000000000F6
:10C010003220EF0043012600008041001040BA00AA
:10C020000160EF0000000600205400006F70000067
:10C030003E430000656E000074650000723C000025
:10C04000426F0000747400006F6D0000000000007B
:10C050003220EF0043032600008041001040BA0068
:10C060000160EF00000006002020000020200000FA
:10C07000416300007469000076650000204C0000F8
:10C080006F7700002020000020200000000000004A
:10C090003220EF0043052600008041001040BA0026
:10C0A0000160EF00000006002020000020200000BA
:10C0B00041630000746900007665000020480000BC
:10C0C00069670000682000002020000000000000D8
:10C0D0003220EF0043072600008041001040BA00E4
:10C0E0000160EF000000060020430000616D0000C9
:10C0F000205000007265000073650000747300003A
:10C10000204F00004E200000202000000000000012
:10C110003220EF0043092600008041001040BA00A1
:10C120000160EF000000060020430000616D000088
:10C1300020500000726500007365000074730000F9
:10C14000204F0000464600002020000000000000B4
:10C150003220EF00430B2600008041001040BA005F
:10C160000160EF000000060020200000204E0000CB
:10C170006F7400002053000075700000706F0000A5
:10C1800072740000656400002020000000000000C0
:10C190003220EF00430D2600008041001040BA001D
:10C1A0000160EF0000000600205300004420000062
:10C1B0004E540000534300002D280000532D000072
:10C1C00056690000646500006F290000000000004F
:10C1D0003220EF00430F2600008041001040BA00DB
:10C1E0000160EF0000000600205300004420000022
:10C1F00020500000414C00002D280000532D00006D
:10C2000056690000646500006F290000000000000E
:10C210003220EF0043112600008041001040BA0098
:10C220000160EF00000006002053000044200000E1
:10C230004E54000053430000204300006F6D000087
:10C24000706F00007369000074650000000000005A
:10C250003220EF0043132600008041001040BA0056
:10C260000160EF00000006002053000044200000A1
:10C2700020500000414C0000204300006F6D000082
:10C28000706F00007369000074650000000000001A
:10C290003220EF0043152600008041001040BA0014
:10C2A0000160EF00000006002041000075740000EE
:10C2B0006F20000053650000617200006368000099
:10C2C000204D00006F6400006520000000000000A9
:10C2D0003220EF0043172600008041001040BA00D2
:10C2E0000160EF0000000600202000002020000078
:10C2F000205300006F6E0000792000004F6E000098
:10C300006C790000202000002020000000000000C8
:10C310003220EF0043192600008041001040BA008F
:10C320000160EF0000000600202000002020000037
:10C33000436100006E6F00006E2000004F6E000031
:10C340006C79000020200000202000000000000088
:10C350003220EF00431B2600008041001040BA004D
:10C360000160EF0000000600202000005061000086
:10C370006E610000736F00006E69000063200000B2
:10C380004F6E00006C7900002020000000000000CB
:10C390003220EF00431D2600008041001040BA000B
:10C3A0000160EF0000000600202000004E6F00003A
:10C3B00020430000616D00006572000061200000F4
:10C3C000496E00007075000074200000000000003D
:10C3D0003220EF00431F2600008041001040BA00C9
:10C3E0000160EF0000000600205300007973000098
:10C3F000746500006D200000496E000020530000AD
:10C40000746100006E6400006279000000000000AA
:10C410003220EF0043212600008041001040BA0086
:10C420000160EF0000000600202000002020000036
:10C430002020000020300000256300002073000051
:10C4400065630000202000002020000000000000A4
:10C450003220EF0043232600008041001040BA0044
:10C460000160EF00000006002020000020200000F6
:10C47000202E0000302500006330000020730000F3
:10C480006563000020200000202000000000000064
:10C490003220EF0043252600008041001040BA0002
:10C4A0000160EF00000006002020000020200000B6
:10C4B000203000002E2500006330000020730000B3
:10C4C0006563000020200000202000000000000024
:10C4D0003220EF0043272600008041001040BA00C0
:10C4E0000160EF0000000600202000002020000076
:10C4F00020200000202000002025000063200000F4
:10C50000202000002020000020200000000000006B
:10C510003220EF0043292600008041001040BA007D
:10C520000160EF0000000600202000002020000035
:10C53000202000002025000063250000632000006B
:10C540007365000063200000202000002000000030
:10C550003220EF00432B2600008041001040BA003B
:10C560000160EF00000006002020000020200000F5
:10C57000202E00002563000025630000302000000D
:10C5800073650000632000002020000020000000F0
:10C590003220EF00432D2600008041001040BA00F9
:10C5A0000160EF00000006002020000020200000B5
:10C5B00020250000632E00002563000030200000CD
:10C5C00073650000632000002020000020000000B0
:10C5D0003220EF00432F2600008041001040BA00B7
:10C5E0000160EF0000000600202000002020000075
:10C5F00020200000202500006325000063200000AB
:10C60000202000002020000020200000000000006A
:10C610003220EF0043312600008041001040BA0074
:10C620000160EF0000000600202000002020000034
:10C630002020000025630000256300002563000022
:10C64000207300006563000020200000000000004F
:10C650003220EF0043332600008041001040BA0032
:10C660000160EF00000006002020000020200000F4
:10C67000202E0000256300002563000025630000D4
:10C68000207300006563000020200000000000000F
:10C690003220EF0043352600008041001040BA00F0
:10C6A0000160EF00000006002020000020200000B4
:10C6B00025630000256300002E2500006330000084
:10C6C00020730000656300002020000000000000CF
:10C6D0003220EF0043372600008041001040BA00AE
:10C6E0000160EF0000000600202000002020000074
:10C6F00020200000202500006325000063250000A5
:10C700006320000020200000202000000000000026
:10C710003220EF0043392600008041001040BA006B
:10C720000160EF00000006004F5300004346000088
:10C73000414900004C5F000045520000524F00008C
:10C74000520A00000D0000003220EF00033B2600DB
:10C75000008041001040BA000160EF0000000600B8
:10C76000414400004452000045520000525F000066
:10C7700045520000524F0000520A00000D00000018
:10C780003220EF00C33C2600008041001040BA0078
:10C790000160EF0000000600535400004143000018
:10C7A0004B450000525200005F450000525200000D
:10C7B0004F5200000A0D0000000000003220EF0080
:10C7C000A33E2600008041001040BA000160EF0047
:10C7D000000006004D410000544800004552000092
:10C7E000525F000045520000524F0000520A000004
:10C7F0000D0000003220EF00634026000080410061
:10C800001040BA000160EF0000000600444D000037
:10C8100041450000525200005F45000052520000A6
:10C820004F5200000A0D0000000000003220EF000F
:10C8300023422600008041001040BA000160EF0052
:10C840000000060020200000204200006567000074
:10C85000696E0000204E00006F770000202000006D
:10C860002020000020200000000000003220EF0007
:10C8700023442600008041001040BA000160EF0010
:10C8800000000600202000002020000020250000DD
:10C89000730000003220EF00634526000080410055
:10C8A0001040BA000160EF000000060020490000BF
:10C8B0006E69000074690000616C00007A65000018
:10C8C0002045000045500000726F00006D20000000
:10C8D000000000003220EF00634726000080410086
:10C8E0001040BA000160EF00000006002045000083
:10C8F00045500000726F00006D200000496E00007E
:10C9000069740000696100006C7A000065640000D1
:10C91000200000003220EF00634926000080410023
:10C920001040BA000160EF0000000600204C00003B
:10C930006F610000646900006E6700002044000021
:10C9400065660000617500006C74000073200000D3
:10C95000000000003220EF00634B26000080410001
:10C960001040BA000160EF00000006002020000027
:10C970002020000020520000657300006574000054
:10C98000204D000075780000202500007520000073
:10C99000000000004200F8003600F800801F780018
:10C9A000200020000C000900B01F780001002000CA
:10C9B0000100780088630200000000008100E800A8
:10C9C000811F78002322AF00FEFF3700201188006E
:10C9D000CF007800E00020000008E600F4FF3700F8
:10C9E0008020A9008020A900A00120000C000900DF
:10C9F0004F1078004F0078003600F9004200F9002F
:10CA0000004006004200F8003600F800801F780061
:10CA1000200020000C000900B01F78000100200059
:10CA200001007800A4630200000000008100E8001B
:10CA3000811F78002322AF00FEFF370020118800FD
:10CA4000CF007800E00020000008E600F4FF370087
:10CA50008060A9008060A900A00120000C000900EE
:10CA60004F1078004F0078003600F9004200F900BE
:10CA7000004006004200F8003600F800801F7800F1
:10CA8000200020000C000900B01F780001002000E9
:10CA900001007800C0630200000000008100E8008F
:10CAA000811F78002322AF00FEFF3700201188008D
:10CAB000CF007800F00020000008E600F4FF370007
:10CAC0008040A9008040A900A00120000C000900BE
:10CAD0004F1078004F0078003600F9004200F9004E
:10CAE000004006004200F8003600F800801F780081
:10CAF000200020000C000900B01F78000100200079
:10CB000001007800DE630200000000008100E80000
:10CB1000811F78002322AF00FEFF3700201188001C
:10CB2000CF007800E00020000008E600F4FF3700A6
:10CB30008080A9008080A900A00120000C000900CD
:10CB40004F1078004F0078003600F9004200F900DD
:10CB5000004006004200F8003600F800801F780010
:10CB6000200020000C000900B01F78000100200008
:10CB700001007800FA630200000000008100E80074
:10CB8000811F78002322AF00FEFF370020118800AC
:10CB9000CF007800D00020000008E600F4FF370046
:10CBA00080A0A90080A0A900A00120000C0009001D
:10CBB0004F1078004F0078003600F9004200F9006D
:10CBC000004006004200F8003600F800801F7800A0
:10CBD000200020000C000900B01F780053CFBF00D8
:10CBE0000160EF004100DD00E4EF2000840240001E
:10CBF000A4088000840298001421EF00947A800039
:10CC00004822DE0083022000041CE10004003600FC
:10CC100000003700536FEC001266040000000000B3
:10CC2000536FEF008680A900A00120000C000900CE
:10CC30004F1078004F0078003600F9004200F900EC
:10CC4000004006004200F8003600F800801F78001F
:10CC5000200020000C000900B01F78000400200014
:10CC6000542C890004002000642C8900040020005A
:10CC7000742C8900802C810000C0B300802C8900B6
:10CC8000802C81000160EF00802C8900902C8100B5
:10CC900000C0B300902C8900902C81000160EF004F
:10CCA000902C8900A02C810000C0B300A02C89002A
:10CCB000A02C81000160EF00A02C8900B02C810025
:10CCC00000C0B300B02C89009500A900000828001E
:10CCD000E422B700E602F8008A25F900502C810012
:10CCE000000278000008280004006000602C890021
:10CCF000602C8100BA8DB600702C8900702C8100E8
:10CD00000000E0004100320000003700702C81007C
:10CD10009225F800F0FF9F009225F9008E25F8007B
:10CD20004F0078004800DE009425F800E0FF9F00E7
:10CD30009425F900902C81004800DE00A42C81008D
:10CD40000960EF00044068009025F800F0FF9F00A4
:10CD50009025F900BACDBF009425F800F0FF9F00A0
:10CD60009425F900BBCDBF009625F800E0FF9F0099
:10CD70009625F900A02C81000160EF00A42C810011
:10CD80004822DE00044068009225F800E0FF9F0082
:10CD90009225F900602C81009225F800F0FF9F0099
:10CDA0009225F900902C81004800DE00B42C81000F
:10CDB0000960EF00044068009025F800E0FF9F0044
:10CDC0009025F900842C810004F0A70001003700B1
:10CDD00008003700842C81000470A6000100370091
:10CDE00003003700BE2DED00FA66040000000000CD
:10CDF000BE2DEC008C25F800BA0DF900A86CA80037
:10CE0000BC2DEF000867040000000000BC2DEC0002
:10CE10000628EC0034408000037D20000418E10067
:10CE200019003E00000037000628EF0010A8AF00F0
:10CE300001003700040037000868EF008500A900F2
:10CE40009500A800120037001028AF00010037003D
:10CE5000090037000868EC00DBCABF0044408000CE
:10CE60000024E10004003900000037001008A80089
:10CE70001028A9000868EF00562FAF000100370006
:10CE8000010037000968EC008500A9009500A800A2
:10CE90008500A900A00120000C0009004F107800B7
:10CEA0004F0078003600F9004200F900004006000B
:10CEB0004200F8003600F800801F780020002000B3
:10CEC0000C000900B01F7800502C810000C0B30096
:10CED000502C89002202AE00FEFF37003011800086
:10CEE0008A25F800E0FF9F008A25F900C4418000F0
:10CEF0004822DE00E3B6200083024200502C81006D
:10CF000080429800C44180004822DE00E3B6200041
:10CF100003004200104278006D24E10004003A0052
:10CF200000003700EE6BEC0010C0B30011E8B70052
:10CF3000C44180004822DE00614242000440780083
:10CF400000E0B700040820000024E10004003E00D7
:10CF5000000037003968EF00B267040000000000ED
:10CF60003968EC0010C8A8002E0AAE000100370096
:10CF70004E003700D04AAF00010037004B003700A9
:10CF8000502C81000160EF00140220000024E10019
:10CF900001003A000C003700502C81000160EF00C6
:10CFA000240220000024E10001003A0006003700BE
:10CFB000502C81000160EF00040320000024E100F8
:10CFC00010003A0000003700745F80004822DE0045
:10CFD00013082000041CE1000A003E000000370096
:10CFE000745F80004822DE0093082000041CE100EA
:10CFF0000400390000003700502C810000C0B3004D
:10D00000502C8900502C81000160EF006804E10081
:10D0100001003A0006003700502C81000160EF004B
:10D02000F40720000024E10010003A00000037005F
:10D0300080C0B3002322AF00FEFF370024E2B70018
:10D040002562EF0000C2B3002322AF00FEFF3700CD
:10D0500024E2B7002562EF0080C0B3002322AF00B6
:10D06000FEFF370024E2B7002562EF00502C81005C
:10D070000160EF007F04E1000C0036000000370083
:10D08000502C81000160EF00F40720000024E10033
:10D090000600360000003700502C81002322AF002C
:10D0A000FEFF370024E2B7002562EF00502C81001C
:10D0B000EFEBB7009560A8008560A900A0012000F3
:10D0C0000C0009004F1078004F0078003600F9007E
:10D0D0004200F900004006004200F8003600F80067
:10D0E000801F7800200020000C000900B01F78008D
:10D0F000502C810000C0B300502C89003202AE00D9
:10D10000FEFF3700B01180008A25F800E0FF9F0085
:10D110008A25F900846380000960EF0003BF2000C6
:10D1200083024200502C810080429800846380007A
:10D130000960EF0003BF20000300420010427800A6
:10D140006D24E10004003A0000003700726CEC002E
:10D1500020C0B30011E8B700846380006142420040
:10D160000440780000E0B700040820000024E1003B
:10D1700004003E0000003700706CEF00C46804003B
:10D1800000000000706CEC0010E8A8002E0AAE0051
:10D190000100370048003700D04AAF0001003700D7
:10D1A00045003700502C81000160EF001402200080
:10D1B0000024E10001003A000C003700502C8100EF
:10D1C0000160EF00240220000024E10001003A0089
:10D1D00006003700502C81000160EF00040320009E
:10D1E0000024E10010003A00000037009463800042
:10D1F0004822DE0013082000041CE1000A003E0063
:10D2000000003700946380004822DE00930820006D
:10D21000041CE1000400390000003700502C81009C
:10D2200000C0B300502C8900502C81000160EF0039
:10D230006804E10010003A0000003700502C810023
:10D240003322AF00FEFF370034E2B7003562EF0053
:10D2500000C2B3003322AF00FEFF370034E2B70054
:10D260003562EF00502C81003322AF00FEFF370003
:10D2700034E2B7003562EF00502C81000160EF000E
:10D280007F04E1000C00360000003700502C8100C4
:10D290000160EF00F40720000024E10006003600E2
:10D2A00000003700502C81003322AF00FEFF370012
:10D2B00034E2B7003562EF00502C810073ECB70008
:10D2C00097C0A80087C0A900A00120000C00090099
:10D2D0004F1078004F0078003600F9004200F90046
:10D2E00000400600949C80006124E10004003A00A4
:10D2F000D262A900D662A90084690400000000007F
:10D30000D262A900D662A800D222A900D622A80023
:10D31000D642A900D242A9001E0009000000000068
:10D32000D822EF0093D3BF00DCE2B700DD62EF004C
:10D330001E00090000000000D642A800D242A90049
:10D340001E000900000000000000060000CBB30032
:10D350008BF3B7008C13A800549C80006924E10073
:10D360000300360080C0B3008AF3B7008C13A90015
:10D370008BD3BF008A53B4008BF3B70010C0B30047
:10D3800092F3B7008BD3BF0093F3B700726902002A
:10D39000000000000040EB008C13AF000000E8002C
:10D3A00000000600851F78008B73EF008C73EF0080
:10D3B0008D13A800549C800033082000041CE10059
:10D3C0000300310030C8B3008AF3B7008D13A90001
:10D3D0008AD3BF008BF3B7008AD3BF000160EF0090
:10D3E0004400DE00704070008CF3B70010C0B30042
:10D3F00092F3B7008CD3BF0093F3B70072690200B9
:10D4000000000000A0002000E60302000000000071
:10D410008AD3BF00EF42600010C0B30092F3B700A0
:10D420000540780093F3B700726902000000000025
:10D43000A0002000E6030200000000000040EB0016
:10D440008D13AF000000E800CF0278000000060056
:10D450007B72EF007C72EF00D49380006824E100BF
:10D460000400360080C0B3007BF2B7003E6A0400BF
:10D47000000000007AD2BF007BF2B7007AD2BF0072
:10D480008AF3B700A6690200000000008A73EF006B
:10D49000D2690200000000007C72EF00E49380007B
:10D4A00043082000041CE100070036009273EF00DF
:10D4B0009373EF0072690200000000007C72EC00C0
:10D4C0004E6A04000000000010C0B30000E0B70086
:10D4D000000006004C72EF004C72EF006492800076
:10D4E0006924E100070031004CD2BF007AF2B70096
:10D4F000286A0200000000004C72EC006E6A040012
:10D50000000000000000060010C0B30092F3B70056
:10D51000E0CAB30093F3B700726902000000000094
:10D52000D282A900D682A9003E01090000000000B5
:10D53000D282A900D682A800803E2000E603020025
:10D540000000000010C0B30092F3B70080C2B30027
:10D5500093F3B700726902000000000010C0B3002E
:10D5600092F3B70020CEB30093F3B70072690200C4
:10D570000000000010C0B30092F3B70000C1B30078
:10D5800093F3B700726902000000000010C0B300FE
:10D5900092F3B7009373EF0072690200000000007D
:10D5A00010C0B30092F3B70000CBB30093F3B70001
:10D5B000726902000000000010C0B30092F3B700CF
:10D5C00000C4B30093F3B7007269020000000000CA
:10D5D00010C0B30092F3B70010CAB30093F3B700C2
:10D5E000726902000000000010C0B30092F3B7009F
:10D5F00000CCB30093F3B700726902000000000092
:10D6000010C0B30092F3B700F0CAB30093F3B700B1
:10D61000726902000000000040062000E6030200DC
:10D620000000000010C0B30092F3B70070CEB3004A
:10D6300093F3B70072690200000000006A6A0200FA
:10D640000000000020032000E603020000000000AC
:10D6500000000600851F78008D73EF008E73EF00C9
:10D66000649C800003022000041CE10020003E00B6
:10D67000649C8000F3032000041CE1001C003900BE
:10D68000649C80000442B100044078008DF3B70030
:10D690008E73EF00749C80006524E100120031005D
:10D6A000649C80004822DE006520B800800278007B
:10D6B000749C80000960EF0004804200E484200034
:10D6C00004004000904278009273EF00054078001B
:10D6D00093F3B70072690200000000008E73EC0043
:10D6E0004A6B040000000000366C040000000000DB
:10D6F000649C800003042000041CE10020003E0024
:10D70000649C8000F3052000041CE1001C0039002B
:10D71000649C80000444B100044078008DF3B7009D
:10D720008E73EF00749C80006524E10012003100CC
:10D73000649C80004822DE006520B80080027800EA
:10D74000749C80000960EF0004804200E48E200099
:10D7500004004000904278009273EF00054078008A
:10D7600093F3B70072690200000000008E73EC00B2
:10D77000926B040000000000366C04000000000002
:10D78000649C800003062000041CE10020003E0091
:10D79000649C8000F3072000041CE1001C00390099
:10D7A000649C80000446B100044078008DF3B7000B
:10D7B0008E73EF00749C80006524E100120031003C
:10D7C000649C80004822DE006520B800800278005A
:10D7D000749C80000960EF0004804200E4982000FF
:10D7E00004004000904278009273EF0005407800FA
:10D7F00093F3B70072690200000000008E73EC0022
:10D80000DA6B040000000000366C04000000000029
:10D810008D73EF008E73EF00749C80006524E1002F
:10D8200012003100649C80004822DE006520B800B0
:10D8300080027800749C80000960EF000480420040
:10D84000E484200004004000904278009273EF00CE
:10D850000540780093F3B7007269020000000000F1
:10D860008E73EC000C6C04000000000010C0B300CC
:10D8700000E0B700CF02780000000600851F7800A6
:10D880008373EF007ED3BF008AF3B700A66902005E
:10D89000000000007FD3BF008AF3B700D269020006
:10D8A000000000008373EF0083D3BF00149C80004E
:10D8B0000024E10015003400149C80004822DE00A2
:10D8C000040078008013B400904278008C13F800B4
:10D8D000E5FF9F008C13F9002A6B02000000000096
:10D8E0009273EF009373EF00726902000000000072
:10D8F0009273EF009373EF00726902000000000062
:10D900008373EC00546C040000000000CF02780028
:10D9100000000600F0FF2F000862AE00050037008F
:10D9200009C2AF00FEFF37001110880009C2AF0026
:10D93000FEFF37000000200009E2AF000000E80011
:10D94000000006000862AE00040037000622A800AE
:10D950000622AF00FEFF3700030037000602A800D2
:10D960000602AF00FEFF3700C11181008A6C020081
:10D97000000000003822F800CF007800C808DE0060
:10D980008A6C020000000000D11181008A6C020044
:10D9900000000000F00120000602B600FDFF3A0082
:10D9A0000642A8000642AF00FEFF3700BE00090095
:10D9B0000000000000000600F0FF2F000862AE002B
:10D9C00011003700321080007F016100FDFF3A0036
:10D9D0000662A8000100A70006A2A9000100A60097
:10D9E00006A2A800321080007F016100FDFF3A000E
:10D9F0000682A8000822AE00FEFF3700001080005B
:10DA000008C2AF0008C2A90000000600851F780008
:10DA10000862AE00040037000622A8000622AF000C
:10DA2000FEFF3700030037000602A8000602AF0021
:10DA3000FEFF3700A19A80008A6C020000000000FF
:10DA400055D3BF00800078008A6C020000000000FF
:10DA50000862AE00040037000622A8000622AF00CC
:10DA6000FEFF3700030037000602A8000602AF00E1
:10DA7000FEFF370054D3BF00E142700085407800BC
:10DA80008A6C020000000000B59A800001002000AE
:10DA9000811F7800CF007800DC6C020000000000DD
:10DAA000804A7800F00120000602B600FDFF3A002F
:10DAB0000642A8000642AF00FEFF3700BE00090084
:10DAC00000000000B59A80000540900000E0B7001B
:10DAD000CF02780000000600F0FF2F001862AE00B1
:10DAE0000500370019C2AF00FEFF37009110880013
:10DAF00019C2AF00FEFF37000000200019E2AF009E
:10DB00000000E800000006001862AE0004003700C4
:10DB10001622A8001622AF00FEFF370003003700D0
:10DB20001602A8001602AF00FEFF3700C19A80005F
:10DB30006C6D02000000000059D3BF008000780027
:10DB40006C6D020000000000D19A80006C6D020034
:10DB500000000000F00120001602B600FDFF3A00B0
:10DB60001642A8001642AF00FEFF3700BE000900B3
:10DB700000000000000006004C72EF00C0118100A0
:10DB800000CBB300C0118900C01181000080FD00EE
:10DB900080C1B3000080FD00C0118900D011810058
:10DBA000F0CFB300D0118900A26C02000000000089
:10DBB000C011810000CBB300C0118900C0118100E9
:10DBC0000080FD0090C1B3000080FD00C0118900FD
:10DBD000D0118100F0CFB300D0118900A26C0200F7
:10DBE00000000000C011810000CBB300C01189000B
:10DBF000C01181000080FD00A0C1B3000080FD00C5
:10DC0000C0118900D0118100F0CFB300D01189007C
:10DC1000A26C020000000000C011810000CBB30024
:10DC2000C0118900C01181000080FD00B0C1B300A7
:10DC30000080FD00C0118900D0118100F0CFB30039
:10DC4000D0118900A26C020000000000C011810008
:10DC500000CBB300C0118900C01181000080FD001D
:10DC6000C0C1B3000080FD00C0118900D011810047
:10DC7000F0CFB300D0118900A26C020000000000B8
:10DC8000C011810000CBB300C0118900C011810018
:10DC90000080FD0000C2B3000080FD00C0118900BB
:10DCA000D011810000C0B300D0118900A26C020025
:10DCB00000000000C011810000CBB300C01189003A
:10DCC000C01181000080FD0010C2B3000080FD0083
:10DCD000C0118900D011810000C0B300D0118900AB
:10DCE000A26C020000000000C011810000CBB30054
:10DCF000C0118900C01181000080FD0020C2B30066
:10DD00000080FD00C0118900D011810000C0B30067
:10DD1000D0118900A26C020000000000C011810037
:10DD200000CBB300C0118900C01181000080FD004C
:10DD300030C2B3000080FD00C0118900D011810005
:10DD400000C0B300D0118900A26C020000000000E6
:10DD5000C011810000CBB300C0118900C011810047
:10DD60000080FD0040C2B3000080FD00C0118900AA
:10DD7000D011810000C0B300D0118900A26C020054
:10DD80000000000000CBB30054F3B7005573EF0060
:10DD9000C4242100B49A8800066D0200000000002F
:10DDA0004CF2B70000CBB30054F3B70010C0B3007F
:10DDB00055F3B700C4242100B49A8800066D020010
:10DDC000000000004CF2B70000CBB30054F3B700E2
:10DDD00020C0B30055F3B700C4242100B49A8800D2
:10DDE000066D0200000000004CF2B70000CBB3004B
:10DDF00054F3B70030C0B30055F3B700C42421007A
:10DE0000B49A8800066D0200000000004CF2B700D2
:10DE100000CBB30054F3B70040C0B30055F3B700D4
:10DE2000C4242100B49A8800066D0200000000009E
:10DE30004CF2B700C011810080CBB300C011890043
:10DE4000C01181000080FD0080C1B3000080FD0092
:10DE5000C0118900D011810010C0B300D011890019
:10DE6000A26C020000000000C011810080CBB30052
:10DE7000C0118900C01181000080FD0090C1B30075
:10DE80000080FD00C0118900D0118100F0CFB300E7
:10DE9000D0118900A26C020000000000C0118100B6
:10DEA00080CBB300C0118900C01181000080FD004B
:10DEB000A0C1B3000080FD00C0118900D011810015
:10DEC000F0CFB300D0118900A26C02000000000066
:10DED000C011810080CBB300C0118900C011810046
:10DEE0000080FD00B0C1B3000080FD00C0118900BA
:10DEF000D0118100F0CFB300D0118900A26C0200D4
:10DF000000000000C011810080CBB300C011890067
:10DF1000C01181000080FD00C0C1B3000080FD0081
:10DF2000C0118900D0118100F0CFB300D011890059
:10DF3000A26C020000000000C011810080CBB30081
:10DF4000C0118900C01181000080FD0000C2B30033
:10DF50000080FD00C0118900D0118100E0CFB30026
:10DF6000D0118900A26C020000000000C0118100E5
:10DF700080CBB300C0118900C01181000080FD007A
:10DF800010C2B3000080FD00C0118900D0118100D3
:10DF900000C0B300D0118900A26C02000000000094
:10DFA000C011810080CBB300C0118900C011810075
:10DFB0000080FD0020C2B3000080FD00C011890078
:10DFC000D011810000C0B300D0118900A26C020002
:10DFD00000000000C011810080CBB300C011890097
:10DFE000C01181000080FD0030C2B3000080FD0040
:10DFF000C0118900D011810000C0B300D011890088
:10E00000A26C020000000000C011810080CBB300B0
:10E01000C0118900C01181000080FD0040C2B30022
:10E020000080FD00C0118900D011810000C0B30044
:10E03000D0118900A26C02000000000080CBB30068
:10E0400054F3B7005573EF00C4242100B49A88003C
:10E05000066D0200000000004CF2B70080CBB30058
:10E0600054F3B70010C0B30055F3B700C424210027
:10E07000B49A8800066D0200000000004CF2B70060
:10E0800080CBB30054F3B70020C0B30055F3B70002
:10E09000C4242100B49A8800066D0200000000002C
:10E0A0004CF2B70080CBB30054F3B70030C0B300DC
:10E0B00055F3B700C4242100B49A8800066D02000D
:10E0C000000000004CF2B70080CBB30054F3B7005F
:10E0D00040C0B30055F3B700C4242100B49A8800AF
:10E0E000066D0200000000004CF2B700C011810074
:10E0F00000C5B300C0118900C01181000080FD007F
:10E1000080C1B3000080FD00C0118900D0118100E2
:10E11000F0CFB300D0118900A26C02000000000013
:10E12000C011810000C5B300C0118900C011810079
:10E130000080FD0090C1B3000080FD00C011890087
:10E14000D0118100F0C1B300D0118900A26C02008F
:10E1500000000000C011810000C5B300C01189009B
:10E16000C01181000080FD00A0C1B3000080FD004F
:10E17000C0118900D011810000C0B300D011890006
:10E18000A26C020000000000C011810000C5B300B5
:10E19000C0118900C01181000080FD00B0C1B30032
:10E1A0000080FD00C0118900D0118100E0C7B300DC
:10E1B000D0118900A26C020000000000C011810093
:10E1C00000C5B300C0118900C01181000080FD00AE
:10E1D000C0C1B3000080FD00C0118900D0118100D2
:10E1E00000C0B300D0118900A26C02000000000042
:10E1F000C011810000C5B300C0118900C0118100A9
:10E200000080FD0000C2B3000080FD00C011890045
:10E21000D011810000C0B300D0118900A26C0200AF
:10E2200000000000C011810000C5B300C0118900CA
:10E23000C01181000080FD0010C2B3000080FD000D
:10E24000C0118900D011810000CEB300D011890027
:10E25000A26C020000000000C011810000C5B300E4
:10E26000C0118900C01181000080FD0020C2B300F0
:10E270000080FD00C0118900D011810000C0B300F2
:10E28000D0118900A26C020000000000C0118100C2
:10E2900000C5B300C0118900C01181000080FD00DD
:10E2A00030C2B3000080FD00C0118900D011810090
:10E2B00010C8B300D0118900A26C02000000000059
:10E2C000C011810000C5B300C0118900C0118100D8
:10E2D0000080FD0040C2B3000080FD00C011890035
:10E2E000D0118100F0CFB300D0118900A26C0200E0
:10E2F0000000000000C5B30054F3B7005573EF00F1
:10E30000C4242100B49A8800066D020000000000B9
:10E310004CF2B70000C5B30054F3B70010C0B3000F
:10E3200055F3B700C4242100B49A8800066D02009A
:10E33000000000004CF2B70000C5B30054F3B70072
:10E3400030C0B30055F3B700C4242100B49A88004C
:10E35000066D0200000000004CF2B700C0CBB30015
:10E3600058F3B70080C1B30059F3B7005A73EF00F8
:10E37000846D020000000000C0CBB30058F3B7006A
:10E3800090C1B30059F3B7005A73EF00846D0200D7
:10E3900000000000C0CBB30058F3B700A0C1B30029
:10E3A00059F3B7005A73EF00846D020000000000BB
:10E3B000C0CBB30058F3B700B0C1B30059F3B700F6
:10E3C0005A73EF00846D020000000000C0CBB30060
:10E3D00058F3B700C0C1B30059F3B7005A73EF0048
:10E3E000846D020000000000C0CBB30058F3B700FA
:10E3F00000C2B30059F3B7005AF3EF00846D020076
:10E4000000000000C0CBB30058F3B70010C2B30047
:10E4100059F3B7005AF3EF00846D020000000000CA
:10E42000C0CBB30058F3B70020C2B30059F3B70014
:10E430005AF3EF00846D020000000000C0CBB3006F
:10E4400058F3B70030C2B30059F3B7005AF3EF00E6
:10E45000846D020000000000C0CBB30058F3B70089
:10E4600040C2B30059F3B7005AF3EF00846D0200C5
:10E4700000000000F40F2000A4638800C0CBB300AC
:10E4800058F3B70080C0B30059F3B70074CCBF0095
:10E490005AF3B700846D020000000000F40F200062
:10E4A000B4638800C0CBB30058F3B70090C0B3008A
:10E4B00059F3B70076CCBF005AF3B700846D020061
:10E4C00000000000C0CBB30058F3B700A0C0B300F9
:10E4D00059F3B7005A73EF00846D0200000000008A
:10E4E000F40F2000C4638800C0CBB30058F3B7001A
:10E4F000B0C0B30059F3B70078CCBF005AF3B700EF
:10E50000846D020000000000C0CBB30058F3B700D8
:10E51000C0C0B30059F3B7005A73EF00846D020016
:10E520000000000020C4B30058F3B70040C0B3009F
:10E5300059F3B7005A73EF00846D02000000000029
:10E5400020C4B30058F3B70050C0B30059F3B7006C
:10E550005A73EF00846D02000000000020C4B30075
:10E5600058F3B70060C0B30059F3B7005A73EF0017
:10E57000846D02000000000020C4B30058F3B7000F
:10E5800070C0B30059F3B7005A73EF00846D0200F6
:10E590000000000020C4B30058F3B70020C0B3004F
:10E5A00059F3B7005AF3EF00846D02000000000039
:10E5B00020C4B30058F3B70030C0B30059F3B7001C
:10E5C0005AF3EF00846D0200000000000000060016
:10E5D000851F78009033EF008E53E20002003A006E
:10E5E00010C0B3008EF3B7000862AE00040037001D
:10E5F0000622A8000622AF00FEFF37000300370006
:10E600000602A8000602AF00FEFF370001CAB300F1
:10E610008A6C0200000000008BD3BF0080027800EB
:10E62000854078008A6C020000000000559C800044
:10E63000854078008A6C0200000000000862AE008D
:10E64000040037000622A8000622AF00FEFF3700B4
:10E65000030037000602A8000602AF00FEFF3700E5
:10E6600011CAB3008A6C0200000000009033EF0072
:10E67000749C800061405200849C80000020E10076
:10E680000C003100809C80008C13B4008002780064
:10E6900011002000811F7800CF007800DC6C0200A0
:10E6A00000000000804A78009033EC0038730400CA
:10E6B00000000000749C8000614052000080FB005C
:10E6C000649C80008402400001002000811F7800CB
:10E6D000CF007800DC6C020000000000804A780067
:10E6E000F00120000602B600FDFF3A000642A80035
:10E6F0000642AF00FEFF3700DE0009000000000008
:10E70000000020008C13B4008002780005409000C7
:10E7100000E0B700CF02780000000600851F7800F7
:10E720006652E2002100320010938000904278008F
:10E73000209380000002780014407800002CE10053
:10E740000E003200109380009042780020938000E9
:10E750000002780014407800002CE1000300310032
:10E7600000C0EB00B87304000000000010C0B3004C
:10E770000F003700C87304000000000010938000F1
:10E780001004E00002003A000060EF0008003700CB
:10E79000109380006232EC00209380006432EC0021
:10E7A0006672ED0090730400000000000060EF004E
:10E7B000CF02780000000600851F78004C72EF0041
:10E7C00004022200749288000402220084928800CD
:10E7D000040222009492880004022200A49288007D
:10E7E00004022200B492880004022200C49288002D
:10E7F00004022200D492880004022200E4928800DD
:10E8000004022200F49288006072EF0020C1B3007D
:10E810008EF3B700E4FC2100549C8800E42421001E
:10E82000649C8800E8720200000000004CF2B7000F
:10E8300020C1B30066F2B700E424210014938800DD
:10E8400064822000249388008E7302000000000080
:10E850000004E00005003A00DAEAA8000060EF00DA
:10E860001C0037006A7404000000000020C1B300DF
:10E8700066F2B700E424210014938800A4832000EA
:10E88000249388008E730200000000000004E00062
:10E8900005003A00DAEAA9000060EF000D00370039
:10E8A0006A74040000000000C602A800C802AF009D
:10E8B00005003700DAEAA80000E0EF0005003700A5
:10E8C0006A74040000000000DAEAA90000E0EF002A
:10E8D00000003700CF02780000000600811F78009A
:10E8E000D1908000805878008048EB00CF007800FD
:10E8F0001A32EC0000000600851F780060C5B300E6
:10E900002EEBB7002F6BEF00306BEF0090C1B30020
:10E9100031EBB70040C1B30032EBB70000C4B30025
:10E9200033EBB700DAEAAE000400370010C8B300DA
:10E9300034EBB700A27404000000000010C0B30064
:10E9400034EBB70000C4B30035EBB70040C2B300EE
:10E9500036EBB700376BEF00386BEF00396BEF0029
:10E9600020C0B3003AEBB70020C0B3003BEBB700C8
:10E9700020C0B3003CEBB70020C0B3003DEBB700B4
:10E9800020C0B3003EEBB70020C0B3003FEBB700A0
:10E9900020C0B30040EBB70020C0B30041EBB7008C
:10E9A00020C1B30042EBB700C0C0B30043EBB700D7
:10E9B00050C0B30044EBB70080C1B30045EBB700D3
:10E9C00080C1B30046EBB70080C1B30047EBB7008E
:10E9D00080C1B30048EBB70080C1B30049EBB7007A
:10E9E00080C1B3004AEBB70080C1B3004BEBB70066
:10E9F00040C1B3004CEBB70040C1B3004DEBB700D2
:10EA000040C1B3004EEBB70040C1B3004FEBB700BD
:10EA100040C1B30050EBB70040C1B30051EBB700A9
:10EA200040C1B30052EBB70070C0B30053EBB70066
:10EA300070C0B30054EBB70070C0B30055EBB70023
:10EA400070C0B30056EBB70070C0B30057EBB7000F
:10EA500070C0B30058EBB70070C0B30059EBB700FB
:10EA600010C0B3005AEBB70010C0B3005BEBB700A7
:10EA700010C0B3005CEBB70010C0B3005DEBB70093
:10EA800010C0B3005EEBB70010C0B3005FEBB7007F
:10EA900010C0B30060EBB700F0CFB30061EBB7007C
:10EAA00062EBEF00F0CFB30063EBB70064EBEF0075
:10EAB000656BEF0066EBEF00F0CFB30067EBB700DC
:10EAC00068EBEF00F0CFB30069EBB7006AEBEF0043
:10EAD0006B6BEF006C6BEF006D6BEF00CF0278009B
:10EAE000000006000862AE00040037000622A800FD
:10EAF0000622AF00FEFF3700030037000602A80021
:10EB00000602AF00FEFF370001CEB3008A6C0200A0
:10EB100000000000C11181008A6C020000000000AA
:10EB2000F00120000602B600FDFF3A000642A800F0
:10EB30000642AF00FEFF3700BE00090000000000E3
:10EB400000000600851F78006A33EF0014002000E3
:10EB5000549B8800549B80006720E100180031001E
:10EB6000549B800067024200840278003822F8003B
:10EB7000E5FF9F003822F9007275020000000000D6
:10EB8000C0118100A0C9B300C0118900C01181006B
:10EB90000080FD00E0C1B3000080FD00C0118900CD
:10EBA000D011810060CBB300D0118900A26C0200AB
:10EBB000000000006A33EC00AA75040000000000A9
:10EBC000CC42A900D042A80014002000549B880029
:10EBD000549B80006720E1001E003100549B8000A0
:10EBE00067024200840278003822F800E5FF9F00A7
:10EBF0003822F90072750200000000005000200069
:10EC0000E603020000000000C011810020C4B30030
:10EC1000C0118900C01181000080FD00F0C0B30068
:10EC20000080FD00C0118900D011810040C4B300F4
:10EC3000D0118900A26C02000000000050002000EA
:10EC4000E6030200000000006A33EC00E8750400EF
:10EC500000000000CF02780000000600851F780049
:10EC60007E13F8008413F9008253E2000C00320096
:10EC7000009C80001004E00009003200209C80000D
:10EC80008433EC0080027800009C80008033EC002C
:10EC9000904A78008273ED00347604000000000092
:10ECA0008253E20007003200209C80008433EC0095
:10ECB00080027800804AEB008273ED0050760400F9
:10ECC000000000007E13F8000000F900CF02780079
:10ECD00000000600A13621000200200012000900F9
:10ECE0008058EB0020C1B30082F3B700A4362100A6
:10ECF000F49B88006813F8008013F9002E76020058
:10ED00000000000070C0B3007EF3B7007F73EF0017
:10ED100020C1B30082F3B700A4362100049C880010
:10ED20003E6C02000000000000000600851F780015
:10ED30008433EF000862AE00040037000622A8000A
:10ED40000622AF00FEFF3700030037000602A800CE
:10ED50000602AF00FEFF370001CAB3008A6C020052
:10ED6000000000007FD3BF0080027800854078005B
:10ED70008A6C020000000000F59B8000854078004E
:10ED80008A6C0200000000008433EF00209C8000A9
:10ED9000149C80000960EF000020E10009003600AB
:10EDA000209C80008013B400904278008540780059
:10EDB0008A6C0200000000008433EC00C676040078
:10EDC00000000000F00120000602B600FDFF3A003E
:10EDD0000642A8000642AF00FEFF3700BE00090051
:10EDE00000000000CF02780000000600851F7800B8
:10EDF0000862AE00040037000622A8000622AF0019
:10EE0000FEFF3700030037000602A8000602AF002D
:10EE1000FEFF370001CAB3008A6C02000000000048
:10EE20007FD3BF0080027800854078008A6C0200A2
:10EE300000000000F59B8000854078008A6C02008D
:10EE400000000000019C80008A6C020000000000AD
:10EE5000F00120000602B600FDFF3A000642A800BD
:10EE60000642AF00FEFF3700BE00090000000000B0
:10EE7000CF02780000000600844080004822DE00B7
:10EE80006124E10007003A00C01181002322AF0095
:10EE9000FEFF370024E2B7002562EF005C77040034
:10EEA00000000000C01181003322AF00FEFF3700D8
:10EEB00034E2B7003562EF0000000600851F7800DD
:10EEC0007A33EF007973EF007E33EF0078D3BF0021
:10EED00082F3B700E4B22000049C8800967602001A
:10EEE000000000007A33EF00D09B8000C49B8000BC
:10EEF0000960EF000020E10009003600E4B22000C4
:10EF0000D39B800004804100000278001440780008
:10EF10007973B4007A33EC007477040000000000C9
:10EF2000C49B80004822DE00F4CFB2000440780089
:10EF300079F3B700C49B80004822DE0061424200A2
:10EF40000440780079F3B70078D3BF007EF3B700B0
:10EF50007F73EF0079D3BF0080F3B700F67602002D
:10EF600000000000D10AAE000F00370001002000B1
:10EF700001007800E8170200000000008100E800AE
:10EF8000811F78003822F800E0FF9F003822F90046
:10EF90003C77020000000000CF007800D000200085
:10EFA0000008E600F2FF3700CF02780000000600FC
:10EFB0007C32EF007E32EF00049524000494880038
:10EFC00004052000149488008432EF008632EF009C
:10EFD0009872EF0081282100020020000F00090034
:10EFE0008058EB0084242100E49388009872EF009D
:10EFF00098D2BF00945680004822DE000024E10031
:10F000000E00360000C1B30082F3B7007C12F80096
:10F010007E13F90084282100049C88009676020063
:10F0200000000000E493800070024200E493880036
:10F030009872EC00F877040000000000842421009E
:10F04000F49388007FD2BF0084F2B7007ED2BF0065
:10F0500085F2B7007FD2BF0086F2B7007ED2BF0034
:10F0600087F2B70080C0B30082F3B7000424210008
:10F07000F49B880004282100049C880096760200F6
:10F0800000000000D36AEF00D40AF800D60AF900A5
:10F09000000006007832EF007A72EF007B72EF001A
:10F0A000C1252100020020001B0009008058EB0050
:10F0B00004052000C49388007A72EF00D493800086
:10F0C000A3082000041CE1000E00360000C1B300BC
:10F0D00082F3B7007812F8007E13F900C4252100EE
:10F0E000049C88009676020000000000C493800013
:10F0F00070024200C49388007A72EC005E780400CB
:10F100000000000004902000C49388007B72EF0090
:10F11000D49380004822DE006624E100150031000F
:10F120007A72EF00D49380006E24E1000E0031006B
:10F13000C0C1B30082F3B7007812F8007E13F90063
:10F14000C4252100049C880096760200000000007F
:10F15000C49380007C024200C49388007A72EC0061
:10F1600092780400000000007B72EC0088780400B4
:10F1700000000000D8770200000000000000060038
:10F18000851F78004C32EF004E32EF005072EF00D6
:10F190005172EF001443230094928800D4A22400FB
:10F1A000A492880054C72600B4928800D412230089
:10F1B000C492880004032000D49288007C7402006A
:10F1C0000000000000C4B30078F3B7005E770200CF
:10F1D000000000004A78020000000000DAEAAE00F9
:10F1E0000A00370020C1B30082F3B700E4FC21001D
:10F1F000F49B880064822000049C880096760200BC
:10F2000000000000167904000000000020C1B300D7
:10F2100082F3B700E4FC2100F49B8800A483200063
:10F22000049C8800967602000000000004FE210085
:10F23000649288004E32EF005072EF00849280009A
:10F240007324E10028003100849280000960EF00FF
:10F250002381200003004200904278000403200034
:10F260000524E10004003E00940320000524E10091
:10F2700001003900030037000040EB00447904002E
:10F280000000000010C0B3006104E10013003A0068
:10F29000749280006520E10010003E00849280009E
:10F2A0000960EF0023812000030042001040780035
:10F2B00051F2B70051D2BF0080F3B7004C12F800F2
:10F2C0007E13F900F6760200000000004E32EC00DA
:10F2D0006492800061024200649288005072EC00E7
:10F2E0001E7904000000000090C0B30082F3B70054
:10F2F00064FE2100F49B880024252100049C8800E2
:10F300009676020000000000CF02780000000600A0
:10F31000851F7800C500200003000900B51F780094
:10F32000800378008404780004F0A1000400E00069
:10F3300006003A0009F0A70002003700050020008F
:10F3400011003700050020000F003700E642520090
:10F350000C0039000003200009F0A6000002200084
:10F360003822F800E0FF9F003822F9003C770200C5
:10F37000000000008502E900F9FF3B005500200075
:10F3800001003700840278006400200005E0A0003E
:10F3900009F0A70005F0A000087122001100090083
:10F3A0008883D8000A7A02000000000081037800F8
:10F3B000883E2000110009008883D8000A7A0200E4
:10F3C00000000000810378004806200011000900B9
:10F3D0008883D8000A7A02000000000081037800C8
:10F3E000A8002000110009008883D8000A7A0200D2
:10F3F000000000000003200000C040003822F80098
:10F40000E0FF9F003822F9003C7702000000000076
:10F410001B003700060320000000E0000E003A0049
:10F4200005E0A6000D0037000402E9000524E10014
:10F43000020032004200AF00000006000000E000C1
:10F4400005003A0005E0A6000400370005F0A6001C
:10F45000060220000100370005E0A1000040430043
:10F46000811F78003822F800E0FF9F003822F90061
:10F470003C77020000000000CF007800000006008A
:10F480002501200003000900CF127800CF02780088
:10F4900000000600851F78000862AE0004003700F7
:10F4A0000622A8000622AF00FEFF37000300370047
:10F4B0000602A8000602AF00FEFF370001CAB30033
:10F4C0008A6C02000000000083D3BF008002780035
:10F4D000854078008A6C020000000000159C8000C6
:10F4E000854078008A6C0200000000000862AE00CF
:10F4F000040037000622A8000622AF00FEFF3700F6
:10F50000030037000602A8000602AF00FEFF370026
:10F5100011CAB3008A6C020000000000259C800024
:10F5200001002000811F7800CF007800DC6C020011
:10F5300000000000804A7800F00120000602B600BA
:10F54000FDFF3A000642A8000642AF00FEFF37006A
:10F55000DE00090000000000259C800005409000AE
:10F5600000E0B700CF02780000000600851F780099
:10F57000861F78000001EB000103780064C11000D1
:10F580004211DD000200DD00800278000C60EC001A
:10F590000C60ED000F00320005007800C42ADD0089
:10F5A0004C00DE00F000B2000003B000A203200017
:10F5B0000200E100010039000D40B4003822F800DB
:10F5C000E0FF9F003822F9003C77020000000000B5
:10F5D000EFFF37004F037800CF02780000000600ED
:10F5E000851F78007A33EF007C33EF007973EF00EA
:10F5F0007E73EF007F73EF007C33EF00E49B8000AD
:10F600006220E100BE00310078D3BF008EF3B70066
:10F610007A13F8008A13F900E4B22000649C880091
:10F62000E8720200000000002EEBB700D10AAE0025
:10F630002300370001002000010078003C17020081
:10F64000000000008100E800811F78003822F800E7
:10F65000E0FF9F003822F9003C7702000000000024
:10F66000CF007800D00020000008E600F2FF37004D
:10F6700078D3BF000160EF00040020008879020009
:10F6800000000000C011810090C2B300C0118900C9
:10F690003C77020000000000C0118100A0C3B3004D
:10F6A000C01189003C77020000000000C0118100F9
:10F6B00000C2B300C01189003C77020000000000C6
:10F6C0007A33EF00D09B8000C49B80000960EF007C
:10F6D0000020E1000F003600E4B22000D39B800040
:10F6E0000480410000027800144078007973B4006F
:10F6F0007A13F8008213F900F4372100249C880063
:10F700004A7A0200000000007A33EC00627B0400B9
:10F7100000000000C49B80004822DE00F4CFB2004D
:10F720000440780079F3B700C49B80004822DE00D3
:10F73000614242000440780079F3B70078D3BF00FB
:10F740007AF3B7007B73EF007A13F8008213F900A5
:10F75000E4372100249C88004A7A0200000000005F
:10F760007EF3B7007ED3BF007953E30028003A0050
:10F77000D10AAE002300370001002000010078000C
:10F780005C170200000000008100E800811F780083
:10F790003822F800E0FF9F003822F9003C77020091
:10F7A00000000000CF007800900020000008E60074
:10F7B000F2FF37007ED3BF000160EF00217022000E
:10F7C000B67A020000000000D1002000010078009D
:10F7D0005C170200000000008100E800811F780033
:10F7E0003822F800E0FF9F003822F9003C77020041
:10F7F00000000000CF007800300120000008E60083
:10F80000F2FF370010C0B30000E0B700710037000E
:10F81000D10AAE0037003700010020000100780057
:10F820007E170200000000008100E800811F7800C0
:10F830003822F800E0FF9F003822F9003C770200F0
:10F8400000000000CF007800900020000008E600D3
:10F85000F2FF37007ED3BF000160EF00217022006D
:10F86000B67A020000000000D100200001007800FC
:10F870007E170200000000008100E800811F780070
:10F880003822F800E0FF9F003822F9003C770200A0
:10F8900000000000CF007800900120000008E60082
:10F8A000F2FF370079D3BF000160EF002170220022
:10F8B000B67A020000000000D101200001007800AB
:10F8C0007E170200000000008100E800811F780020
:10F8D0003822F800E0FF9F003822F9003C77020050
:10F8E00000000000CF007800B00220000008E60011
:10F8F000F2FF37007C33EC00FE7A040000000000C9
:10F90000D10AAE003200370001002000010078006B
:10F91000B8170200000000008100E800811F780095
:10F920003822F800E0FF9F003822F9003C770200FF
:10F9300000000000CF007800D00020000008E600A2
:10F94000F2FF37007ED3BF000160EF00217022007C
:10F95000B67A0200000000001101200001007800CA
:10F96000B8170200000000008100E800811F780045
:10F970003822F800E0FF9F003822F9003C770200AF
:10F9800000000000CF007800D00120000008E60051
:10F99000F2FF370079D3BF000160EF002170220031
:10F9A000B67A020000000000C0118100A0C0B300C0
:10F9B000C01189003C77020000000000C0118100E6
:10F9C000D0C0B300C01189003C77020000000000E5
:10F9D0000060EF00CF0278000000060080C0B30096
:10F9E0008EF3B70004242100549C8800C424210015
:10F9F000649C8800E8720200000000004CF2B7002E
:10FA00006492800004C5B20007003A00649280004E
:10FA10004822DE0094C4B20003003A0074928000D1
:10FA200004C5B20007003200D36AEF00842421002D
:10FA3000A456880084242100B456880000E0EF001A
:10FA40000B0037004FD2BF00D3EAB70051D2BF003E
:10FA5000D4EAB70050D2BF00D5EAB70053D2BF00F6
:10FA6000D6EAB70052D2BF00D7EAB7000060EF0075
:10FA700000000600851F780000C4B30078F3B700CB
:10FA8000F07A0200000000006104E100130032007F
:10FA9000D10AAE000F0037000100200001007800FD
:10FAA00004180200000000008100E800811F7800B7
:10FAB0003822F800E0FF9F003822F9003C7702006E
:10FAC00000000000CF007800400220000008E6009F
:10FAD000F2FF37007C740200000000002ECBBF0054
:10FAE000D0EAB7002FCBBF00D1EAB70031CBBF00BF
:10FAF000E2EAB70032CBBF00E1EAB70033CBBF0088
:10FB0000D2EAB700DAEAAE000500370034CBBF0016
:10FB1000DAEAB700DAEAA800947D040000000000E9
:10FB200034CBBF00DAEAB70035CBBF0035EAB70007
:10FB300036CBBF0036EAB70037CBBF00DCEAB700F0
:10FB400038CBBF00DDEAB70039CBBF00DBEAB70036
:10FB50003ACBBF00FBEAB7003BCBBF00FCEAB700E3
:10FB60003CCBBF00FDEAB7003DCBBF00FEEAB700CB
:10FB70003ECBBF00FFEAB7003FCBBF0000EBB700B2
:10FB800040CBBF0001EBB70041CBBF0003EBB70098
:10FB900042CBBF00DFEAB70043CBBF00DEEAB700CD
:10FBA00044CBBF00E0EAB70045CBBF00E3EAB700B3
:10FBB00046CBBF00E4EAB70047CBBF00E5EAB70099
:10FBC00048CBBF00E6EAB70049CBBF00E7EAB70081
:10FBD0004ACBBF00E8EAB7004BCBBF00E9EAB70069
:10FBE0004CCBBF00EBEAB7004DCBBF00ECEAB7004F
:10FBF0004ECBBF00EDEAB7004FCBBF00EEEAB70037
:10FC000050CBBF00EFEAB70051CBBF00F0EAB7001E
:10FC100052CBBF00F1EAB70053CBBF00F3EAB70005
:10FC200054CBBF00F4EAB70055CBBF00F5EAB700EC
:10FC300056CBBF00F6EAB70057CBBF00F7EAB700D4
:10FC400058CBBF00F8EAB70059CBBF00F9EAB700BC
:10FC50005ACBBF0006EBB7005BCBBF0007EBB7008A
:10FC60005CCBBF0008EBB7005DCBBF0009EBB70072
:10FC70005ECBBF000AEBB7005FCBBF000BEBB7005A
:10FC800060CBBF000CEBB70061CBBF0084ECB700CA
:10FC900062CBBF0083ECB70063CBBF0082ECB70040
:10FCA00064CBBF0081ECB70065CBBF0080ECB70030
:10FCB00066CBBF007EECB70067CBBF007DECB70022
:10FCC00068CBBF007CECB70069CBBF007BECB70012
:10FCD0006ACBBF007AECB7006BCBBF0004EBB70078
:10FCE0006CCBBF000EEBB7000ECBBF00F047B200ED
:10FCF0007804E100010036000E6BEF006DCBBF0011
:10FD00000FEBB700745880004822DE007824E10031
:10FD1000010036000F6BEF002E2AEF00EE7C020090
:10FD200000000000CF02780000000600851F780068
:10FD30006633EF006453E20002003A0010C0B300E3
:10FD400064F3B7000862AE00040037000622A80082
:10FD50000622AF00FEFF3700030037000602A800AE
:10FD60000602AF00FEFF3700019B80008A6C020094
:10FD700000000000059B8000C82ADE000548B30093
:10FD8000854078008A6C0200000000000862AE0026
:10FD9000040037000622A8000622AF00FEFF37004D
:10FDA000030037000602A8000602AF00FEFF37007E
:10FDB00060D3BF00E1427000854078008A6C020089
:10FDC000000000006633EF00249B80006140520079
:10FDD000349B80000020E1000C003100309B80004B
:10FDE0006213B4008002780011002000811F7800A7
:10FDF000CF007800DC6C020000000000804A780030
:10FE00006633EC00E47E040000000000249B8000C8
:10FE1000614052000080FB00149B8000840240007F
:10FE200001002000811F7800CF007800DC6C020008
:10FE300000000000804A7800F00120000602B600B1
:10FE4000FDFF3A000642A8000642AF00FEFF370061
:10FE5000BE00090000000000000020006213B40092
:10FE6000800278000540900000E0B700CF027800E3
:10FE700000000600851F7800D0CABF002EEBB70037
:10FE8000D1CABF002FEBB700306BEF00E2CABF0052
:10FE900031EBB700E1CABF0032EBB700D2CABF00F6
:10FEA00033EBB700DACABF0034EBB70035CABF0086
:10FEB00035EBB70036CABF0036EBB700DCCABF006F
:10FEC00037EBB700DDCABF0038EBB700DBCABF00B5
:10FED00039EBB700FBCABF003AEBB700FCCABF0062
:10FEE0003BEBB700FDCABF003CEBB700FECABF004A
:10FEF0003DEBB700FFCABF003EEBB70000CBBF0031
:10FF00003FEBB70001CBBF0040EBB70003CBBF0016
:10FF100041EBB700DFCABF0042EBB700DECABF004B
:10FF200043EBB700E0CABF0044EBB700E3CABF0031
:10FF300045EBB700E4CABF0046EBB700E5CABF0017
:10FF400047EBB700E6CABF0048EBB700E7CABF00FF
:10FF500049EBB700E8CABF004AEBB700E9CABF00E7
:10FF60004BEBB700EBCABF004CEBB700ECCABF00CD
:10FF70004DEBB700EDCABF004EEBB700EECABF00B5
:10FF80004FEBB700EFCABF0050EBB700F0CABF009D
:10FF900051EBB700F1CABF0052EBB700F3CABF0084
:10FFA00053EBB700F4CABF0054EBB700F5CABF006B
:10FFB00055EBB700F6CABF0056EBB700F7CABF0053
:10FFC00057EBB700F8CABF0058EBB700F9CABF003B
:10FFD00059EBB70006CBBF005AEBB70007CBBF0009
:10FFE0005BEBB70008CBBF005CEBB70009CBBF00F1
:10FFF0005DEBB7000ACBBF005EEBB7000BCBBF00D9
:020000040001F9
:100000005FEBB7000CCBBF0060EBB70084CCBF0048
:1000100061EBB70083CCBF0062EBB70082CCBF00BE
:1000200063EBB70081CCBF0064EBB70080CCBF00AE
:1000300065EBB7007ECCBF0066EBB7007DCCBF00A0
:1000400067EBB7007CCCBF0068EBB7007BCCBF0090
:1000500069EBB7007ACCBF006AEBB70004CBBF00F6
:100060006BEBB7000ECBBF006CEBB7000FCBBF0044
:100070006DEBB70000C4B30078F3B7005E77020001
:100080000000000000C4B30078F3B700F07A02006B
:10009000000000006104E10011003200D10AAE004E
:1000A0000F00370001002000010078003618020020
:1000B000000000008100E800811F78003822F8006D
:1000C000E0FF9F003822F9003C77020000000000AA
:1000D000CF007800800220000008E600F2FF370021
:1000E000CF02780000000600851F7800D18AAE009C
:1000F00003003700F49A80006124E10017003A0001
:10010000D18AA80080CBB30060F3B7006173EF0021
:1001100050C0B30064F3B70004C82000149B8800EB
:10012000967E02000000000080ECB70000CBB30018
:1001300060F3B7006173EF0050C0B30064F3B70021
:10014000A4C72000149B8800967E020000000000D7
:100150007AECB7003A7F02000000000081CCBF00BB
:100160008CECB70082CCBF008DECB70083CCBF0015
:100170008EECB70084CCBF008FECB7007ACCBF0008
:1001800086ECB7007BCCBF0087ECB7007CCCBF000F
:1001900088ECB7007DCCBF0089ECB7007ECCBF00F7
:1001A0008AECB7008B6CEF00CF02780000000600ED
:1001B000A82DEF00A80DF800AA0DF900A1CA200093
:1001C00002002000FD0009008058EB00A82CA900C7
:1001D00000000600851F7800C5002000030009000C
:1001E000B51F7800800378008404780004F0A10033
:1001F0000400E00006003A0009F0A7000200370002
:100200000500200010003700050020000E00370018
:10021000E64252000B0039000003200009F0A6005E
:1002200000022000801F78004F0078006E740200EA
:10023000000000008502E900FAFF3B0055002000A5
:1002400001003700840278006400200005E0A0006F
:1002500009F0A70005F0A0000871220011000900B4
:100260008883D800688102000000000081037800C4
:10027000883E2000110009008883D80068810200B0
:1002800000000000810378004806200011000900EA
:100290008883D80068810200000000008103780094
:1002A000A8002000110009008883D800688102009E
:1002B000000000000003200000C04000801F780004
:1002C0004F0078006E740200000000001A00370032
:1002D000060320000000E0000E003A0005E0A60042
:1002E0000D0037000402E9000524E100020032009D
:1002F0004200AF00000006000000E00005003A00E8
:1003000005E0A6000400370005F0A6000602200064
:100310000100370005E0A10000404300811F780084
:10032000801F78004F0078006E740200000000000B
:10033000CF0078000000060025012000030009001E
:10034000CF127800CF02780000000600851F7800E9
:100350006C33EF006E73EF006F73EF0014902800A2
:10036000849B880024002800949B880034002E0081
:10037000A49B880044002800B49B880054202700D8
:10038000C49B880064002400D49B880074902600DD
:10039000E49B880084002C00F49B88009470270064
:1003A000049C8800A4002800149C8800B400240049
:1003B000249C8800C4002000349C8800D4002400C1
:1003C000449C8800E4002000549C8800F400240031
:1003D000649C880004012000749C88001491210012
:1003E000849C880024812100949C88003401220090
:1003F000A49C880044812100B49C880054A1200062
:10040000C49C880064412000D49C88007441200072
:10041000E49C880084A12200F49C8800944122007E
:10042000049D8800A4812500149D8800B431270014
:10043000249D8800C4F12F00349D8800D4812700BA
:10044000449D8800E4412A00549D8800F4612900FD
:10045000649D880004F22000749D8800140222002C
:10046000849D880024222300949D8800346221000A
:10047000A49D880044822000B49D880054F22C0082
:10048000C49D880064022100D49D88007402260067
:10049000E49D880084F22B00F49D880094222000C3
:1004A000049E8800A4022800149E8800B402200044
:1004B000249E8800C4022000349E8800D4822E002E
:1004C000449E8800E4022E00549E880014502A00A6
:1004D000649E880024002000749E880034002E0052
:1004E000849E880044002800949E880054202700A1
:1004F000A49E880064002400B49E880074902600A6
:10050000C49E880084002C00D49E8800947027002C
:10051000E49E8800A4002800F49E8800B400240013
:10052000049F8800C4002000149F8800D400240089
:10053000249F8800E4002000349F8800F4002400F9
:10054000449F880004012000549F88001401220069
:10055000649F880024812100749F88003401220058
:10056000849F880044812100949F880054A120002A
:10057000A49F880064412000B49F8800744120003B
:10058000C49F880084A12200D49F88009441220047
:10059000E49F8800A4812500F49F8800B4312700DF
:1005A00004A08800C4F12F0014A08800D481270083
:1005B00024A08800E4412A0034A08800F4612900C6
:1005C00044A0880004F2200054A0880014022200F5
:1005D00064A088002422230074A0880034622100D3
:1005E00084A088004482200094A0880054F22C004B
:1005F000A4A0880064022100B4A088007402260030
:10060000C4A0880084F22B00D4A08800942220008B
:10061000E4A08800A4022800F4A08800B40220000E
:1006200004A18800C402200014A18800D4822E00F6
:1006300024A18800E4022E0034A188001490280030
:1006400044A188002400280054A1880034002A0016
:1006500064A188005420270074A18800640024004D
:1006600084A188007490260094A1880084002C0046
:10067000A4A1880094702700B4A18800A4002800D9
:10068000C4A18800B4002400D4A18800C4002000C4
:10069000E4A18800D4002400F4A18800E400200034
:1006A00004A28800F400240014A2880004012000A1
:1006B00024A288001401220034A288002481210091
:1006C00044A288003401220054A288004481210001
:1006D00064A2880054A1200074A288006441200014
:1006E00084A288007441200094A2880084A1220082
:1006F000A4A2880094412200B4A28800A48125000D
:10070000C4A28800B4312700D4A28800C4F12F000D
:10071000E4A28800D4812700F4A28800E4412A00E2
:1007200004A38800F461290014A3880004F22000C7
:1007300024A388001402220034A38800242223006A
:1007400044A388003462210054A38800448220001E
:1007500064A3880054F22C0074A388006402210072
:1007600084A388007402260094A3880084F22B00DE
:10077000A4A3880094222000B4A38800A402280027
:10078000C4A38800B4022000D4A38800C4022000BF
:10079000E4A38800D4822E00F4A38800E4022E0093
:1007A00004A488008234EF0014402A0024A48800A6
:1007B00024002F0034A4880034002A0044A48800B8
:1007C0005420270054A488006400240064A48800F6
:1007D0007490260074A4880084002C0084A48800EF
:1007E0009470270094A48800A4002800A4A4880082
:1007F000B4002400B4A48800C4002000C4A488006D
:10080000D4002400D4A48800E4002000E4A48800DC
:10081000F4002400F4A488000401200004A588004A
:100820001401220014A588002481210024A5880039
:100830003401220034A588004481210044A58800A9
:1008400054A1200054A588006441200064A58800BC
:100850007441200074A5880084A1220084A588002A
:100860009441220094A58800A4812500A4A58800B5
:10087000B4312700B4A58800C4F12F00C4A58800B6
:10088000D4812700D4A58800E4412A00E4A588008B
:10089000F4612900F4A5880004F2200004A6880071
:1008A0001402220014A688002422230024A6880013
:1008B0003462210034A688004482200044A68800C7
:1008C00054F22C0054A688006402210064A688001B
:1008D0007402260074A6880084F22B0084A6880087
:1008E0009422200094A68800A4022800A4A68800D0
:1008F000B4022000B4A68800C4022000C4A6880068
:10090000D4822E00D4A68800E4022E00E4A688003B
:10091000DE34EF001470260004A7880024002200B3
:1009200014A7880034802A0024A7880044002800E7
:1009300034A788005420270044A7880064002400BE
:1009400054A788007490260064A7880084002C00B7
:1009500074A788009470270084A78800A40028004A
:1009600094A78800B4002400A4A78800C400200035
:10097000B4A78800D4002400C4A78800E4002000A5
:10098000D4A78800F4002400E4A788000401200014
:10099000F4A788001401220004A888002481210003
:1009A00014A888004481210024A8880054A12000B4
:1009B00034A888006441200044A8880074412000C5
:1009C00054A8880084A1220064A888009401220011
:1009D00074A88800A481250084A88800B4B12300ED
:1009E00094A88800C4F12F00A4A88800D48127000F
:1009F000B4A88800E4412A00C4A88800F461290052
:100A0000D4A8880004F22000E4A888001402220080
:100A1000F4A888002422230004A98800344221007D
:100A200014A988004482200024A9880054F22C00D4
:100A300034A988006402210044A9880074022600B9
:100A400054A9880084F22B0064A988009422200015
:100A500074A98800A402280084A98800B402200098
:100A600094A98800C4022000A4A98800D4822E0082
:100A7000B4A98800E4022E00C4A988003A35EF002A
:100A800014B02700E4A9880024002C00F4A98800F1
:100A900034802A0004AA88004400280014AA880090
:100AA0005420270024AA88006400240034AA880067
:100AB0007490260044AA880084002C0054AA880060
:100AC0009470270064AA8800A400280074AA8800F3
:100AD000B400240084AA8800C400200094AA8800DE
:100AE000D4002400A4AA8800E4002000B4AA88004E
:100AF000F4002400C4AA880004012000D4AA8800BD
:100B000014012200E4AA880024812100F4AA8800AC
:100B10004481210004AB880054A1200014AB88005C
:100B20006441200024AB88007441200034AB88006D
:100B300084A1220044AB88009401220054AB8800B9
:100B4000A451240064AB8800B431270074AB880042
:100B5000C4F12F0084AB8800D481270094AB8800B7
:100B6000E4412A00A4AB8800F4612900B4AB8800FA
:100B700004F22000C4AB880014022200D4AB880029
:100B800024222300E4AB880034422100F4AB880027
:100B90004482200004AC880054F22C0014AC88007D
:100BA0006402210024AC88007402260034AC880062
:100BB00084F22B0044AC88009422200054AC8800BE
:100BC000A402280064AC8800B402200074AC880041
:100BD000C402200084AC8800D4822E0094AC88002B
:100BE000E4022E00A4AC88009635EF001420230008
:100BF000C4AC880024002000D4AC8800340022005B
:100C0000E4AC880044002800F4AC8800542027009D
:100C100004AD88006400240014AD880074902600A0
:100C200024AD880084002C0034AD88009470270027
:100C300044AD8800A400280054AD8800B400200012
:100C400064AD8800C400280074AD8800D400200082
:100C500084AD8800E400280094AD8800F4002000F2
:100C6000A4AD880004012800B4AD88004421200010
:100C7000C4AD880054A12000D4AD880064212000B8
:100C8000E4AD880074212000F4AD880084012200C6
:100C900004AE88009481200014AE8800A441210095
:100CA00024AE8800B431270034AE8800C4F12F0090
:100CB00044AE8800D481270054AE8800E441280067
:100CC00064AE8800F461290074AE880004F220004C
:100CD00084AE88001402220094AE880024222300EF
:100CE000A4AE880034622100B4AE880044422500DE
:100CF000C4AE880054922000D4AE88006402220062
:100D0000E4AE880074022D00F4AE880084F22B005B
:100D100004AF88009422200014AF8800A4022800A9
:100D200024AF8800B402200034AF8800C402200041
:100D300044AF8800D4822E0054AF8800E4022E0015
:100D400064AF8800EE35EF001420240084AF8800E3
:100D50002400200094AF880034002600A4AF88004F
:100D600044002C00B4AF880054202700C4AF880092
:100D700064002400D4AF880074902600E4AF88009B
:100D800084002C00F4AF88009470270004B0880021
:100D9000A400280014B08800B400200024B088000B
:100DA000C400280034B08800D400200044B088007B
:100DB000E400280054B08800F400200064B08800EB
:100DC0000401280074B088004421200084B0880009
:100DD00054A1200094B0880064212000A4B08800B1
:100DE00074212000B4B0880084012200C4B08800BF
:100DF00094D12000D4B08800A4412100E4B0880040
:100E0000B4312700F4B08800C4F12F0004B1880089
:100E1000D481270014B18800E441280024B188005F
:100E2000F461290034B1880004F2200044B1880044
:100E30001402220054B188002422230064B18800E7
:100E400034A2210074B188004442250084B1880096
:100E50005492200094B1880064022200A4B188005A
:100E600074022D00B4B1880084F22B00C4B1880054
:100E700094222000D4B18800A4022800E4B18800A4
:100E8000B4022000F4B18800C402200004B288003B
:100E9000D4822E0014B28800E4022E0024B288000E
:100EA0004636EF001440250044B28800240020009C
:100EB00054B2880034802A0064B2880044002C00B8
:100EC00074B288005420270084B288006400240093
:100ED00094B2880074902600A4B2880084002C008C
:100EE000B4B2880094702700C4B28800A40028001F
:100EF000D4B28800B4002000E4B28800C400280006
:100F0000F4B28800D400200004B38800E400280074
:100F100014B38800F400200024B3880004012800E2
:100F200034B388004401200044B3880054A1200059
:100F300054B388006421200064B388007421200029
:100F400074B388008401220084B388009441200097
:100F500094B38800A4412100A4B38800B4312700D1
:100F6000B4B38800C4F12F00C4B38800D481270033
:100F7000D4B38800E4612B00E4B38800F441290075
:100F8000F4B3880004F2200004B4880014022200A4
:100F900014B488002422230024B488003462210081
:100FA00034B4880044A22A0044B488005452250076
:100FB00054B488006422230064B4880074022600BC
:100FC00074B4880084F22B0084B48800942220003A
:100FD00094B48800A4022800A4B48800B4022000BD
:100FE000B4B48800C4022000C4B48800D4822E00A7
:100FF000D4B48800E4022200E4B488009E36EF00F6
:101000001490260004B588002400280014B5880038
:1010100034802A0024B588005420270034B5880085
:101020006400240044B588007490260054B58800FC
:1010300084002C0064B588009470270074B5880083
:10104000A400280084B58800B400200094B588006E
:10105000C4002800A4B58800D4002000B4B58800DE
:10106000E4002800C4B58800F4002000D4B588004E
:1010700004012800E4B5880014012200F4B58800BA
:101080002481290004B688003401220014B68800A7
:1010900044C1290024B6880054A1200034B6880039
:1010A0006421200044B688007421200054B68800D2
:1010B0008401220064B688009441200074B6880040
:1010C000A441210084B68800B431270094B688007A
:1010D000C4F12F00A4B68800D4812700B4B68800DC
:1010E000E4612B00C4B68800F4412900D4B688001E
:1010F00004F22000E4B6880014022200F4B688004E
:101100002422230004B788003462210014B7880029
:101110004442250024B788005492200034B7880048
:101120006402220044B7880074022D0054B788007E
:1011300084F22B0064B788009422200074B78800E2
:10114000A402280084B78800B402200094B7880065
:10115000C4022000A4B78800D4822E00B4B788004F
:10116000E4022E00C4B78800FA36EF00149026007F
:10117000E4B7880024002800F4B7880034002B006E
:1011800004B8880044002C0014B8880054202700BC
:1011900024B888006400240034B8880074902600C5
:1011A00044B8880084002C0054B88800947027004C
:1011B00064B88800A400280074B88800B400200037
:1011C00084B88800C400280094B88800D4002000A7
:1011D000A4B88800E4002800B4B88800F400200017
:1011E000C4B8880004012800D4B888001401220083
:1011F000E4B8880024812900F4B888003401220072
:1012000004B9880044C1290014B9880054A1200001
:1012100024B988006421200034B98800742120009A
:1012200044B988008401220054B988009441200008
:1012300064B98800A441210074B98800B431270042
:1012400084B98800C4F12F0094B98800D4812700A4
:10125000A4B98800E4612B00B4B98800F4412900E6
:10126000C4B9880004F22000D4B988001402220016
:10127000E4B9880024222300F4B9880034622100F4
:1012800004BA88004442250014BA88005492200011
:1012900024BA88006402220034BA880074022D0047
:1012A00044BA880084F22B0054BA880094222000AB
:1012B00064BA8800A402280074BA8800B40220002E
:1012C00084BA8800C402200094BA8800D4822E0018
:1012D000A4BA8800E4022E00B4BA880014F02800F2
:1012E000C4BA880024D02000D4BA880034002B006F
:1012F000E4BA880044002C00F4BA88005420270087
:1013000004BB88006400240014BB8800749026008D
:1013100024BB880084002C0034BB88009470270014
:1013200044BB8800A400280054BB8800B4002000FF
:1013300064BB8800C400280074BB8800D40020006F
:1013400084BB8800E400280094BB8800F4002000DF
:10135000A4BB880004012800B4BB880044212000FD
:10136000C4BB880054A12000D4BB880064212000A5
:10137000E4BB880074212000F4BB880084012200B3
:1013800004BC880094D1200014BC8800A441210032
:1013900024BC8800B431270034BC8800C4F12F007D
:1013A00044BC8800D481270054BC8800E441280054
:1013B00064BC8800F461290074BC880004F2200039
:1013C00084BC88001402220094BC880024222300DC
:1013D000A4BC880034A22100B4BC8800444225008B
:1013E000C4BC880054922000D4BC8800640222004F
:1013F000E4BC880074022D00F4BC880084F22B0049
:1014000004BD88009422200014BD8800A402280096
:1014100024BD8800B402200034BD8800C40220002E
:1014200044BD8800D4822E0054BD8800E4022E0002
:1014300064BD8800AE37EF001400270084BD88002B
:101440002480200094BD880034002B00A4BD8800B7
:1014500044002C00B4BD880054202700C4BD88007F
:1014600064002400D4BD880074902600E4BD880088
:1014700084002C00F4BD88009470270004BE88000E
:10148000A400280014BE8800B400200024BE8800F8
:10149000C400280034BE8800D400200044BE880068
:1014A000E400280054BE8800F400200064BE8800D8
:1014B0000401280074BE88004421200084BE8800F6
:1014C00054A1200094BE880064212000A4BE88009E
:1014D00074212000B4BE880084012200C4BE8800AC
:1014E00094D12000D4BE8800A4412100E4BE88002D
:1014F000B4312700F4BE8800C4F12F0004BF880077
:10150000D481270014BF8800E441280024BF88004C
:10151000F461290034BF880004F2200044BF880031
:101520001402220054BF88002422230064BF8800D4
:1015300034A2210074BF88004442250084BF880083
:101540005492200094BF880064022200A4BF880047
:1015500074022D00B4BF880084F22B00C4BF880041
:1015600094222000D4BF8800A4022800E4BF880091
:10157000B4022000F4BF8800C402200004C0880028
:10158000D4822E0014C08800E4022E0024C08800FB
:101590000638EF001470280044C0880024002000A2
:1015A00054C0880034002F0064C0880044802700A5
:1015B00074C088005420270084C088006400240080
:1015C00094C0880074902600A4C0880084002C0079
:1015D000B4C0880094702700C4C08800A40028000C
:1015E000D4C08800B4002000E4C08800C4002800F3
:1015F000F4C08800D400200004C18800E400280062
:1016000014C18800F400200024C1880004012800CF
:1016100034C188004421200044C1880054A1200026
:1016200054C188006421200064C188007421200016
:1016300074C188008401220084C188009481200044
:1016400094C18800A4412100A4C18800B4312700BE
:10165000B4C18800C4F12F00C4C18800D481270020
:10166000D4C18800E4612B00E4C18800F441290062
:10167000F4C1880004F2200004C288001402220091
:1016800014C288002422230024C2880034A221002E
:1016900034C288004442250044C28800549220008D
:1016A00054C288006402220064C2880074022D00C3
:1016B00074C2880084F22B0084C288009422200027
:1016C00094C28800A4022800A4C28800B4022000AA
:1016D000B4C28800C4022000C4C28800D4822E0094
:1016E000D4C28800E4022E00E4C288005E38EF0015
:1016F0000460200004C388003480200014C38800E4
:10170000F408250024C388007492220034C38800A2
:101710001423210044C388002413280054C38800E4
:101720003443280064C388004403200074C3880045
:101730005403200084C3880064D3270094C3880026
:1017400074132A00A4C38800541E2400B4C3880064
:10175000644E2800C4C38800746E2000D4C388007F
:10176000449F2100E4C38800F4002200F4C38800F1
:101770000460200004C488003480200014C4880061
:10178000F408250024C488007492220034C4880020
:1017900014A3210044C488002413240054C48800E6
:1017A0003443280064C488004403200074C48800C3
:1017B0005423200084C488006403200094C488005B
:1017C00074132000A4C48800545E2200B4C48800AE
:1017D000644E2000C4C48800743E2600D4C488002F
:1017E000449F2100E4C48800F4002200F4C488006F
:1017F0000420200004C588003480200014C588001F
:10180000F408250024C588007492220034C588009D
:101810001423210044C588002413280054C58800DF
:101820003443280064C588004403200074C5880040
:101830005403200084C5880064D3270094C5880021
:1018400074132A00A4C58800541E2400B4C588005F
:10185000644E2800C4C58800746E2000D4C588007A
:10186000449F2100E4C58800F4002200F4C58800EC
:101870000420200004C688003480200014C688009C
:10188000F408250024C688007492220034C688001B
:1018900014A3210044C688002413240054C68800E1
:1018A0003443280064C688004403200074C68800BE
:1018B0005423200084C688006403200094C6880056
:1018C00074132000A4C68800545E2200B4C68800A9
:1018D000644E2000C4C68800743E2600D4C688002A
:1018E000449F2100E4C68800F4002200F4C688006A
:1018F000549B800067024200040078006FF3B70039
:101900006FD3BF003822F800E0FF9F003822F900B3
:10191000727502000000000020032000E6030200B0
:1019200000000000D10AAE002200370001002000B4
:101930000100780024020200000000008100E8009D
:10194000811F78003822F800E0FF9F003822F9005C
:101950003C77020000000000CF00780070002000FB
:101960000008E600F2FF3700509B800004002000D2
:101970008879020000000000C0118100A0C3B300FC
:10198000C01189003C77020000000000C0118100F6
:1019900000C2B300C01189003C77020000000000C3
:1019A000C011810000C2B300C01189003C77020061
:1019B00000000000549B80000960EF00B3AF2000DE
:1019C00084824100154078000160EF000080B20081
:1019D000250032001080B200670032003080B20073
:1019E000A90032001080B200EB0032007080B2001B
:1019F0002D0132001080B2006F0132003080B20041
:101A0000B10132001080B200F3013200F080B20068
:101A1000350232001080B200770232003080B2000E
:101A2000B90232001080B200FB0232007080B200B6
:101A30003D0332001080B2007F0332002080B200EC
:101A4000C1033200F081B200020432001080B20003
:101A5000430432003080B20084043200C081B200FE
:101A6000C5043200D5043700C011810020C4B30082
:101A7000C0118900C01181000080FD00F0C0B300DA
:101A80000080FD00C0118900D011810040C2B30068
:101A9000D0118900A26C0200000000006C33EF003E
:101AA000649B8000E30220000418E1001F00360060
:101AB000659B8000C12ADD000437210004804200BC
:101AC000749B800000429000749B8800659B80009E
:101AD000C12ADD00E18242000500780004372100C0
:101AE00004004000104078006FF3B700C01181007F
:101AF000A0C9B300C01189006ED3BF003822F8001E
:101B0000F0FF9F003822F9006FD3BF003A22F8009F
:101B1000E0FF9F003A22F900A26C020000000000E2
:101B20006C33EC00508D040000000000D10AAE00C0
:101B30000F00370001002000010078003E02020083
:101B4000000000008100E800811F78003822F800C2
:101B5000E0FF9F003822F9003C77020000000000FF
:101B6000CF007800200220000008E600F2FF3700D6
:101B70003897040000000000C011810020C4B300A9
:101B8000C0118900C01181000080FD00F0C0B300C9
:101B90000080FD00C0118900D011810040C2B30057
:101BA000D0118900A26C0200000000006C33EF002D
:101BB000649B8000E30220000418E1001F0036004F
:101BC000659B8000C12ADD00C43C210004804200E6
:101BD000749B800000429000749B8800659B80008D
:101BE000C12ADD00E182420005007800C43C2100EA
:101BF00004004000104078006FF3B700C01181006E
:101C0000A0C9B300C01189006ED3BF003822F8000C
:101C1000F0FF9F003822F9006FD3BF003A22F8008E
:101C2000E0FF9F003A22F900A26C020000000000D1
:101C30006C33EC00D88D040000000000D10AAE0027
:101C40000F00370001002000010078006E02020042
:101C5000000000008100E800811F78003822F800B1
:101C6000E0FF9F003822F9003C77020000000000EE
:101C7000CF007800F00120000008E600F2FF3700F6
:101C80003897040000000000C011810020C4B30098
:101C9000C0118900C01181000080FD00F0C0B300B8
:101CA0000080FD00C0118900D011810040C2B30046
:101CB000D0118900A26C0200000000006C33EF001C
:101CC000649B8000D30220000418E1001F0036004E
:101CD000659B8000C12ADD0084422100048042000F
:101CE000749B800000429000749B8800659B80007C
:101CF000C12ADD00E1824200050078008442210013
:101D000004004000104078006FF3B700C01181005C
:101D1000A0C9B300C01189006ED3BF003822F800FB
:101D2000F0FF9F003822F9006FD3BF003A22F8007D
:101D3000E0FF9F003A22F900A26C020000000000C0
:101D40006C33EC00608E040000000000D10AAE008D
:101D50000F00370001002000010078009C02020003
:101D6000000000008100E800811F78003822F800A0
:101D7000E0FF9F003822F9003C77020000000000DD
:101D8000CF007800200220000008E600F2FF3700B4
:101D90003897040000000000C011810020C4B30087
:101DA000C0118900C01181000080FD00F0C0B300A7
:101DB0000080FD00C0118900D011810040C2B30035
:101DC000D0118900A26C0200000000006C33EF000B
:101DD000649B8000D30220000418E1001F0036003D
:101DE000659B8000C12ADD00444821000480420038
:101DF000749B800000429000749B8800659B80006B
:101E0000C12ADD00E182420005007800444821003B
:101E100004004000104078006FF3B700C01181004B
:101E2000A0C9B300C01189006ED3BF003822F800EA
:101E3000F0FF9F003822F9006FD3BF003A22F8006C
:101E4000E0FF9F003A22F900A26C020000000000AF
:101E50006C33EC00E88E040000000000D10AAE00F4
:101E60000F0037000100200001007800CC020200C2
:101E7000000000008100E800811F78003822F8008F
:101E8000E0FF9F003822F9003C77020000000000CC
:101E9000CF007800F00120000008E600F2FF3700D4
:101EA0003897040000000000C011810020C4B30076
:101EB000C0118900C01181000080FD00F0C0B30096
:101EC0000080FD00C0118900D011810040C2B30024
:101ED000D0118900A26C0200000000006C33EF00FA
:101EE000649B8000D30220000418E1001F0036002C
:101EF000659B8000C12ADD00044E21000480420061
:101F0000749B800000429000749B8800659B800059
:101F1000C12ADD00E182420005007800044E210064
:101F200004004000104078006FF3B700C01181003A
:101F3000A0C9B300C01189006ED3BF003822F800D9
:101F4000F0FF9F003822F9006FD3BF003A22F8005B
:101F5000E0FF9F003A22F900A26C0200000000009E
:101F60006C33EC00708F040000000000D10AAE005A
:101F70000F0037000100200001007800FA02020083
:101F8000000000008100E800811F78003822F8007E
:101F9000E0FF9F003822F9003C77020000000000BB
:101FA000CF007800000220000008E600F2FF3700B2
:101FB0003897040000000000C011810020C4B30065
:101FC000C0118900C01181000080FD00F0C0B30085
:101FD0000080FD00C0118900D011810040C2B30013
:101FE000D0118900A26C0200000000006C33EF00E9
:101FF000649B8000D30220000418E1001F0036001B
:10200000659B8000C12ADD00C4532100048042008A
:10201000749B800000429000749B8800659B800048
:10202000C12ADD00E182420005007800C45321008E
:1020300004004000104078006FF3B700C011810029
:10204000A0C9B300C01189006ED3BF003822F800C8
:10205000F0FF9F003822F9006FD3BF003A22F8004A
:10206000E0FF9F003A22F900A26C0200000000008D
:102070006C33EC00F88F040000000000D10AAE00C1
:102080000F00370001002000010078002803020043
:10209000000000008100E800811F78003822F8006D
:1020A000E0FF9F003822F9003C77020000000000AA
:1020B000CF007800D00120000008E600F2FF3700D2
:1020C0003897040000000000C011810020C4B30054
:1020D000C0118900C01181000080FD00F0C0B30074
:1020E0000080FD00C0118900D011810040C2B30002
:1020F000D0118900A26C0200000000006C33EF00D8
:10210000649B8000B30220000418E1001F00360029
:10211000659B8000C12ADD008459210004804200B3
:10212000749B800000429000749B8800659B800037
:10213000C12ADD00E18242000500780084592100B7
:1021400004004000104078006FF3B700C011810018
:10215000A0C9B300C01189006ED3BF003822F800B7
:10216000F0FF9F003822F9006FD3BF003A22F80039
:10217000E0FF9F003A22F900A26C0200000000007C
:102180006C33EC008090040000000000D10AAE0027
:102190000F00370001002000010078005403020006
:1021A000000000008100E800811F78003822F8005C
:1021B000E0FF9F003822F9003C7702000000000099
:1021C000CF007800200220000008E600F2FF370070
:1021D0003897040000000000C011810020C4B30043
:1021E000C0118900C01181000080FD00F0C0B30063
:1021F0000080FD00C0118900D011810040C2B300F1
:10220000D0118900A26C0200000000006C33EF00C6
:10221000649B8000B30220000418E1001F00360018
:10222000659B8000C12ADD00045F2100048042001C
:10223000749B800000429000749B8800659B800026
:10224000C12ADD00E182420005007800045F210020
:1022500004004000104078006FF3B700C011810007
:10226000A0C9B300C01189006ED3BF003822F800A6
:10227000F0FF9F003822F9006FD3BF003A22F80028
:10228000E0FF9F003A22F900A26C0200000000006B
:102290006C33EC000891040000000000D10AAE008D
:1022A0000F003700010020000100780084030200C5
:1022B000000000008100E800811F78003822F8004B
:1022C000E0FF9F003822F9003C7702000000000088
:1022D000CF007800200220000008E600F2FF37005F
:1022E0003897040000000000C011810020C4B30032
:1022F000C0118900C01181000080FD00F0C0B30052
:102300000080FD00C0118900D011810040C2B300DF
:10231000D0118900A26C0200000000006C33EF00B5
:10232000649B8000B30220000418E1001F00360007
:10233000659B8000C12ADD00846421000480420086
:10234000749B800000429000749B8800659B800015
:10235000C12ADD00E182420005007800846421008A
:1023600004004000104078006FF3B700C0118100F6
:10237000A0C9B300C01189006ED3BF003822F80095
:10238000F0FF9F003822F9006FD3BF003A22F80017
:10239000E0FF9F003A22F900A26C0200000000005A
:1023A0006C33EC009091040000000000D10AAE00F4
:1023B0000F0037000100200001007800B403020084
:1023C000000000008100E800811F78003822F8003A
:1023D000E0FF9F003822F9003C7702000000000077
:1023E000CF007800300220000008E600F2FF37003E
:1023F0003897040000000000C011810020C4B30021
:10240000C0118900C01181000080FD00F0C0B30040
:102410000080FD00C0118900D011810040C2B300CE
:10242000D0118900A26C0200000000006C33EF00A4
:10243000649B8000D30220000418E1001F003600D6
:10244000659B8000C12ADD00046A210004804200EF
:10245000749B800000429000749B8800659B800004
:10246000C12ADD00E182420005007800046A2100F3
:1024700004004000104078006FF3B700C0118100E5
:10248000A0C9B300C01189006ED3BF003822F80084
:10249000F0FF9F003822F9006FD3BF003A22F80006
:1024A000E0FF9F003A22F900A26C02000000000049
:1024B0006C33EC001892040000000000D10AAE005A
:1024C0000F0037000100200001007800040C02001A
:1024D000000000008100E800811F78003822F80029
:1024E000E0FF9F003822F9003C7702000000000066
:1024F000CF007800300220000008E600F2FF37002D
:102500003897040000000000C011810020C4B3000F
:10251000C0118900C01181000080FD00F0C0B3002F
:102520000080FD00C0118900D011810040C2B300BD
:10253000D0118900A26C0200000000006C33EF0093
:10254000649B8000E30220000418E1001F003600B5
:10255000659B8000C12ADD00C46F21000480420019
:10256000749B800000429000749B8800659B8000F3
:10257000C12ADD00E182420005007800C46F21001D
:1025800004004000104078006FF3B700C0118100D4
:10259000A0C9B300C01189006ED3BF003822F80073
:1025A000F0FF9F003822F9006FD3BF003A22F800F5
:1025B000E0FF9F003A22F900A26C02000000000038
:1025C0006C33EC00A092040000000000D10AAE00C1
:1025D0000F0037000100200001007800360C0200D7
:1025E000000000008100E800811F78003822F80018
:1025F000E0FF9F003822F9003C7702000000000055
:10260000CF007800400220000008E600F2FF37000B
:102610003897040000000000C011810020C4B300FE
:10262000C0118900C01181000080FD00F0C0B3001E
:102630000080FD00C0118900D011810040C2B300AC
:10264000D0118900A26C0200000000006C33EF0082
:10265000649B8000B30220000418E1001F003600D4
:10266000659B8000C12ADD00847521000480420042
:10267000749B800000429000749B8800659B8000E2
:10268000C12ADD00E1824200050078008475210046
:1026900004004000104078006FF3B700C0118100C3
:1026A000A0C9B300C01189006ED3BF003822F80062
:1026B000F0FF9F003822F9006FD3BF003A22F800E4
:1026C000E0FF9F003A22F900A26C02000000000027
:1026D0006C33EC002893040000000000D10AAE0027
:1026E0000F0037000100200001007800680C020094
:1026F000000000008100E800811F78003822F80007
:10270000E0FF9F003822F9003C7702000000000043
:10271000CF007800300220000008E600F2FF37000A
:102720003897040000000000C011810020C4B300ED
:10273000C0118900C01181000080FD00F0C0B3000D
:102740000080FD00C0118900D011810040C2B3009B
:10275000D0118900A26C0200000000006C33EF0071
:10276000649B8000B30220000418E1001F003600C3
:10277000659B8000C12ADD00047B210004804200AB
:10278000749B800000429000749B8800659B8000D1
:10279000C12ADD00E182420005007800047B2100AF
:1027A00004004000104078006FF3B700C0118100B2
:1027B000A0C9B300C01189006ED3BF003822F80051
:1027C000F0FF9F003822F9006FD3BF003A22F800D3
:1027D000E0FF9F003A22F900A26C02000000000016
:1027E0006C33EC00B093040000000000D10AAE008E
:1027F0000F00370001002000010078009A0C020051
:10280000000000008100E800811F78003822F800F5
:10281000E0FF9F003822F9003C7702000000000032
:10282000CF007800400220000008E600F2FF3700E9
:102830003897040000000000C011810020C4B300DC
:10284000C0118900C01181000080FD00F0C0B300FC
:102850000080FD00C0118900D011810040C2B3008A
:10286000D0118900A26C0200000000006C33EF0060
:10287000649B8000B30220000418E1001F003600B2
:10288000659B8000C12ADD00848021000480420015
:10289000749B800000429000749B8800659B8000C0
:1028A000C12ADD00E1824200050078008480210019
:1028B00004004000104078006FF3B700C0118100A1
:1028C000A0C9B300C01189006ED3BF003822F80040
:1028D000F0FF9F003822F9006FD3BF003A22F800C2
:1028E000E0FF9F003A22F900A26C02000000000005
:1028F0006C33EC003894040000000000D10AAE00F4
:102900000F0037000100200001007800CC0C02000D
:10291000000000008100E800811F78003822F800E4
:10292000E0FF9F003822F9003C7702000000000021
:10293000CF007800400220000008E600F2FF3700D8
:102940003897040000000000C0118100A0C9B30046
:10295000C0118900C01181000080FD00E0C1B300FA
:102960000080FD00C0118900D0118100A0C0B3001B
:10297000D0118900A26C0200000000006C33EF004F
:10298000649B80007020E1001F003100659B800087
:10299000C12ADD000486210004804200749B80006F
:1029A00000429000749B8800659B8000C12ADD0076
:1029B000E182420005007800048621000400400006
:1029C000104078006FF3B700C011810020C4B3003D
:1029D000C01189006ED3BF003822F800F0FF9F00BD
:1029E0003822F9006FD3BF003A22F800E0FF9F00C1
:1029F0003A22F900A26C0200000000006C33EC00E7
:102A0000C094040000000000D10AAE000F0037009F
:102A10000100200001007800FE0C02000000000010
:102A20008100E800811F78003822F800E0FF9F0055
:102A30003822F9003C77020000000000CF00780047
:102A4000700220000008E600F2FF3700389704000B
:102A500000000000C0118100A0C9B300C0118900AE
:102A6000C01181000080FD00E0C1B3000080FD00C6
:102A7000C0118900D0118100A0C0B300D01189001D
:102A8000A26C0200000000006C33EF00649B800029
:102A90007020E1001F003100659B8000C12ADD002D
:102AA0000488210004804200749B80000042900052
:102AB000749B8800659B8000C12ADD00E182420092
:102AC00005007800048821000400400010407800D0
:102AD0006FF3B700C011810020C4B300C01189009A
:102AE0006ED3BF003822F800F0FF9F003822F900B3
:102AF0006FD3BF003A22F800E0FF9F003A22F900AE
:102B0000A26C0200000000006C33EC00469504004B
:102B100000000000D10AAE000F00370001002000C5
:102B200001007800340D0200000000008100E80080
:102B3000811F78003822F800E0FF9F003822F9005A
:102B40003C77020000000000CF0078006002200007
:102B50000008E600F2FF370038970400000000008C
:102B6000C0118100A0C9B300C0118900C01181004B
:102B70000080FD00E0C1B3000080FD00C0118900AD
:102B8000D0118100A0C0B300D0118900A26C020056
:102B9000000000006C33EF00649B80007020E100B7
:102BA0001F003100659B8000C12ADD00048A2100DE
:102BB00004804200749B800000429000749B880057
:102BC000659B8000C12ADD00E1824200050078009B
:102BD000048A210004004000104078006FF3B70021
:102BE000C011810020C4B300C01189006ED3BF00A2
:102BF0003822F800F0FF9F003822F9006FD3BF00A1
:102C00003A22F800E0FF9F003A22F900A26C02008D
:102C1000000000006C33EC00CC95040000000000C4
:102C2000D10AAE000F00370001002000010078003B
:102C3000680D0200000000008100E800811F78009C
:102C40003822F800E0FF9F003822F9003C770200AC
:102C500000000000CF007800A00220000008E6007D
:102C6000F2FF37003897040000000000C011810017
:102C7000A0C9B300C0118900C01181000080FD000F
:102C8000E0C1B3000080FD00C0118900D0118100B7
:102C9000A0C0B300D0118900A26C020000000000A7
:102CA0006C33EF00649B80007020E1001F00310056
:102CB000659B8000C12ADD00048C21000480420055
:102CC000749B800000429000749B8800659B80008C
:102CD000C12ADD00E182420005007800048C210059
:102CE00004004000104078006FF3B700C01181006D
:102CF00020C4B300C01189006ED3BF003822F80091
:102D0000F0FF9F003822F9006FD3BF003A22F8008D
:102D1000E0FF9F003A22F900A26C020000000000D0
:102D20006C33EC005296040000000000D10AAE00A3
:102D30000F0037000100200001007800A20D020002
:102D4000000000008100E800811F78003822F800B0
:102D5000E0FF9F003822F9003C77020000000000ED
:102D6000CF007800800220000008E600F2FF370064
:102D70003897040000000000D10AAE000F003700B1
:102D80000100200001007800DA0D020000000000C0
:102D90008100E800811F78003822F800E0FF9F00E2
:102DA0003822F9003C77020000000000CF007800D4
:102DB000200220000008E600F2FF3700C011810069
:102DC000A0C9B300C0118900C01181000080FD00BE
:102DD000E0C1B3000080FD00C0118900D011810066
:102DE000A0C0B300D0118900A26C02000000000056
:102DF000C011810020C4B300C0118900C01181003E
:102E00000080FD00F0C0B3000080FD00C01189000B
:102E1000D011810040C2B300D0118900A26C020021
:102E200000000000D10AAE000F00370001002000B2
:102E3000010078000A0E0200000000008100E80096
:102E4000811F78003822F800E0FF9F003822F90047
:102E50003C77020000000000CF00780080002000D6
:102E60000008E600F2FF3700389704000000000079
:102E7000CF02780000000600851F78006833EF005D
:102E8000A27502000000000014002000449B88008E
:102E9000449B80006720E100070031006813F800C0
:102EA0006A13F900A6810200000000006833EC00FC
:102EB0004897040000000000D10AAE000F00370060
:102EC0000100200001007800000202000000000064
:102ED0008100E800811F78003822F800E0FF9F00A1
:102EE0003822F9003C77020000000000CF00780093
:102EF000600120000008E600F2FF3700CF027800F2
:102F000000000600851F78006833EF006A33EF0089
:102F10006C73EF006D73EF006E73EF0034102900D7
:102F2000849B880044002000949B8800540020006B
:102F3000A49B880064002000B49B880074002000DB
:102F4000C49B880084002000D49B8800940020004B
:102F5000E49B8800A4002000F49B8800B4002000BB
:102F6000049C8800C4002000149C8800D400200029
:102F7000249C8800E4002000349C8800F400200099
:102F8000449C880004012000549C88001401200007
:102F9000649C880024012000749C88003401200077
:102FA000849C880044012000949C880054012000E7
:102FB000A49C880064012000B49C88007401200057
:102FC000C49C880084012000D49C88009431200097
:102FD000E49C8800A4012000F49C8800B401200037
